:020000040800F2
:10800000D8CB0020698F0008198300081B83000863
:108010001D8300081F830008218300080000000062
:10802000000000000000000000000000598200086D
:1080300025830008000000008D820008797C01087B
:10804000838F0008838F0008838F0008838F0008C8
:10805000838F0008838F0008838F0008838F0008B8
:10806000838F0008838F0008838F0008838F0008A8
:10807000838F0008838F0008838F0008838F000898
:10808000838F0008838F0008838F0008838F000888
:10809000838F0008838F0008838F0008838F000878
:1080A000838F0008838F0008838F0008838F000868
:1080B000838F0008838F0008838F0008838F000858
:1080C000838F0008838F0008838F0008838F000848
:1080D000838F0008CB800108838F00084F8301083D
:1080E000838F0008838F0008838F0008838F000828
:1080F000838F0008838F0008838F0008838F000818
:10810000838F0008838F0008838F0008838F000807
:10811000E7820108838F0008DD380108838F00089B
:10812000838F0008838F0008838F0008838F0008E7
:1081300000F002F800F080F80AA090E8000C8244F9
:108140008344AAF10107DA4501D100F075F8AFF2D6
:10815000090EBAE80F0013F0010F18BFFB1A43F025
:1081600001031847F8620300186303000A444FF044
:10817000000C10F8013B13F0070408BF10F8014B86
:108180001D1108BF10F8015B641E05D010F8016BCB
:10819000641E01F8016BF9D113F0080F1EBF10F82F
:1081A000014BAD1C0C1B09D16D1E58BF01F801CB52
:1081B000FAD505E014F8016B01F8016B6D1EF9D5D5
:1081C0009142D6D3704700000023002400250026EA
:1081D000103A28BF78C1FBD8520728BF30C148BF2A
:1081E0000B607047642921F0AB85732922F0198157
:1081F0000020704710B510BD70477047704770473A
:1082000054656D636F54535441543800000000614D
:10821000000000671FB521F01AFF22F0EFF90400FB
:108220000020002123F0A8FF401C606000200021F6
:1082300023F0B8FFE0601FBD22F0A8FB1146FFF756
:10824000E9FF02F0F0FA22F019FE03B4FFF7D2FFC3
:1082500003BC0FF0A1FD00001A4B19680868B0E8D4
:10826000F00F80F309884FF0000080F311884EF082
:108270000D0E70470000000003480068006880F39E
:10828000088862B600DF00BF08ED00E0EFF3098068
:108290000C4B1A6820E9F00F106008B54FF0BF00D2
:1082A00080F311880FF0ABFA4FF0000080F31188D3
:1082B000BDE8084019680868B0E8F00F80F3098845
:1082C000704700BFB002002001B44FF0BF0080F340
:1082D000118801BC704701B44FF0000080F3118891
:1082E00001BC70470B49D1F800C04A685CF8043BF8
:1082F0001068184442F8040B8C4528BFA1F1DC0C2F
:108300008A4228BFA1F1DC02C1F800C04A6020F017
:108310000040704770C500207047FEE7FEE7FEE7AB
:10832000FEE7704770477047704700000CB50022A9
:10833000019200925248016841F4803101604FF48B
:10834000A063016801F4003100910199491C019179
:10835000009911B901999942F3D10168890302D5B5
:108360000121009100E000920099012930D1454996
:108370000A6842F010020A600A6822F003020A60EA
:108380000A6842F002020A60416841604168416047
:10839000416841F480614160416821F47C11416091
:1083A000416841F4E8114160016841F08071016069
:1083B00001688901FCD5416821F0030141604168F1
:1083C00041F0020141604168C1F381010229FAD103
:1083D0000CBDABE710B52A48016841F0010101600E
:1083E0004168294A114041600168284A11400160F2
:1083F000016821F480210160416821F4FE0141609F
:108400004FF41F018160FFF7E4FF21494FF0006046
:10841000086010BD10B51A4A506800F00C011D4BE1
:108420001D4800290ED004290ED008290ED0036063
:108430005168194AC1F30311121D515C0268CA4008
:10844000026010BD0360F3E70360F1E7516801F4D7
:108450007011536803F48033022404EB914133B16B
:1084600053689B0307D50D4B59430160E0E70B4B65
:1084700059430160DCE7074B59430160D8E700002E
:1084800000100240002002400000FFF8FFFFF6FE4F
:1084900008ED00E000127A001400002000093D0001
:1084A0009A48994941609A494160704797480169E3
:1084B00041F08001016170479448C068C10701D054
:1084C00001207047410701D502207047C00601D541
:1084D000032070470020704770B50446FFF7ECFF9B
:1084E0000546012D05D10FF08BFD641EA4B2002CB2
:1084F000F4D104B9FF25284670BD70B5054645F690
:10850000FF763046FFF7E8FF002812D17F4C206944
:1085100040F0020020616561206940F04000206168
:108520003046FFF7D9FF012803D0216921F002016D
:10853000216170BD70B506460D46FF20FFF7CCFFE8
:1085400000280ED1714C206940F001002061358077
:10855000FF20FFF7C1FF012803D0216921F00101AD
:10856000216170BD008870472DE9F04105460E4637
:108570001746002407E036F814102846FFF7DAFF04
:10858000AD1C641CA4B2BC42F5D3BDE8F081C107A8
:1085900003D030F8010C000A70470088C0B2704761
:1085A00010B50446002307E02046FFF7DBFF21F863
:1085B0001300A41C5B1C9BB29342F5D310BD2DE9A4
:1085C000F05F82460F461546AAF10062B2F5002F11
:1085D00052D2FFF765FF4FEAD228C2F34906C6F52B
:1085E0008064A54200D82C46DFF828B137E0321865
:1085F0003BF812208A4203D1401C80B2A042F6D33D
:10860000A04214D24846FFF778FF002006E0821906
:1086100037F810102BF81210401C80B2A042F6D38D
:1086200048464FF480623B49FFF79EFF04E0224634
:1086300039465046FFF798FFA54202D1BDE8F05FEA
:1086400034E708F10108002607EB44070AEB440A67
:10865000281B85B24FF48064A54200D82C464FF009
:10866000006000EBC82942142A494846FFF798FFEA
:1086700000204FF6FF71C1E7BDE8F09F30B504461A
:108680000D46002306E02046FFF781FFE854641CF6
:108690005B1C9BB29342F6D330BD70472DE9F04787
:1086A000ADF5006D0D46904600240746A0F1006030
:1086B000B0F5002F23D200264FF48069EA4615E07A
:1086C0006878000215F8021B08442146641CA4B215
:1086D0002AF811004A46944206D1002469463846D9
:1086E000FFF742FF07F50067B61CB6B24645E7D371
:1086F000002C04D0224669463846FFF735FF0DF5B9
:10870000006DBDE8F08700002301674500200240AE
:10871000AB89EFCD680900202A4908432A4908603F
:10872000704770B50F23C27801260178002A1ED049
:10873000254A126802F4E062C2F5E062120AC2F150
:108740000404D3404578A54082781A402A43120198
:1087500001F1E02181F80024007800F01F018E4033
:108760004009800000F1E020C0F8006170BD01F018
:108770001F0086404809800000F1E020C0F88061B9
:1087800070BD124A114001430F48001F016070473D
:108790000D4A121D002903D0116801431160704772
:1087A00011688143116070474FF0E021042804D024
:1087B000086920F0040008617047086940F004006F
:1087C000086170470000FA050CED00E080FFFF1F14
:1087D00010B5DB4988420AD144150121204607F033
:1087E0005AFB2046BDE81040002107F054BBD54994
:1087F00088420AD104150121204607F04CFB20468F
:10880000BDE81040002107F046BBCF4988420AD19D
:108810000121CC03204607F03EFB2046BDE8104076
:10882000002107F038BB10BD10B54268C74B1A4095
:108830000C790B6842EA0422134343608268C44BFC
:108840001A40D1E9024323434C7942EA44021343DC
:108850008360C26A22F47002097C491EC9B242EAEE
:108860000151C16210BD002101600171417181603F
:10887000C160012101747047002904D0816841F072
:10888000010181607047816821F0010181607047BA
:10889000002904D0816841F480718160704781684B
:1088A00021F4807181607047C9B2002A03D0426808
:1088B0000A434260704742688A4342607047816859
:1088C00041F008018160704701460020896809076E
:1088D00000D501207047816841F004018160704734
:1088E000014600208968490700D50120704700290A
:1088F00004D0816841F4A00181607047816821F44F
:10890000A00181607047014600208968490200D5B6
:1089100001207047426822F46042491E42EA413118
:1089200041607047002904D0416841F40061416012
:108930007047416821F400614160704770B50726B7
:1089400009290AD9C568A1F10A0404EB4404A64028
:10895000B543A3401D43C56007E0056901EB410431
:10896000A640B543A3401D4305611F23072A09D232
:10897000446B521E02EB820293409C4391400C4395
:10898000446370BD0D2A09D2046BD21F02EB820230
:1089900093409C4391400C43046370BDC46A0D3AFC
:1089A00002EB820293409C4391400C43C46270BD31
:1089B000002904D0816841F480118160704781688A
:1089C00021F4801181607047C06C80B270475C48B0
:1089D0004C3000687047002904D0416841F4806140
:1089E00041607047416821F480614160704700290F
:1089F00004D0416841F4805141607047416821F4DE
:108A0000805141607047826822F4E0420A438260EC
:108A10007047002904D0816841F4004181607047AB
:108A2000816821F4004181607047002904D0816889
:108A300041F4021181607047816821F40211816064
:108A40007047014600208968890200D501207047DF
:108A500070B5072609290AD9C568A1F10A0404EBF3
:108A60004404A640B543A3401D43C56007E0056923
:108A700001EB4104A640B543A3401D430561836B50
:108A8000C3F30154121B921C02EB82021F24944078
:108A9000A34391400B43836370BD826B22F4401269
:108AA000491E42EA01518163704708B50090009861
:108AB000084400900098026008BD08B50090009836
:108AC0000844283000900098006880B208BD4268D1
:108AD000204B1A400A4342607047416282627047ED
:108AE000426822F01F020A4342607047144908316D
:108AF000002804D0086840F4000008607047086847
:108B000020F40000086070470246002012680A4204
:108B100000D001207047C9430160704710B502467C
:108B200000200B0A5468C9B20C401168194202D0E7
:108B3000002C00D0012010BD090AC9430160704714
:108B40000024014000280140003C0140FFFEF0FFEE
:108B5000FDF7F1FFFFFD3FFF10B59C49884209D1A9
:108B60000121042007F097F90021BDE810400420FE
:108B700007F091B99649884209D10121082007F0F0
:108B80008AF90021BDE81040082007F084B9914916
:108B9000884209D10121102007F07DF90021BDE8AC
:108BA0001040102007F077B98B49884209D1012184
:108BB000202007F070F90021BDE81040202007F0C8
:108BC0006AB98649884209D10121402007F063F93A
:108BD0000021BDE81040402007F05DB9804988427F
:108BE00009D10121802007F056F90021BDE810408D
:108BF000802007F050B97B4988420AD184150121B1
:108C0000204607F048F92046BDE81040002107F053
:108C100042B910BD10B50121084607F03CF900210A
:108C2000BDE81040012007F036B92DE9F0410022DF
:108C3000CC7804F00F03E40601D58C7823430C783C
:108C40004FF00F0714F0FF0F4FF0010C1CD0056818
:108C50000CFA02F40E882640A64211D1960007FABB
:108C600006F825EA080503FA06F848EA0505CE786D
:108C7000282E02D0482E02D002E0446100E00461B8
:108C8000521C082AE4D305600A88FF2A1ED94568C9
:108C9000002202F108060CFA06F40E882640A642CD
:108CA00010D1960007FA06F825EA080503FA06F837
:108CB00048EA0505CE78282E00D14461CE78482EAA
:108CC00000D10461521C082AE3D34560BDE8F0815D
:108CD0004FF6FF710180022181700421C17070473D
:108CE0000246002092680A4200D001207047806846
:108CF00080B2704702460020D2680A4200D00120AC
:108D00007047C06880B27047016170474161704729
:108D1000002A01D00161704741617047C16070470E
:108D200041F480328261816182618169806970472A
:108D300010B52D4B1A684FF68074224042EA00109D
:108D40000843186010BD2949C8617047F0B5264C2A
:108D5000002801DAE36900E06368C0F30346420DCE
:108D6000120185B2C0F301579540032F07D0C2020C
:108D70000CD50322B240934343F0706209E023F024
:108D80007062636823F07063636002E0AB4343F09A
:108D9000706201B12A43002801DAE261F0BD62602D
:108DA000F0BD10B58A07120F0F23934021F0030482
:108DB0000D4921448C689C438C608B689040034330
:108DC0008B6010BD0949DC31086070470008014024
:108DD000000C014000100140001401400018014047
:108DE000001C014000200140000001400000204222
:108DF0000D49086070470C49486070470A4988600F
:108E0000704709494AF6AA200860704706494CF69F
:108E1000CC400860704701460020034AD2680A42ED
:108E200000D0012070470000003000404D4A00296A
:108E300003D011880143118070471188814311804C
:108E400070474848001D018841F0100101807047BB
:108E50004448001D018821F01001018070474148FD
:108E60001C3000883F491831098840EA01407047AA
:108E700000B50246FFF7E5FF3A49100C18310880AB
:108E8000081D02805DF804EBE2E700B50246FFF73B
:108E9000D8FF3449C2F3034008310880081D02801E
:108EA0005DF804EBD4E700B50246FFF7CAFF2D4991
:108EB000100C20310880081D02805DF804EBC7E724
:108EC0002848103000880007010B2648143000881D
:108ED0000843704770B50024224D2D1D06E0641C28
:108EE000E4B264200FF0ACF81E2C02D8288880066B
:108EF000F5D570BD70B500241A4D2D1D288820F0C1
:108F00000800288006E0641CE4B264200FF098F8A2
:108F10001E2C02D828880007F5D570BD0146002018
:108F2000104A121D12880A4200D0012070470D49D4
:108F3000091D0A8882430A8070470A49091D098869
:108F4000C2B21140074A1288024202D009B1012080
:108F50007047002070470349091D0A8882430A8030
:108F60007047000000280040094880470948004732
:108F7000FEE7FEE7FEE7FEE7FEE7FEE7FEE7FEE7C9
:108F8000FEE7FEE704480549054A064B7047000026
:108F9000D583000831810008D8C50020D8CB002037
:108FA000D8C70020D8C700207CB5002201920092CB
:108FB0006B4601AA1EF079FC0B4D012490B1401CB8
:108FC0000FD019F0FDFA0199884202DB009A904215
:108FD00006DDB1F5800F04D204490098884200D321
:108FE0002C707CBD2C707CBD6C060020FFFF3F0008
:108FF00002F0FF0343EA032242EA024221F0FEB8F4
:109000000000000000000000000000000000000060
:109010000000000000000000000000000000000050
:10902000F74A01211160F749087001200FF03EBA9C
:1090300010B5F5480124047019F0BEFAF348C06871
:1090400019F0C1FAF24902200870F248047010BD0C
:10905000012080F31388F0480168F04A01F4E061D0
:1090600011430160BFF3408FFEE7F0B587B00121E7
:10907000202006F0FAFE0121042006F0F6FE012170
:10908000102006F0F2FE0121082006F0EEFE01217C
:10909000402006F0EAFEE24810250224007AE14E64
:1090A00004280BD34020ADF818008DF81B508DF824
:1090B0001A4006A9DC48FFF7B8FD0AE00420ADF825
:1090C00018008DF81B508DF81A4006A93046FFF79E
:1090D000ACFD4FF40040ADF814008DF817508DF83A
:1090E0001640374605A93846FFF79FFDADF81040FA
:1090F0008DF813508DF8124004A93846FFF795FDFE
:109100000820ADF80C008DF80F508DF80E4003A923
:109110003846FFF78AFD0126ADF808608DF80B5040
:109120008DF80A4002A93846FFF77FFDADF80460CC
:109130008DF807508DF8064001A9BC48FFF775FD72
:1091400007B0F0BD10B545F25550FFF751FE0520B0
:10915000FFF751FE4FF47A60FFF750FEFFF756FE1F
:10916000BDE81040FFF74DBEFFF74BBE2DE9F84FAD
:1091700040F2053008F0FBFAAD49087040F2F625E0
:10918000284608F0F4FA6C1EFF2807D10021284673
:1091900008F0EEFA6421204608F0EAFA204608F0CA
:1091A000E6FA0446284608F0E2FAA24904EB002059
:1091B00008809B4F012697F8F302012806D987F80B
:1091C000F362012140F2F32008F0D2FA9A495E20BE
:1091D00008800021942008F0CBFA40F2D32008F058
:1091E000C6FA04464FF4357008F0C1FA934904EB0F
:1091F00000200881072008F0BAFAFF2804D00820D0
:1092000008F0B5FAFF2803D10921072008F0B0FAC9
:1092100040F2625008F0ABFA89490870787900256D
:10922000FF282ED102F088FA0021052008F0A0FACC
:109230006121042008F09CFA01F041FD87F8DA5022
:10924000787A00F03F017972092008F091FA002441
:10925000002104F5A17008F08BFA641CE4B2072C1D
:10926000F6D30024002104F2491008F081FA641CAE
:10927000E4B2072CF6D397F86E00012801D987F8DD
:109280006E5040F29C44204608F071FA6D49087017
:109290004FF0FE0AFF2801D0012805D881F800A070
:1092A0005146204608F064FA97F85902FF2808D181
:1092B00097F85A02FF2804D1C82087F8590287F886
:1092C0005A5297F87800DFF8808138B104210128DC
:1092D00012D0022820D003282AD124E0294687F87A
:1092E0009B509B2008F044FA314688F8006040F219
:1092F000673008F03DFA1BE097F89B0020B987F82B
:109300009B109B2008F034FA294688F8005040F260
:10931000673008F02DFA0BE040F2673008F027FACA
:1093200088F8000004E087F89B109B2008F020FAE2
:1093300046480570464997F89B00087045490870F3
:1093400008B145480670DFF8149199F8000016F04E
:1093500098FA4349088099F800204249424832B1BE
:1093600097F86C200A8097F86D10018005E097F857
:1093700071200A8097F8701001804FF0000B0024D4
:1093800004F1B900009008F0F2F930B1009808F04B
:10939000EEF9032801D24FF0010B641CE4B2052C56
:1093A000EED33248BBF1010F05D0057097F8CC0021
:1093B0002F4910B10AE00670F8E797F8CB0028B9FA
:1093C00097F8CE0010B997F8CD00C0B129480570C4
:1093D00017F8CD0F7A7800EB0220274A80B2108070
:1093E000BA7BCD3F032A05D00E7097F8D310012227
:1093F00004F01CFEB879FF2843D0F8B351E03EE0FA
:10940000A00121420E6900206C060020000000200F
:1094100072060020700600200CED00E00400FA0542
:109420001C6D002000140140000C014000080140A8
:10943000C303002064000020480000200412002024
:10944000D50300204C0400207B000020C203002034
:109450006E0000203B000020680000203A00002041
:1094600054000020C4030020C60300207800002020
:109470007E0000208C0000209600002001E00D708E
:10948000B8E787F806A087F8F352FE48A0F800A0D6
:1094900001460122FC48FFF792F8B979062008F04E
:1094A00067F94FF42E7B584608F061F987F8B80247
:1094B0000C2805D987F8B8520021584608F058F909
:1094C00097F8D902012806D987F8D952002140F22D
:1094D000D92008F04DF997F8DC02012806D987F861
:1094E000DC5200214FF4377008F042F900244FF0AD
:1094F000030A381990F8F710FF2906D180F8F7A071
:10950000032104F1F70008F033F9641CE4B2082CDD
:10951000EFD397F8B802192805D987F8B852002177
:10952000584608F025F9012008E0391891F8BA22C8
:10953000FF2A01D181F8BA52401CC0B297F8B81284
:10954000491C8142F1D8D1490D8097F80201FF28CA
:1095500003D197F80121FF2A05D02843000297F88C
:10956000012102430A801B2008F001F904461C2057
:1095700008F0FDF804EB002A2F2008F0F8F8044664
:10958000302008F0F4F804EB0020C14C824501D2F1
:10959000267000E02570312008F0E9F8824632207C
:1095A00008F0E5F80AEB002B452008F0E0F88246C9
:1095B000462008F0DCF80AEB0020834501D26670F3
:1095C00000E0657040F2673008F0D1F888F80000DC
:1095D000012801D988F8006097F86103B8B997F8B5
:1095E000E10097F87E10884203D397F87D108842F7
:1095F0000DD9C8203C4687F8E100C821E12008F0D9
:10960000B7F894F8591294F85A0216F042F9F62075
:1096100008F0ADF887F8F6009E48017841F00701A0
:1096200001709D48007810B3787A40F0010078729C
:1096300089F80060787A00F0FB017972092008F05F
:1096400097F87B2020F0EEFC40F25324204608F0EF
:109650008EF8022803D90021204608F089F840F24C
:10966000EF24204608F083F8FF2807D00AE0787A34
:1096700000F0FE00787289F80050DBE700212046F8
:1096800008F076F808F0C0F884488088002806D1F1
:10969000BDE8F84F40F2E171842001F0D1BEBDE891
:1096A000F88F10B501210D2006F0DFFBBDE810405A
:1096B00001217B48FFF74ABB7A4DDFF8EC91DFF8D8
:1096C000EC817B4EDFF8ECA1DFF8ECB17B4F00249E
:1096D0007C71B8F800207979CA40D00702D0685C64
:1096E000401C6854685C06280FD36C5419F80100BC
:1096F00010B1401E09F8010019F8010028B9D0077F
:1097000003D00022694801F052FA7879401CC0B2B7
:1097100078710328DDD37C71BBF800207979CA40C9
:10972000D00702D0705C401C7054705C06280FD3C8
:1097300074541AF8010010B1401E0AF801001AF81A
:10974000010028B9D00703D000225B4801F02FFAAE
:109750007879401CC0B278710328DDD342F21070D2
:109760000EF06EFCB4E786B0FFF762FC002019F043
:10977000F5FB00201AF074FA514814F00AFF514921
:109780001420087050490B200870504902200870BE
:109790004F49052008704F4C4F4E002520780C286B
:1097A00002D1FFF745FC25702078132808D1FFF778
:1097B0003FFC002019F0D2FB00201AF051FA25706E
:1097C00096F82B0078B9757100234FF4167243494F
:1097D00001A8009518F0C7FE024622B100233F49B8
:1097E00001A81AF00DFA05200EF02AFCD6E7002693
:1097F0003B48012404703B4F97F8D800002804D060
:10980000C0EB0010810038480180DFF878B00025F7
:10981000DFF8D880FFF7A8FC3549087808B1401E6A
:109820000870087808B933480570DFF8A89099F8EF
:1098300000000D280BD13878ABF800007878ABF831
:109840000200114802220F491030FEF7B8FE99F8C5
:1098500000000E280BD1B878ABF80000F878ABF810
:1098600002000948022207492030FEF7A8FE224ADA
:109870001078012803D121490878401C08701F483E
:1098800001783DE0500000200077000874020020BD
:1098900078020020390000203B00002068110020E1
:1098A00000043000D50000209E000020860000202B
:1098B000D20000209B000020880000200000002033
:1098C000647000206C0400206A0400206B040020F7
:1098D0006D0400201303002050160020CC06002049
:1098E000280000201C6D00205C0000207211002068
:1098F0000D0300200C030020170300201803002094
:10990000052901D915700570FE490878012806D18E
:10991000887918B1CD71401E887100E0CC71FA4988
:109920000878012806D1887918B1CD71401E887158
:1099300000E0CC71F5490878012806D1887918B182
:10994000CD71401E887100E0CC71F1490878012882
:1099500006D1887918B1CD71401E887100E0CC71B4
:10996000EC490878012806D1887918B1CD71401EDC
:10997000887100E0CC7197F8D80050B1E6490888AA
:1099800008B1401E0880E54809880278114300D1DB
:109990000470761CF6B23C2E07D397F85C0318B11E
:1099A000DF480178491E01700026DD48007830B993
:1099B00097F85C0318B187F85C53DA48847099F81B
:1099C0000000102803D189F8005001F0B5FE99F885
:1099D0000000112809D003F020FFD3490880DFF8E8
:1099E0004CA3DAF80000B8B121E0D1480570142486
:1099F0004FF45A7640F26C75B44205D0652C03D012
:109A0000FF21204607F0B4FE641CA4B2AC42F3D39D
:109A100001F092FEFFF71CFB97F8B90238B104F091
:109A200005F888F8044088F8024088F80140C14AE7
:109A3000107801280CD1C0490878401CC0B20870C9
:109A4000052805D115700D7002F04CFFB5488470E3
:109A5000DAF8000098B197F8631081B1401ECAF897
:109A6000000060B99B2007F082FEB449087087F8B7
:109A70009B00B349087088F80240AA484570B14974
:109A80000888012801D9401E0880AF49088808B11C
:109A9000401E0880088838B997F8ED00FF2803D0E9
:109AA0000121AA48FFF732F997F8ED00FF2803D10A
:109AB0000121A648FFF728F9A549087818B188F8C8
:109AC0000140401E0870A349087818B188F8024088
:109AD000401E0870087858B99F480470DFF87CA2CF
:109AE0009AF80000012801D102F051FB8AF80050D9
:109AF0009B49087818B1401E087088F803409949BE
:109B0000087808B1401E0870087878B9964801783E
:109B100001290BD105700F2089F8000088F8014059
:109B200088F8024088F805409048057090490888F8
:109B3000401E80B2088008B98E480470DFF8389261
:109B400099F8000010B1401E89F8000099F8000053
:109B500020B900220121894801F029F899F8010073
:109B600010B1401E89F8010099F8010020B90022C7
:109B70000321824801F01BF899F8020010B1401E41
:109B800089F8020099F8020020B9002205217B48DB
:109B900001F00DF899F8030010B1401E89F8030098
:109BA00099F8030020B900220721744800F0FFFF54
:109BB00099F8040010B1401E89F8040099F80400D7
:109BC00020B9002209216D4800F0F1FF99F8050045
:109BD00010B1401E89F8050099F8050020B900224F
:109BE0000B21664800F0E3FF99F8060010B1401E13
:109BF00089F8060099F8060020B900220D215F4877
:109C000000F0D5FF4FF47A700EF01AFA02E60EB5A6
:109C1000DFF86CB101278BF800708BF801708BF8BE
:109C200002708BF803708BF804708BF806700121BA
:109C30004648FFF769F85449524808603F480178A0
:109C40003F4801704FF6FF76ED21CDE9001647F64B
:109C50001760002302901A462421F02008F0A0F992
:109C600047F61965CDE9016538200E210090C8231B
:109C7000464A084608F078F96921662009F0EEF8AE
:109C80009421662009F0EAF8BF21662009F0E6F881
:109C9000CDE900653EA36C220A21012008F04AF9B3
:109CA000CDE900653BA397220A21012008F042F983
:109CB000CDE9006538A3C2220A21012008F03AF953
:109CC0000024DFF8609099F80600401CC0B289F8C3
:109CD0000600052801D989F80640DFF8548098F875
:109CE000000001287ED002287DD004287CD00528E1
:109CF0007BD00728FCD0062878D00828FCD009287B
:109D000075D04BE086110020901100209A110020A0
:109D1000AE110020A41100205C0000205A00002099
:109D20001203002000000020440000204C0000200E
:109D30001303002069000020660000203B00002083
:109D40002C000020240300203E00002000080140D9
:109D500030000020310000206A0000202D0000208B
:109D600032000020EE000020EF000020F000002074
:109D700060000020620000209C0200209A02002067
:109D800072110020080100200401002064CA0308A9
:109D90005345540046414E00535953000B2876D08A
:109DA0000F2875D0FE490878002872D0002008706E
:109DB000FC49097801296DD099F80200C8B308F070
:109DC0009AFE8BF801708BF802708BF803708BF899
:109DD00004706921662009F041F89421662009F099
:109DE0003DF805E032E040E055E0C5E0D1E0DDE0DF
:109DF000BF21662009F032F8AFF26C03CDE90065AF
:109E00006C220A21012008F095F8AFF27803CDE921
:109E1000006597220A21012008F08CF8AFF2880330
:109E2000CDE90065C2220A21012008F083F889F8F3
:109E30000240DD490878002871D000200870DB4816
:109E4000077099F8060005286AD030E1284607F027
:109E5000B6FECDE900651E22D5A31146012008F00B
:109E600069F80EF00DF9FFF7F3F888F8004028467E
:109E700007F0A5FECDE900651E22D0A31146012002
:109E800008F058F801F058FC02F02AFD55E2D3E042
:109E9000D7E0F4E0F5E088F80040CA4890F86500A3
:109EA00001280FD0B8B102281ED0032825D00428DD
:109EB0002CD0052835D006283CD0072843D00828C8
:109EC0004AD051E04FF4964840460DF075FFBE4829
:109ED000C0F8088048E04FF4165840460DF06CFF7B
:109EE000B948C0F808803FE04FF4164840460DF0EE
:109EF00063FFB548C0F8088036E04FF4614840463B
:109F00000DF05AFFB048C0F808802DE04FF4E1385A
:109F100040460DF051FFAC48C0F8088024E0BDE099
:109F2000BEE04FF4963840460DF046FFA648C0F814
:109F3000088019E04FF4966840460DF03DFFA248B6
:109F4000C0F8088010E04FF4965840460DF034FFFA
:109F50009D48C0F8088007E04FF4615840460DF076
:109F60002BFF9948C0F80880974890F82B000328E9
:109F70008CD10EF085F8E0E194480088C1B2C0F3BE
:109F8000072015F02CFD002001F0EAFF88F80040C2
:109F9000D3E18E480088C1B2C0F3072015F079FCE8
:109FA000012001F0DDFF88F80040C6E188F800409C
:109FB000844890F8821001293BD090F86500092868
:109FC00033D2DFE800F0050A0F14191E23282D00F4
:109FD0004FF416500DF0F0FE2BE04FF496400DF0CC
:109FE000EBFE26E04FF416400DF0E6FE21E04FF4C4
:109FF00061400DF0E1FE1CE04FF4E1300DF0DCFEBD
:10A0000017E04FF496300DF0D7FE12E04FF4966053
:10A010000DF0D2FE0DE04FF496500DF0CDFE08E0AD
:10A020004FF461500DF0C8FE03E04FF496400DF080
:10A03000C3FE0EF025F880E115F01DF888F8004009
:10A040007BE1AFF2B423CDE900656C220A21012047
:10A0500007F070FFAFF2C423CDE9006597220A2113
:10A06000012007F067FFAFF2D023CDE90065C222DF
:10A070000A21012007F05EFF88F800405DE1012021
:10A0800095E640B95248008884380F2803D302204F
:10A0900008F012FD4DE103F018F84AE10120CDE689
:10A0A0004C480022B0F90010104609F0F5FADFF82C
:10A0B000148198F85C03F8B1DFF81C9199F800005E
:10A0C00018B908F018FD89F80070CDE9006543A3C0
:10A0D0006C220021012007F02DFFCDE9006541A38E
:10A0E00097220021012007F025FF98F80610202272
:10A0F000002008F021FDA5E098F8080004284DD9BB
:10A1000039480078012804D099F8071001291FD098
:10A110001FE008F0F0FC4FF4784ACDE900A533A326
:10A1200067220021012007F005FFCDE900A531A33A
:10A1300092220021012007F0FDFECDE900A52FA30A
:10A14000BD220021012007F0F5FE89F8077079E0B3
:10A1500058B12D48B0F9000007F03EFF2B480078B9
:10A1600008F01DF908F065F96CE089F8074008F07F
:10A17000C2FC8BF801708BF802708BF803708BF8BF
:10A1800005708BF804706921662008F067FE942141
:10A19000662008F063FEBF21662039E047E000003A
:10A1A0003502002069000020330000203402002026
:10A1B0005570646174696E670000000052657374C5
:10A1C000617274001C6D00205016002042000020B7
:10A1D0004800002062020020110300204D4F44423D
:10A1E0005553000049440000420200204869676856
:10A1F00000000000566F6C74616765006F6E20523E
:10A200005334383500000000540000202C0000209A
:10A2100008F024FE47F61761CDE90161ED20002327
:10A2200000901A462D21EF2007F0BAFE0AE0FC4804
:10A23000B0F9000007F0D0FEFA48007808F0AFF857
:10A2400008F0F7F84FF00009484603F0AFFE09F1B7
:10A25000010909F0FF09B9F1090FF5D308F00BFA6C
:10A2600008F01EF998F80800042811D9EE48007883
:10A27000012806D0ED48007838B1012009F099F99D
:10A280000FE0002009F095F90BE009F025F908E04E
:10A29000E648007818B1012009F08BF901E009F0D7
:10A2A0001BF99BF8070048B1CDE901650023E04A9E
:10A2B0001A210D20009407F057FE08E0CDE9016552
:10A2C00000231A461A210D20009407F069FE9BF81E
:10A2D000080048B1CDE901650D23D64A1A21184678
:10A2E000009407F041FE08E0CDE901650D2300224E
:10A2F0001A211846009407F053FE9BF8070010B18E
:10A30000401E8BF807009BF8080010B1401E8BF828
:10A310000800C9488079022814D050B1012808D01B
:10A32000CDE901651A21D223C44A0846009407F0FA
:10A330001BFEC348007803F059F84FF496700DF0F7
:10A340007FFEBEE4CDE901651A21D223BD4A08464D
:10A35000009407F009FEECE7BB4800240470BB48FA
:10A36000047006F061FEBA48047006F0D0FE1420B6
:10A370000DF066FEF9E700240EF0A8F84FF4007126
:10A38000B448FEF7C3FCB44D4FF49640461095F820
:10A390006510092930D2DFE801F005090C11161B00
:10A3A00020252A0030460DF007FD27E00DF004FDC2
:10A3B00024E04FF416400DF0FFFC1FE04FF4614025
:10A3C0000DF0FAFC1AE04FF4E1300DF0F5FC15E069
:10A3D0004FF496300DF0F0FC10E04FF496600DF065
:10A3E000EBFC0BE04FF496500DF0E6FC06E04FF46A
:10A3F00061500DF0E1FC01E00DF0DEFC30460DF0A7
:10A4000037FD96494FF4C8700880954908800020B0
:10A410000026291881F8A961401CC0B20828F8D389
:10A42000DFF84092904FDFF84482DFF844A2DFF873
:10A4300044B299F8000038B1401EC0B289F800005B
:10A44000012801D113F0A8FA387830B13878401ECD
:10A450003870387808B90DF013FEB8F80A003228C1
:10A4600003D2401CA8F80A0014E0A8F80A6007F01C
:10A47000CBF98148828881490A8082798A70C279C1
:10A48000CA70027A0A7102787D490A7042784A706D
:10A4900080788870C82C1DD100249AF800001428F8
:10A4A0001ED015281ED07748774902680A60426896
:10A4B0004A60007A087209200EF000F895F86002F0
:10A4C0009BF80010884205D085F860124FF4187090
:10A4D00007F04EF9641CA4B20A200DF0B1FDA8E704
:10A4E0006A48E1E76A48DFE708B50AF0DAF95A4D49
:10A4F00047352878697800EB012166480180A97802
:10A50000EA7801EB0221418029796A7901EB022185
:10A510008180A979EA7901EB0221C180297A6A7ADE
:10A5200001EB02210181A97AEA7A01EB0221418142
:10A53000297B6A7B01EB02218181A97BEA7B01EB0C
:10A540000221C18104215448FEF7E0FB4FF4007161
:10A550004048FEF7D9FB45200BF08FF9434C00270C
:10A56000E7704E4E4FF032084FF0010901230022F0
:10A570004B494C48CDF800800BF0EFFA08B986F84B
:10A580000090E078401CC0B2E0700A28EED330782A
:10A59000012800D03770DFF810A1444E444FDFF897
:10A5A0008480DFF810B1042543480178491C01700C
:10A5B00009F02AFE09F0BDFFFEF7D6FD4FF0000CB2
:10A5C00084F804C00020244A131893F89E1202292C
:10A5D00001D0042923D1DFF8E4E03EF810E0BEF119
:10A5E000010F02D02379C3B186E09AF80010A9B90F
:10A5F000357087F8009088F8005082F89B5093F8E7
:10A600009E12022906D192F86310C1EB0111890054
:10A61000CBF8001084F804906EE051E06CE070E03C
:10A62000540000202C000020420200200C030020D7
:10A63000ECCB030890CE0308902200207CD60308C0
:10A64000F800002034D10308FC000020F3000020B3
:10A65000F7000020000C01401C6D00205E0200206D
:10A660005C020020220300202003002000000020C4
:10A67000130300209002002068110020E80300204E
:10A68000E003002028D40208B603002031D40208D9
:10A690003AD40208B81100200018014041020020FD
:10A6A0008402002080020020290000203B000020BE
:10A6B000370000204C00002048020020F01100204C
:10A6C00092F8B93213B104290DD015E0DBF800106F
:10A6D00091B986F800C03D7088F800C082F89BC030
:10A6E0008AF800C008E086F800C03D7088F800C015
:10A6F00082F89BC08AF800C0E44981F8049081F890
:10A700000290401CC0B20828FFF45DAF0AF0CAF9FD
:10A71000DF4890F8EF12012935D1DE4A90F8F112A6
:10A720001288511A00D5494290F8B42391422ADD8B
:10A7300084F8009084F8019090F86310FF2902D10A
:10A740003C2180F8631090F86310A9B1C1EB0111AE
:10A750008900CBF80010D04981F80090357088F856
:10A760000050417A41F001014172092007F000F8E0
:10A7700087F8009002206070C44880F8029080F84A
:10A78000019080F804904FF496700DF059FC0BE79F
:10A7900000240025C14900200870C1490870C14942
:10A7A000FF200870C049087040F6B8300DF048FC32
:10A7B000DFF8F892BE4EBF4FDFF8D48299F8000060
:10A7C00015F05FF83080B7F90810884203D038815F
:10A7D000AE49012048706D1CADB298F8800100EBC5
:10A7E0008000A84204D2012015F0C0FA002502E042
:10A7F000002015F0BBFA641CE4B2052C09D998F8C6
:10A80000DB0003280BD0012003F0CFFC002404F070
:10A8100030FD0AF066FCC8200DF012FCCEE70220E5
:10A8200003F0C3FCF2E72DE9FF470024A249080327
:10A83000FDF7A7FFFEF735FF4FF4A060FDF76CFFB3
:10A84000FEF792FC48200DF0C7FB40F2CF216420B8
:10A8500009F062F806F0E0FEFEF774FC06F0E4FB97
:10A8600000F02DFAFEF701FC0AF0A0F9002101200A
:10A870000AF0FEFA002102200AF0FAFA0021032071
:10A880000AF0F6FA002104200AF0F2FA002105206D
:10A890000AF0EEFA7E4E894996F86A000870FEF7D3
:10A8A00065FCFEF761FCFEF75FFC01218448FEF7C2
:10A8B0002BFA07F0D3FA834800250582824996F8DF
:10A8C0009B000870DFF8D081012788F800707F4A6C
:10A8D0000721117086F87A53C82186F87B1396F801
:10A8E0007F10012901D97A490F7096F8B9226F4972
:10A8F0000AB988B10F70087814F0C3FF6C4908805A
:10A9000098F80020734874494AB196F86C20028088
:10A9100096F86D00088008E004200870EBE796F8D0
:10A920007120028096F87000088096F892106B48AB
:10A930004FF00308012905D080F82B8096F8D80045
:10A9400018B104E080F82B50F8E76548057014F062
:10A9500092FB6448311991F8B2100155641CE4B2BD
:10A96000072CF7D3FEF700FC0126FEF7FDFB142CA5
:10A970000AD206F0B1FF012806D0641CE4B26420BC
:10A980000DF05EFB002EF0D10620CDE900054FF45E
:10A99000617602950023324653A1574803950CF087
:10A9A00046FD0220CDE900054FF4C8790295002349
:10A9B0004A4652A1534803950CF039FD0524CDE9D0
:10A9C0000045029500234A464FA1514803950CF0DB
:10A9D0002EFDCDE900850295002364224DA151484A
:10A9E00003950CF024FDCDE9008502950023642237
:10A9F0004DA1514803950CF01AFDCDE90075029563
:10AA0000002364224DA1514803950CF010FDCDE9BF
:10AA100000450295002332464DA14F4803950CF0A6
:10AA200006FDCDE900750295002364224BA14F4835
:10AA300003950CF0FCFCCDE90045029500234FF492
:10AA400016724BA14D4803950CF0F1FC0CF0CCFFB5
:10AA500004B00020BDE8F087494D00264FF47A7716
:10AA6000287870B1401EC1B2297051B9002400226B
:10AA70002146444800F09BF8641CE4B2032CF6D352
:10AA80002E7038460DF0DCFAEAE700007211002063
:10AA90001C6D0020560200203A00002073000020A8
:10AAA000940200209502002096020020370000202A
:10AAB00054000020000000200080000877000020E3
:10AAC00000080140DC1100203B000020390000207C
:10AAD00034000020C4030020C603002050160020CC
:10AAE0005A000020C4000020436F6E74726F6C4CDB
:10AAF0006F6769630000000091A70008496E7075D8
:10AB000074000000E9A40008434F4D4D0000000010
:10AB100077A300084B65797061647348616E646C5B
:10AB20006500000059A3000844697370616C795294
:10AB300065667265736800000F9C0008536F667449
:10AB40007761726574696D6572000000EF970008A7
:10AB50004D5354500000000067970008436F6F6C1E
:10AB6000696E674C6F636B4F75740000B99600088F
:10AB7000576966697461736B000000000B6F010810
:10AB8000720000208000002048437047C84000F059
:10AB90000100704701238B40DBB20178002A02D00C
:10ABA000194301707047DA43114001707047012367
:10ABB0008B409BB20188002A02D019430180704764
:10ABC000DA4311400180704701228A40D1B20078F7
:10ABD000084201D1002070470120704770B540F253
:10ABE0007A4006F0C4FDFE4D287040F27C4006F02D
:10ABF000BEFD4FF6FF7404EA0020688040F27B40FF
:10AC000006F0B5FD69880844688040F27D4006F092
:10AC1000AEFDF44D287040F27F4006F0A8FD04EA36
:10AC20000020688040F27E4006F0A1FD698808445B
:10AC300068804FF4906006F09AFDEB4D287040F26A
:10AC4000824006F094FD04EA0020688040F28140D2
:10AC500006F08DFD69880844688040F2894006F05E
:10AC600086FDE24D287040F28B4006F080FD04EA3C
:10AC70000020688040F28A4006F079FD6988084427
:10AC8000688040F2834006F072FDD94D287040F292
:10AC9000854006F06CFD04EA0020688040F28440A4
:10ACA00006F065FD69880844688070BD01EB0021ED
:10ACB00009B27F2801D908B27047084670472DE9CC
:10ACC000F84F6E2006F053FDDFF8288388F86E00F9
:10ACD0000024012805D988F86E4000216E2006F076
:10ACE00047FD0025C44E4FF48F67284606F03FFD10
:10ACF000A5F15F02A42A1FD298F86E1001EBC103E0
:10AD000003EB411106EBC10313F812C0844507D8C9
:10AD100003EB42025278824202D308F805000DE0AC
:10AD2000B64800EB8100284410F85F1C08F80510B5
:10AD3000284606F01DFD01E008F805006D1CADB2C7
:10AD4000BD42D2D998F85D00FF2801D188F85D4056
:10AD5000AB4998F85D000870AB4D0222A94928461E
:10AD6000FDF71EFCA74E327898F80610FF291BD07D
:10AD7000D1B1914205D03180012231462846FDF7FC
:10AD80001EFC00256F46284606F0F1FC78556D1C28
:10AD9000ADB2042DF7D39C4B9B4D9DF800101033A2
:10ADA0002035FF2910D01BE0022296492846FDF7E6
:10ADB000F7FB307888F80600FF2801D00028E0D1A2
:10ADC000FE2088F80600DCE79DF80100FF2807D187
:10ADD0009DF80200FF2803D19DF80300FF282ED024
:10ADE000F1B398F80000814224D09DF8010098F852
:10ADF000012090421ED09DF8022098F80250AA42ED
:10AE000018D09DF8032098F80350AA4212D0318040
:10AE100070801D4602227B492846FDF7D0FB9DF835
:10AE2000021031809DF80310718002227549284676
:10AE3000FDF7C5FB98F8D902FF2830D036E0022292
:10AE400070491846FDF7ACFB307888F80000B07800
:10AE500088F8010002226B492846FDF7A1FB00E0BB
:10AE600006E0307888F80200B07888F80300E1E75F
:10AE7000022264491846FDF793FB307888F80000F9
:10AE8000B07888F8010002225E492846FDF788FB69
:10AE9000307888F80200B07888F80300CAE788F8AC
:10AEA000D942002140F2D92006F062FC98F87E03D6
:10AEB000FF280DD188F87E4388F87D43002140F2B9
:10AEC0007D3006F055FC002140F27E3006F050FC4B
:10AED00098F87E034B4D0002283D98F87D130143FE
:10AEE000298398F81B1098F81C00012601EB00221A
:10AEF00098F82F00454900EB0020824201D20E70E5
:10AF000000E00C7098F8310098F8322000EB022233
:10AF100098F8450000EB0020824201D24E7000E01C
:10AF20004C704FF45A77384606F021FC38490870C7
:10AF3000FF2804D10C702146384606F019FC98F819
:10AF40005C00344BFF2803D198F85B10FF290AD02E
:10AF500098F85B10FFF7AAFE188098F8811320205C
:10AF6000FF290AD01BE01C8000215B2006F000FCBA
:10AF700000215C2006F0FCFBEFE74F2188F88113ED
:10AF8000662188F8821388F8831388F8844388F848
:10AF9000850388F8860388F8870388F8880398F87B
:10AFA00089236F21FF2A11D14C2288F8892388F840
:10AFB0008A13772288F88B2388F88C4388F88D03CE
:10AFC00088F88E0388F88F0388F8900398F8912307
:10AFD0006427FF2A2ED14D2288F8912365221BE099
:10AFE00086110020901100209A110020A411002049
:10AFF000AE1100201C6D0020DAD902086ADC0208BC
:10B000004002002050000020007700087802002055
:10B01000160300206802002088F8922388F89373B2
:10B0200088F8944388F8950388F8960388F897037E
:10B0300088F8980398F89923FF2A11D1482288F8B4
:10B040009923692288F89A2388F89B4388F89C03FF
:10B0500088F89D0388F89E0388F89F0388F8A0036A
:10B0600098F8A123FF2A12D1412288F8A123752242
:10B0700088F8A223742288F8A32388F8A41388F8F8
:10B08000A54388F8A60388F8A70388F8A80398F8CA
:10B0900089034C2800D0EE7198F8ED00FF2806D007
:10B0A000C0EB00104FF6FF7101EA8000E88298F8CB
:10B0B000A903FF2801D188F8A94398F89702FF282F
:10B0C00011D198F89602FF280DD1002140F2972067
:10B0D00006F04EFB88F89742012140F2962006F0D8
:10B0E00047FB88F8966298F82D04FF280ED10025BA
:10B0F00005F22D4080B2002106F03AFB08EB050076
:10B1000080F82D446D1CADB22E2DF1D313F06CFEE2
:10B1100098F882004546022801D985F8824095F8C2
:10B120009200DFF82CB4012804D985F8924003205E
:10B130008BF82B0095F8B403FF2806D11E2185F863
:10B14000B4134FF46D7006F013FB40F28C4006F020
:10B150000EFB00EB80004000FE4908804FF47A723D
:10B16000904201D90A8005E0B0F5FA7F02D24FF48F
:10B170002F70088040F28D4006F0F9FAF649087009
:10B18000FFF72CFD95F8F102FF2800D010B9A020A0
:10B1900085F8F102F149A879087040F28F4A5046CB
:10B1A00006F0E5FADFF8B8934FF49268FF2804D16F
:10B1B000404606F0DCFAFF283AD0504606F0D7FAAF
:10B1C000C9F80000404606F0D2FAD9F8001041EA6A
:10B1D0000020C9F8000040F2914006F0C8FAD9F802
:10B1E000001041EA0040C9F8000040F2924006F029
:10B1F000BEFAD9F8001041EA0060C9F80000002149
:10B20000DFF86093002001EB41024FEA820801EB76
:10B21000410209EBC20208EB40032B4493F8B5C38B
:10B22000BCF1180F11D902EB400C8CF8014010E072
:10B230002878697840EA0120A97840EA0140E97855
:10B2400040EA0160C9F80000D9E702EB400A8AF839
:10B2500001C093F8B6333B2B02D902F8104001E04D
:10B2600002F81030401C80B20628D4D3491C89B2A1
:10B270000829C7D30020BC492A1892F82D240A5463
:10B28000401C80B22E28F7D395F878043238652810
:10B2900001D385F8787440F2954006F068FAB34F10
:10B2A0000002388040F2944006F061FA3988084381
:10B2B000388040F2974006F05AFAAD4F00023880CD
:10B2C00040F2964006F053FA398808433880002748
:10B2D000A046E81990F86712FF2907D180F8678225
:10B2E00007F2672080B2002106F042FA7F1CBFB24D
:10B2F000092FEED395F88101FF2806D185F88181C9
:10B30000002140F2811006F033FA95F88001FF2801
:10B3100006D185F8808100214FF4C07006F028FA2C
:10B320000021944A944F002007EB811343F820201A
:10B33000401C80B21028F9D3491C89B20729F2D3E6
:10B340009BF82B00032838D10024DFF830A20AF242
:10B3500066390AF1D60AE1B25046FFF735FC40B132
:10B36000E1B24846FFF730FC21F044FE07EB8411C0
:10B37000C861641CA4B2052CEDD305215046FFF72B
:10B3800023FC50B195F8620395F86313000200B2F4
:10B39000084421F017FEC7F85C0106215046FFF76C
:10B3A00013FC50B195F8640395F86513000200B2E0
:10B3B000084421F007FEC7F89C0195F85F03FF28B9
:10B3C00012D195F860132846FF290DD180F85F83CC
:10B3D00080F86083002140F25F3006F0C9F9002157
:10B3E0004FF4587006F0C4F9E879092803D0092110
:10B3F000072006F0BDF995F85F0040F2613415288A
:10B4000005D1314685F86163204606F0B1F995F81B
:10B41000A200152805D1314685F86163204606F063
:10B42000A7F94FF4187006F0A2F95549087095F87D
:10B430002903FF2802D1052085F82903BDE8F88FEC
:10B440001CB502460846843A4E4CC1B2072A0ED2B9
:10B45000DFE802F0040E190D242F3900A17862787C
:10B46000CDE900212378E279A17906F08CFA1CBDA0
:10B47000A1786278CDE900212378E279C1B2A08871
:10B4800006F081FA1CBDA1786278CDE9002123780D
:10B49000A179C2B2A08806F076FA1CBDA1786278C4
:10B4A000CDE90021E279C3B2A179A08806F06BFA58
:10B4B0001CBDA078CDE900102378E279A179A0889D
:10B4C00006F061FA1CBD6078CDE900012378E279CD
:10B4D000A179A08806F057FA1CBD10B501210F20F4
:10B4E00006F046F90021102006F042F90121112052
:10B4F00006F03EF90021BDE81040122006F038B9F0
:10B5000070B50024204D04F5B070295D06F030F9C7
:10B51000641CE4B2072CF6D370BD70B500241B4D3B
:10B5200024F00100295C04F11B0006F021F9A41CA1
:10B53000E4B2152CF4D3012424F00100285A010AA6
:10B5400004F11B0006F014F9A41CE4B2162C1FE051
:10B550005016002098020020100300201C03002039
:10B560000C000020F2730020C47300206E02002043
:10B570006C02002000007F43047200201C6D00203C
:10B58000900200206811002085D4020844D40208EB
:10B59000D2D30024FE4D24F00100295C04F13100D7
:10B5A00006F0E6F8A41CE4B2152CF4D3012424F030
:10B5B0000100285A010A04F1310006F0D9F8A41C50
:10B5C000E4B2162CF3D370BD2DE9F0410025DFF86D
:10B5D000C4830024C5EBC50000EB080605EB850716
:10B5E0003819315D00F5A17006F0C2F8641CE4B2B0
:10B5F000052CF5D36D1CEDB2022DEAD3BDE8F08128
:10B6000070B50024E44D04F22D10295D06F0B0F869
:10B61000641CE4B2152CF6D370BD2DE9F041074649
:10B620000024DE4D0126062F21D2DFE807F07F033C
:10B630007F214462DA48015D04F2031006F098F8B5
:10B64000012C07D10321A02006F092F80321A120AC
:10B6500006F08EF8072C04D2002104F1B20006F0A7
:10B6600087F801216F2006F083F885F86F605DE0B0
:10B67000CC48015D04F2031006F07AF8012C07D1E2
:10B680000221A02006F074F80221A12006F070F833
:10B69000072C04D2002104F1B20006F069F804215D
:10B6A0009B2006F065F803216F2006F061F8032067
:10B6B00085F86F003AE0BC48015D04F2031006F023
:10B6C00057F8012C07D10221A02006F051F80221E1
:10B6D000A12006F04DF8072C04D2002104F1B2009D
:10B6E00006F046F801216F2006F042F885F86F60F9
:10B6F0001CE0AE48015D04F2031006F039F8012C9D
:10B7000007D10221A02006F033F80221A12006F083
:10B710002FF8072C04D2002104F1B20006F028F81B
:10B7200001216F2006F024F885F86F60641CE4B2F4
:10B730002A2CFFF478AF61E72DE9F0415F249C4D9E
:10B74000964E4FF48177652C19D096F86E0000EB79
:10B75000C00101EB401005EB8000204410F85F1C95
:10B76000204606F005F896F86E0000EBC00101EBEC
:10B77000401005EB8000204410F85F0C3055641C2D
:10B78000A4B2BC42DFD996F86E1040F259256C1C69
:10B7900011B1012913D024E0C821284605F0E8FFA3
:10B7A0000021204605F0E4FF284605F0E0FF86F87A
:10B7B0005902204605F0DBFF86F85A0211E0A82165
:10B7C000284605F0D5FF0221204605F0D1FF284686
:10B7D00005F0CDFF86F85902204605F0C8FF86F82F
:10B7E0005A0274480078FFF718FFFFF709FFFFF7C8
:10B7F000EBFEFFF792FEFFF783FEFFF76EFE4F2191
:10B8000040F2813005F0B4FF662140F2823005F04D
:10B81000AFFF662140F2833005F0AAFF00214FF40C
:10B82000617005F0A5FF202140F2853005F0A0FFF2
:10B83000202140F2863005F09BFF202140F2873026
:10B8400005F096FF20214FF4627005F091FF4C2126
:10B8500040F2893005F08CFF6F2140F28A3005F00C
:10B8600087FF772140F28B3005F082FF00214FF4F3
:10B87000637005F07DFF202140F28D3005F078FFE8
:10B88000202140F28E3005F073FF202140F28F30EE
:10B8900005F06EFF20214FF4647005F069FF4D2123
:10B8A00040F2913005F064FF652140F2923005F0DE
:10B8B0005FFF642140F2933005F05AFF00214FF4FE
:10B8C000657005F055FF202140F2953005F050FFDE
:10B8D000202140F2963005F04BFF202140F29730B6
:10B8E00005F046FF20214FF4667005F041FF482126
:10B8F00040F2993005F03CFF692140F29A3005F0A2
:10B9000037FF002140F29B3005F032FF20214FF439
:10B91000677005F02DFF202140F29D3005F028FFD3
:10B92000202140F29E3005F023FF202140F29F307D
:10B9300005F01EFF20214FF4687005F019FF41212A
:10B9400040F2A13005F014FF752140F2A23005F05D
:10B950000FFF742140F2A33005F00AFF6F214FF46E
:10B96000697005F005FF002140F2A53005F000FFE9
:10B97000202140F2A63005F0FBFE202140F2A73046
:10B9800005F0F6FE20214FF46A7005F0F1FE13E099
:10B990005AD402085ADE020870D402081C6D002036
:10B9A000B2DD0208DCDD020806DE020830DE020835
:10B9B0006ADC0208770000200021922005F0D8FE02
:10B9C000002448274FF0470807EB4405A8B205F0CC
:10B9D000CEFEFF2809D108EB440080B2002105F01B
:10B9E000C7FEA8B2002105F0C3FE641CA4B2082C57
:10B9F000EAD3012086F8B80201214FF42E7005F039
:10BA0000B7FE0E2140F2BA2005F0B2FE0E2086F8F5
:10BA1000BA0296F848030025FF2873D106F552763E
:10BA20005420307053217170B0704121F170307129
:10BA300038207071B571F571A6F5527654214FF426
:10BA4000527005F095FE532140F2493005F090FE0A
:10BA5000542140F24A3005F08BFE412140F24B3038
:10BA600005F086FE54214FF4537005F081FE382115
:10BA700040F24D3005F07CFE002140F24E3005F0E2
:10BA800077FE002140F24F3005F072FE00214FF4A6
:10BA9000547005F06DFE002140F2513005F068FE53
:10BAA000002140F2523005F063FE002140F2533095
:10BAB00005F05EFE00214FF4557005F059FE00219F
:10BAC00040F2553005F054FE002140F2563005F0AA
:10BAD0004FFE002140F2573005F04AFE00214FF49E
:10BAE000567005F045FE002140F2593005F040FE49
:10BAF000002140F25A3005F03BFE002140F25B305D
:10BB000005F036FEC82140F2AA3005F031FE0021D2
:10BB100040F2AB3005F02CFEC8214FF46B7005F0FD
:10BB200027FE002140F2AD3005F022FE282140F230
:10BB3000AE3005F01DFE102140F2AF3005F018FECA
:10BB40001E214FF46C7005F013FE0F2140F2B1304E
:10BB500005F00EFE322140F2B23005F009FE05215B
:10BB600040F2B33005F004FE06214FF4A87005F052
:10BB7000FFFD1E2140F2511005F0FAFD08214FF49F
:10BB8000A97005F0F5FD1E2140F2531005F0F0FDFF
:10BB900012214FF4AA7005F0EBFD1E2140F2551062
:10BBA00005F0E6FD16214FF4AB7005F0E1FD1E2116
:10BBB00040F2571005F0DCFD002140F2B92005F0FD
:10BBC000D7FD96F89702FF280DD196F89602FF2828
:10BBD00009D1002140F2972005F0CAFD012140F271
:10BBE000962005F0C5FD40F2E1718420FFF728FCA6
:10BBF0000024301990F86712FF2907D180F86752A6
:10BC000004F2672080B2002105F0B2FD641CA4B2EA
:10BC1000092CEED3002404F5A17080B2002105F0B8
:10BC2000A7FD641CA4B2072CF5D3002404F249102C
:10BC300080B2002105F09CFD641CA4B2072CF5D352
:10BC4000DCE42DE9F041FE4C40F25A26204694F8FF
:10BC50006E10771E90F87E0000297DD000EBC000AA
:10BC60000525B0FBF5F020307B34C1B2E1707E20B9
:10BC700005F07EFDA07800EBC000B0FBF5F02030B1
:10BC8000C1B2A1707D2005F073FD14F8040C00EB27
:10BC9000C000B0FBF5F02030C1B204F8041C7720DE
:10BCA00005F066FD94F8660000EBC000B0FBF5F00F
:10BCB0002030C1B284F86610E12005F059FD94F8F7
:10BCC000DE0194F8DF1100EB012080B200EBC00030
:10BCD000B0FBF5F000F5A07082B2110A84F8DF1114
:10BCE00084F8DE21304605F043FD94F8DE11384635
:10BCF00005F03EFDA07EE17E00EB012080B200EB6E
:10BD0000C000B0FBF5F000F5A07080B2010AE1764A
:10BD1000A076962005F02CFDA17E952005F028FD4B
:10BD2000207F617F00EB012080B200EBC000B0FB00
:10BD3000F5F000F5A07080B2010A617720779820B5
:10BD400005F016FD217F972005F012FDA07FE17F11
:10BD500000EB012080B200E041E000EBC000B0FB4E
:10BD6000F5F000F5A07080B2010AE177A0779A2083
:10BD700005F0FEFCA17F992005F0FAFC14F8070DF0
:10BD8000617800EB012080B200EBC000B0FBF5F061
:10BD900000F5A07080B2010A61702070752005F076
:10BDA000E7FC14F8071B742005F0E2FC14F8090DF9
:10BDB000617800EB012080B200EBC000B0FBF5F031
:10BDC00000F5A07080B2010A61702070732005F048
:10BDD000CFFC2178BDE8F041722005F0C9BC2038C5
:10BDE000C0B2092500EB8000B0FBF5F07B34C1B296
:10BDF000E1707E2005F0BCFCA0782038C0B200EBDA
:10BE00008000B0FBF5F0C1B2A1707D2005F0B0FC60
:10BE100014F8040C2038C0B200EB8000B0FBF5F041
:10BE2000C1B204F8041C772005F0A2FC94F8660067
:10BE30002038C0B200EB8000B0FBF5F0C1B284F84E
:10BE40006610E12005F094FC94F8DE0194F8DF110F
:10BE500000EB0120A0F5A07080B200EB8000B0FBE9
:10BE6000F5F082B2110A84F8DF1184F8DE21304641
:10BE700005F07EFC94F8DE11384605F079FCA07ED2
:10BE8000E17E00EB0120A0F5A07080B200EB800005
:10BE9000B0FBF5F080B2010AE176A076962005F0BD
:10BEA00067FCA17E952005F063FC207F617F00EB9D
:10BEB0000120A0F5A07080B200EB8000B0FBF5F08F
:10BEC00080B2010A61772077982005F051FC217F2C
:10BED000972005F04DFCE17F5A4EA07F06EB012133
:10BEE000084480B200EB8000B0FBF5F080B2010A9C
:10BEF000E177A0779A2005F03BFCA17F992005F01F
:10BF000037FC14F8070D617806EB0121084480B274
:10BF100000EB8000B0FBF5F080B2010A6170207088
:10BF2000752005F025FC14F8071B742005F020FC93
:10BF300014F8090D617806EB0121084480B200EB8A
:10BF40008000B0FBF5F080B2010A617020707320B0
:10BF500005F00EFC2178BDE8F041722005F008BC28
:10BF600010B5374C012823D09A2005F000FC70341E
:10BF700084F82A00992005F0FAFB84F82900702043
:10BF800005F0F5FB2070712005F0F1FB6070752065
:10BF900005F0EDFB6071742005F0E9FB2071732062
:10BFA00005F0E5FBE070722005F0E1FBA07010BD2C
:10BFB00040F25A2005F0DBFB793484F8E10140F2CD
:10BFC000592005F0D4FB84F8E0016C2005F0CFFB8C
:10BFD00004F80D0C6D2005F0CAFB04F80C0C96203B
:10BFE00005F0C5FB6077952005F0C1FB2077982010
:10BFF00005F0BDFBE077972005F0B9FBA07710BDF9
:10C000002DE9F043DFF838800F4A414698F8B9929D
:10C01000D07C91F8615359EA000991F87D000B4FEB
:10C0200000EB800300EB800091F8C5104FEA40045C
:10C0300002F12C064FF0050C13D098F8590207E0D6
:10C040001C6D0020C0FEFFFF28000020130300200D
:10C0500098F85A8200EB0820084400B250834DB390
:10C060002CE098F8990098F89A8000EB082000B22C
:10C0700050830A2903D00844508385B115E00A2172
:10C0800090FBF1F801FB1808B8F1000FF5D090FB18
:10C09000F1F801FB1801401A0A305083EDE7B2F9BC
:10C0A0001A00B0EB430F00DD5483508B308087F8CB
:10C0B00000C007E0B0EB430F00DD5483508B3080AD
:10C0C000062038700020D07282F808C0BDE8F083E6
:10C0D0002DE9F041DFF8E4C3F94A9CF8B70090730A
:10C0E0009CF8B982D07C614658EA000891F87E003D
:10C0F00091F8615300EB800300EB8000F14F91F861
:10C10000C5104FEA400402F12C060AD09CF85902EF
:10C110009CF85AC200EB0C20401A00B250834DB379
:10C120002CE09CF899009CF89AC000EB0C2000B21F
:10C1300050830A2903D0401A508385B115E00A21A3
:10C1400090FBF1FC01FB1C0CBCF1000FF5D090FB47
:10C15000F1FC01FB1C01401A0A385083EDE7B2F9EB
:10C160001A00B0EB430F00DA5483508B3080072065
:10C17000387007E0B0EB430F00DA5483508B308007
:10C18000082038700020D0720520107258E52DE983
:10C19000F041CB4CC94D01262179687A002914D091
:10C1A00040F001016972A674092005F0E1FA95F8E2
:10C1B0006300C0EB0010800060622179E17485F8B3
:10C1C0009B1095F8B902C8B11BE000F0FE0169723E
:10C1D0000027A774092005F0CBFABB4807706762F7
:10C1E0002179E17485F89B1095F8B90210B99B206C
:10C1F00005F0BEFAA7710420E07303E09B2005F070
:10C20000B7FAE673E07CE070B048067118E570B5E7
:10C21000AB4A012555711079042801D2401C1071D8
:10C220001079A64B002404280DD90020191891F884
:10C230009E12022901D0042900D15570401CC0B2C1
:10C240000828F3D3147193F86F10137904209942DE
:10C2500000D21071D47250729D4E3570107906F074
:10C260009EF8347070BD70B5954901224A71087905
:10C27000002801D0401E087190480B7990F86F009B
:10C28000984200D208710024CC7204204872904D6C
:10C290002A70087906F083F82C7070BD10B58749B4
:10C2A000002491F86B00002825D191F8A9030228F9
:10C2B00002D2401C81F8A90391F8A00028B991F896
:10C2C000A903022801D181F8A94391F8A10030B94E
:10C2D00091F8A903012802D1022081F8A90391F85D
:10C2E000A903022801D981F8A94391F8A91340F2C2
:10C2F000A93005F03DFA7248C4720421817210BD64
:10C3000010B56E49002491F86B0000281DD191F8FA
:10C31000A90310B1401E81F8A90391F8A00028B923
:10C3200091F8A903022801D181F8A94391F8A1004D
:10C3300028B991F8A903012801D181F8A94391F8FE
:10C34000A91340F2A93005F013FA5D48C472042124
:10C35000817210BD7CB55F4843F6EF464FF6FF751E
:10C36000007847F6196401281CD0022833D003282E
:10C3700017D1CDE9005458A36C220A21012005F001
:10C38000D9FDCDE9005455A397220A21012005F0DB
:10C39000D1FDCDE9005652A3C2220A21012005F0A9
:10C3A000C9FD7CBDCDE900564BA36C220A210120BA
:10C3B00005F0C0FDCDE9005448A397220A210120D1
:10C3C00005F0B8FDCDE9005445A3C2220A210120A1
:10C3D00005F0B0FD7CBDCDE900543FA36C220A21DD
:10C3E000012005F0A7FDCDE900563CA397220A21C4
:10C3F000012005F09FFDCDE9005439A3C2220A2196
:10C40000012005F097FD7CBD7CB5324843F6EF4630
:10C410004FF6FF75007847F6196401281CD00228F2
:10C4200033D0032817D1CDE900542BA36C220A2165
:10C43000012005F07FFDCDE9005428A397220A21B1
:10C44000012005F077FDCDE9005625A3C2220A217F
:10C45000012005F06FFD7CBDCDE900561EA36C22C6
:10C460000A21012005F066FDCDE900541BA39722A7
:10C470000A21012005F05EFDCDE9005418A3C22277
:10C480000A21012005F056FD7CBDCDE9005412A320
:10C490006C220A21012005F04DFDCDE900560FA3C5
:10C4A00097220A21012005F045FDCDE900540CA397
:10C4B000C2220A21012005F03DFD7CBD1C6D00203B
:10C4C0002800002013030020D80000207211002053
:10C4D00010000020F00000205345540046414E005B
:10C4E000535953002DE9F041022006F0E5FAF74ECA
:10C4F000F74BF84D308C06F11E0477280ED07D28BE
:10C500000CD0702843D071284AD0822851D0002105
:10C5100001226B2854D05E2871D07FE0772819D093
:10C5200095F8610301282ED095F87E00B4F900102B
:10C53000401C81420DDD95F86E0000EBC00202EB5D
:10C54000401003EBC00090F83C00814201DD491E21
:10C550002180C8E095F86103012813D1B4F90010D7
:10C5600095F87E0081420DDD95F86E0000EBC0026B
:10C5700002EB401003EBC00090F83000814201DD77
:10C58000491E2180AFE02088401E2080ABE021883A
:10C590000A392180C9B285F8701005F0E9F8A2E0E7
:10C5A00021880A392180C9B285F8711005F0E0F8B8
:10C5B00099E0B4F90000002801DD401E208092E0DF
:10C5C000B4F90000032802DB401E20808BE0022823
:10C5D00002D001280AD086E095F87900032801D01E
:10C5E000012801D821807EE022807CE095F8790046
:10C5F000032801D0012876D8218074E0FFE7377D39
:10C6000067B1B4F9000095F8CF10884202DD401EF2
:10C61000208068E095F8D100208064E05D2801D199
:10C62000377DD7B1572818D072281AD0652821D065
:10C6300095F86E1001EBC10707EB411103EBC10345
:10C64000A0F15F0113F81130B4F900108B424AD009
:10C65000491E2180E5283CD040E02088401E2080F3
:10C6600041E02088401E2080010A85F89A1085F854
:10C67000990038E0B4F9000090B1072813D00128E0
:10C6800014D0082815D0042815D0052816D0032862
:10C6900017D0022818D0062818D0401E208022E08B
:10C6A000072020801FE0062020801CE0082020803A
:10C6B00019E0218017E00520208014E0032020806D
:10C6C00011E0022020800EE022800CE00420208077
:10C6D00009E095F85F10012900D122805F2802D17E
:10C6E000208800B92280308C642802D1207885F817
:10C6F00064004BE570B5022006F0DEF9734B744C14
:10C70000744A188C03F11E01772804D07E2802D0C9
:10C710005E2834D042E092F861331BB10888401C97
:10C72000088070BD772815D092F87D00B1F90030EF
:10C73000401E8342F5DA92F86E0000EBC00202EB75
:10C74000401004EBC00090F83F008342E9DA5B1C24
:10C750000B8070BDB1F9003092F87D008342F8DAA9
:10C7600092F86E0000EBC00202EB401004EBC00038
:10C7700090F831008342ECDA5B1C0B8070BD1D7DAC
:10C7800065B1B1F9000092F8D130984202DA401C4C
:10C79000088070BD92F8CF00088070BD02256B281C
:10C7A00002D05E2819D01AE0B1F900303BB992F8F6
:10C7B0007900032801D0012801D80D8070BD92F8BE
:10C7C0006E0000EBC00202EB401004EBC000407EA4
:10C7D0009842F3DD5B1C0B8070BD1B7D13B370288A
:10C7E00024D071282CD0722834D082283AD06528E1
:10C7F0003FD092F86E3003EBC30505EB431304EB17
:10C80000C304A0F15F0304EB43035C78B1F900308B
:10C810009C4201D05B1C0B806428DDD1087882F833
:10C82000640070BD0888401C088070BD0B880A3306
:10C830000B80D9B282F87010BDE8704004F098BF48
:10C840000B880A330B80D9B282F87110BDE87040B2
:10C8500004F08EBF0888401C0880010A993251708C
:10C86000107070BDB1F900000228FADA401C08808F
:10C8700070BDB1F90000062811D0072812D0A0B170
:10C88000082815D0012816D0022816D0032817D062
:10C89000052818D00428EBD10620088070BD072099
:10C8A000088070BD0020088070BD0820088070BD21
:10C8B0000120088070BD0D8070BD0320088070BD10
:10C8C0000520088070BD0420088070BD280000206D
:10C8D000DAD902081C6D00204FF47A700BF0B0BB5F
:10C8E000FCF7B6BB2DE9F05FDFF8FCB3FF4E0BF1B0
:10C8F0001E05BBF820000127DFF8F4A3FD4CB5F9B5
:10C9000000104FF00208942806D0642809D05A4637
:10C910005E28127D0ED00EE0C80701D18AF8008093
:10C9200080E094F86410642004F022FF287884F8F2
:10C93000640077E012B15E2820D034E094F85F0004
:10C94000022801D013286DD1EB48DFF8B09300889E
:10C95000081AA9F80000C1B25B2004F009FFB9F879
:10C960000000C0F307215C2004F002FFB9F80000CA
:10C9700084F85B00000A84F85C0053E09AB1C9B205
:10C98000062004F0F5FE2878A071D74928310880E8
:10C990000122DB48FBF713FEDA49A07908700C206E
:10C9A0008AF800003EE083280DD0CF4A1E32B2F94B
:10C9B000002002EB82025200952814D09B281BD045
:10C9C000722826D02EE0C80706D00121832004F06B
:10C9D000CFFE8BF8107025E00221832004F0C8FE02
:10C9E0008BF810801EE0D1B2C2F3072012F051FF85
:10C9F0000120FFF7B5FA15E0C9B28BF8131084F8DF
:10CA00009B108BF804109B2004F0B2FEB7703771B6
:10CA100008E02A80D1B2C2F3072012F0E0FF002024
:10CA2000FFF79EFABBF82000B5F90010225C8A429D
:10CA300075D021545E2802D0C9B204F099FEBBF82B
:10CA400020006A2807D1297804F092FE2878FEF7A2
:10CA5000E4FDFFF745FFBBF820006E2807D12978D9
:10CA600084F86E1004F084FE3770FFF7EAF8BBF824
:10CA70002000792803D1FFF733FFFFF72DFFBBF824
:10CA800020005F2804D1297884F85F1004F070FE3C
:10CA9000BBF820006B281AD12888042809D194F803
:10CAA000E500012805D0394684F8E570E52004F05A
:10CAB0005FFE288805280AD194F8E600012806D0F0
:10CAC00084F8E67094F86210E62004F051FEBBF89A
:10CAD00020008D4E4FF00009652878D1297804F0A8
:10CAE00047FEB5F9000080B1012819D0022821D0F5
:10CAF000032829D0042832D005283BD0062844D06A
:10CB000007284DD0082856D05FE084F865904FF490
:10CB100016500BF051F94FF41650B06055E00CE18F
:10CB200084F865704FF496400BF046F94FF4964048
:10CB3000B0604AE084F865804FF416400BF03CF991
:10CB40004FF41640B06040E0032084F865004FF4D5
:10CB500061400BF031F94FF46140B06035E00420E2
:10CB600084F865004FF4E1300BF026F94FF4E13022
:10CB7000B0602AE0052084F865004FF496300BF091
:10CB80001BF94FF49630B0601FE0062084F8650072
:10CB90004FF496600BF010F94FF49660B06014E01B
:10CBA000072084F865004FF496500BF005F94FF418
:10CBB0009650B06009E0082084F865004FF4615099
:10CBC0000BF0FAF84FF46150B0600BF059FABBF873
:10CBD000200083280FD12878C00706D001218320A8
:10CBE00004F0C6FD8BF8107005E00221832004F0EC
:10CBF000BFFD8BF81080BBF820006C2801D06D2899
:10CC000025D10A216C2827D094F86D20B5F90000B1
:10CC100002EB8202B0EB420F0DDB90FBF1F0401C07
:10CC2000C1B284F86D106D2004F0A2FD94F86D106F
:10CC3000022013F030F80120FFF792F99BF8110061
:10CC400040F001008BF81100304880F80090BBF8EC
:10CC50002000602818D01DE094F86C20B5F9000081
:10CC600002EB8202B0EB420FE5DB90FBF1F0401CDF
:10CC7000C1B284F86C106C2004F07AFD94F86C104A
:10CC8000012013F008F8D6E7297884F860106020B6
:10CC900004F06EFDBBF820006F280DD194F86F00F2
:10CCA0009BF81310884207D204218BF8131084F8E4
:10CCB0009B109B2004F05CFDBBF82000922811D152
:10CCC000B5F9000012490840012838D0032086F841
:10CCD0002B0084F892900021922004F049FD04205A
:10CCE0008AF8000016E000002800002072110020E1
:10CCF000130300201C6D00207C020020680200202D
:10CD0000007700081C03002050160020730000204C
:10CD100001000080BBF8200082280ED1B5F9000088
:10CD200001281ED0022823D00021822004F020FDFB
:10CD300084F8829009208AF80000BDE8F09F86F808
:10CD40002B9084F8927012F04FF8002016F088FFB4
:10CD50000121922004F00CFD0021822004F008FD46
:10CD6000C0E70121822004F003FD84F88270E1E72E
:10CD70000221822004F0FCFC84F88280DAE770B59E
:10CD800086B005F0B8FEFE4CFE4D03AA218C6B4622
:10CD90005E2902D1207D012820D095292BD09B2906
:10CDA00036D000205E3901EB810105EB81010D5C7D
:10CDB00015540D18AD7A1D54401CC0B20A28F6D384
:10CDC000012005F079FE694603A806F030F8EC4929
:10CDD000208CED4A1E315E2827D037E0002029182C
:10CDE00091F84C64165491F856141954401CC0B272
:10CDF0000A28F4D3E4E70020291891F86064165457
:10CE000091F86A141954401CC0B20A28F4D3D7E729
:10CE10000020291891F87464165491F87E1419545E
:10CE2000401CC0B20A28F4D3CAE7237D73B19379BA
:10CE300092F8D150AB4201D9957104E092F8CF50ED
:10CE4000AB4200D2957192790A800CE0832814D00D
:10CE50000A23722814D095281CD0822825D0922825
:10CE600027D0125C0A805E2805D1207D002802D1DF
:10CE7000C6480088088006B027E5227C0A80F2E7D1
:10CE800012F8995F527805EB022212B292FBF3F28C
:10CE90000A80E8E792F8595292F85A2205EB0222EA
:10CEA00012B292FBF3F20A80DDE792F882200A8048
:10CEB000D9E7B74A92F82B2012B100220A80D2E7B4
:10CEC00001220A80CFE7AE485E21027B002A0AD009
:10CED0000184AD4991F87F10032901D19521018486
:10CEE0000021017502E001840121017547E770B559
:10CEF000012005F0E1FD022005F0DEFDA049088CCF
:10CF0000942801D10A7B42B10D7B002463239E4A01
:10CF1000012D07D05E2816D019E05E20088401207C
:10CF2000087525E092F87F20032A02D00B840C7547
:10CF30001EE0952804D09B28F9D195200884F6E7B7
:10CF40009B200884F3E70D7D0DB10C7510E092F87D
:10CF50007F40042C0FD0602831D09223822830D01B
:10CF6000832836D0722836D0922837D0401C0884C7
:10CF7000BDE8704003E75E2806D0A0F16802022AEF
:10CF800005D2401C0884F3E769200884F0E76A288A
:10CF900006D0A0F16C02022A05D2401C0884E7E703
:10CFA0006C200884E4E7822801D10A7C22B16E2833
:10CFB000DED194200884DBE784200884D8E70B8442
:10CFC000D6E792F8830010B183200884D0E70B8461
:10CFD000CEE70B84CCE776200884C9E79320088449
:10CFE000C6E72DE9F041012005F066FD022005F0BD
:10CFF00063FD6349644E5E22087B88B196F87F002A
:10D00000032801D00A8427E0088C952802D09B28A9
:10D0100003D021E09B2008841EE0952008841BE0BB
:10D02000088C00235E2805D10C7D1CB19420088457
:10D030000B7511E05E2801D10C7D84B196F87F70EC
:10D0400082248325042F0DD0632830D0922831D03C
:10D05000762837D0401E0884BDE8F0418FE60120D5
:10D060000875F9E7682806D0A0F16902012A05D8F9
:10D07000401E0884F0E70A840B75EDE76C2806D0A3
:10D08000A0F16D02012A05D8401E0884E4E76A2059
:10D090000884E1E7942805D09228DDD1087C20B1EE
:10D0A0000D84D9E76E200884D6E70C84D4E760208D
:10D0B0000884D1E796F88300012801D00C84CBE7DF
:10D0C0000D84C9E774200884C6E77CB52C4C47F66C
:10D0D000196204F11E01208CB1F900104FF6FF73A4
:10D0E000772874D012DCA0F15E0019282DD2DFE879
:10D0F00000F0336E6E2C2C6EA0F36E6E2C2C6E6EC8
:10D100002C2C5A6E75756E2C6E2C6E0080285ED09D
:10D1100009DCA0F17800082817D2DFE800F0586A8F
:10D120005858585858FE94286CD008DC822874D07F
:10D13000832841D0922871D0932806D162E09B28A1
:10D140006DD0E52843D0E62841D002B02022BDE8CA
:10D150007040002005F0F0BC207D30B102B02022EC
:10D16000BDE87040002005F0E7BC074890F86E006D
:10D1700090B102B04622BDE8704000200AE00000F5
:10D18000280000203ED502081C6D0020620200200D
:10D190005016002005F0D0BC02B04322BDE870401C
:10D1A000002005F0C9BC41B1CDE90032F7A3C2228D
:10D1B0000021012004F0BEFE7CBDCDE90032F5A3C4
:10D1C000C2220021012004F0B5FE7CBDFFE702B0C1
:10D1D0002022BDE87040002005F0AEBC0A2091FB83
:10D1E000F0F002B001B2BDE870402022002005F04E
:10D1F000A3BCCDE90032E9A3C2220021012004F042
:10D2000099FEE2E7C8070BD0CDE90032E4A3C222C1
:10D210000021012004F08EFED7E747E066E011E030
:10D22000CDE90032DFA3C2220021012004F082FEFA
:10D23000CBE7CDE90032DCA3C2220021012004F0BB
:10D2400079FEC2E70529C0D2DFE801F0030C151E04
:10D250002700CDE90032D6A3C2220021012004F02C
:10D2600069FEB2E7CDE90032D2A3C222002101203B
:10D2700004F060FEA9E7CDE90032D0A3C22200216C
:10D28000012004F057FEA0E7CDE90032CDA3C22271
:10D290000021012004F04EFE97E7CDE90032CBA338
:10D2A000C2220021012004F045FE8EE701290AD0A8
:10D2B000022912D0CDE90032C6A3C22200210120EA
:10D2C00004F038FE81E7CDE90032C4A3C222002178
:10D2D000012004F02FFE78E726E0CDE90032C1A35B
:10D2E000C2220021012004F025FE6EE7BF48014064
:10D2F000012909D0CDE90032BDA3C22200210120BD
:10D3000004F018FE61E708E0CDE90032BAA3C222BA
:10D310000021012004F00EFE57E702B02022BDE8F4
:10D3200070405A2005F008BCC1B101291FD0022964
:10D3300026D003292DD0042934D005293BD0062935
:10D3400042D0072949D008298BD1CDE90032ACA3BE
:10D35000C2220021012004F0EDFD36E7CDE90032C4
:10D36000A9A3C2220021012004F0E4FD2DE7CDE9AC
:10D370000032A7A3C2220021012004F0DBFD24E734
:10D38000CDE90032A4A3C2220021012004F0D2FD85
:10D390001BE7CDE90032A2A3C2220021012004F044
:10D3A000C9FD12E7CDE900329FA3C222002101206E
:10D3B00004F0C0FD09E7CDE900329DA3C22200219F
:10D3C000012004F0B7FD00E7CDE900329AA3C222A4
:10D3D0000021012004F0AEFDF7E6CDE9003298A36C
:10D3E000C2220021012004F0A5FDEEE670B5964DA5
:10D3F000964C0026297894F87F000939122951D2D9
:10D40000DFE801F0090C505015180F1B12202550B1
:10D410003F4245484B4EFEF7F3FD43E0FEF758FE12
:10D4200040E0FEF7F4FE3DE0FEF71DFF3AE0FEF7B8
:10D4300091FF37E0FEF7E8FF34E0052832D0FEF731
:10D440002DFF2FE005282DD0FEF75AFF2AE005F02A
:10D4500052FBFFF738FD94F87F007D4C40B1042863
:10D4600006D0022808D0032806D0052804D019E0E9
:10D470002673FFF728FD15E0FFF725FD0120207337
:10D4800010E0FFF734FD0DE0FFF7ABFD0AE0FFF71A
:10D4900031F907E0FFF726F804E0FFF723FA01E08F
:10D4A000FFF720FA2E7070BD00218438694A0728E2
:10D4B00012D2DFE800F004060A080C0E1000918872
:10D4C0000AE0917908E0117A06E0D17904E0117858
:10D4D00002E0517800E0917808B2704710B503F08F
:10D4E000AAFF802004F021F803F0D2FF08B1002049
:10D4F00010BDFE2004F019F803F0CAFF08B10020A7
:10D5000010BD03F0AEFF012010BD10B5044603F0BE
:10D5100092FF802004F009F803F0BAFF08B1002060
:10D5200010BD3CB1F52004F000F803F0B1FF28B1C4
:10D53000002010BDF32003F0F8FFF6E703F091FFA1
:10D54000012010BD70B50E4603F075FF812003F079
:10D55000ECFF03F09DFF012004F008F84FF6FF7187
:10D5600001EA0025012004F001F840EA050400204A
:10D5700003F0FCFF03F075FF3480012070BD01F063
:10D580000203834268D00020704765E02D462D20BD
:10D59000000000002D432D20000000003441000059
:10D5A0004E4F00005945530031303020200000001C
:10D5B0004F6666004D6F6465310000004D6F646515
:10D5C000320000004D6F6465330000004175746FD8
:10D5D0000000000052533438350000005A494742D9
:10D5E00045450000204155544F00000001000080D7
:10D5F0004D4F4442555300004241434E45540000B4
:10D6000031343430302000003936303020200000F2
:10D6100031393230302000003338343030200000CF
:10D62000353736303020000031313532303020008F
:10D6300037363830302000003132303020000000E2
:10D640003438303020000000F80000201C6D00202D
:10D65000280000206811002021F0030150B140F2A1
:10D66000E2404143C81701EB104000143C381080E1
:10D67000012089E744F2A4404143C81701EB104060
:10D680000014A0F590504D3800B20A2190FBF1F043
:10D690001080EDE770B5054603F0CDFE812003F064
:10D6A00044FF03F0F5FE08B1002070BD012003F037
:10D6B0005DFF4FF6FF7101EA0024012003F056FFE1
:10D6C000204484B2002003F051FF03F0CAFE022D73
:10D6D0000AD044F2A4404443F9480A2100EB244014
:10D6E00090FBF1F080B270BD40F2E24044436FF035
:10D6F0003B0000EB2440F5E710B503F09CFE8020D2
:10D7000003F013FF03F0C4FE08B1002010BDE720B2
:10D7100003F00BFF03F0BCFE08B1002010BD03F0C6
:10D720008AFE812003F001FF03F0B2FE08B1002061
:10D7300010BD002003F01AFF044603F092FEE0B291
:10D7400010BD70B50646C1F1FA001EF0F2FF4FF0B1
:10D750003332DC4B1FF040F804460D4630461EF0D5
:10D76000E8FF22462B461EF065FD1EF0B3FF00B217
:10D7700070BD2DE9F047044608461FF023FCD2494E
:10D780001FF0EEFA1FF052FA1EF03AFB1EF020FDD9
:10D79000064620461EF0CDFFCC4F0D460446002223
:10D7A0003B461FF019F81EF013FD8146DFF8208379
:10D7B000DFF820A320462946424653461EF03AFD94
:10D7C00004460D4648461FF031FA22462B461EF00D
:10D7D000EDFD1EF0FDFC014630461FF053FA1FF030
:10D7E00025FA8946064600223B461FF029F90446E1
:10D7F0000D4630464946424653461EF0EDFF22464E
:10D800002B461EF0D3FD1EF065FF00B2BDE8F08789
:10D8100063214FF4607003F0ABBFAF498A88920771
:10D820000BD08A790D2A15D2DFE802F014393B3E7D
:10D830004144474A4D5053575B008A790D2A09D21B
:10D84000DFE802F00807090C0F1215181B1E21252E
:10D850002900C87998E6C8791F3095E6C8793B3029
:10D8600092E6C8795A308FE6C87978308CE6C87964
:10D87000973089E6C879B53086E6C879D43083E632
:10D88000C879F33080E6C87900F211107CE6C879D7
:10D8900000F5987078E6C87900F5A77074E6C87945
:10D8A00072E6C8791F306FE6C8793C306CE6C879FB
:10D8B0005B3069E6C879793066E6C879983063E606
:10D8C000C879B63060E6C879D5305DE6C879F430FD
:10D8D0005AE6C87900F5897056E6C87900F2311029
:10D8E00052E6C87900F24F104EE600B5FFF795FFFB
:10D8F0007A498883C0F3C70200F0070178481044D2
:10D9000000F22D40FDF760F908B1012000BD0020B4
:10D9100000BD2DE9F043724D704901266A7A714FBE
:10D92000CB7C4FF0040C02F0FE044FF000080528F9
:10D930000FD2DFE800F00E03101E2100CE7342F07C
:10D94000010068728E7481F813C081F804C0BE7142
:10D95000BE70BDE8F08381F80FC06C7281F8128050
:10D96000002BF6D081F8138081F80480BE71BE7060
:10D97000EFE70A20C873ECE70C20C8736C7281F8DB
:10D980001280002BE5D081F8138081F80480BE71ED
:10D99000BE70DEE710B5504A147A002C03D0127A1C
:10D9A000012902D002E00722FAE708224C490728A1
:10D9B0003AD2DFE800F039040D161F283100521E5C
:10D9C00002EB4200084490F8150400F007032BE036
:10D9D000521E02EB4200084490F81504C0F3C20343
:10D9E00022E0521E02EB4200084490F8160400F0B8
:10D9F000070319E0521E02EB4200084490F8160497
:10DA0000C0F3C20310E0521E02EB4200084490F83B
:10DA1000170400F0070307E0521E02EB420008441F
:10DA200090F81704C0F3C20358B210BD2DE9FC5F93
:10DA3000002711F0D9F92848007AE8B32648007A7F
:10DA4000401E00F0FF09FFF750FF274A00287CD056
:10DA5000264801784478C1EB011104EB8104244984
:10DA60000C808378C478C3EB031304EB83034B80EF
:10DA700003794479C3EB031304EB83038B8083792D
:10DA8000C479C3EB031304EB8303CB80037A447A9A
:10DA9000C3EB031304EB83030B81C37A807AC0EBDF
:10DAA000001003EB80004881002409EB490802EBD9
:10DAB0004805285DFF2800E01CE01ED054E000006F
:10DAC000B3EDFFFF3333C3BF00007A4400A0314001
:10DAD000CDCCCCCCCCFCA24068110020280000208A
:10DAE0001C6D002072110020A471002025710020FF
:10DAF000240900204FF00609A5E7FF494FF6FF7003
:10DB000021F8140008EB5400FC4A019010440090E6
:10DB100090F81504E10741D0C10801F0030119B3E1
:10DB2000E1073ED000F0C70AFF2109EB4900800061
:10DB300000EB440B0BEB020080F8B51380F8B61332
:10DB40000BF2B53003F014FE00E0DEE00BF2B6306D
:10DB5000FF2103F00DFE009880F815A401985146AE
:10DB600000F2154003F004FE641CE4B2062CA0D3BE
:10DB7000DFF88C9399F80000E8B30020DE4901F14A
:10DB80000E0231F8103022F81030401CC0B20628C6
:10DB9000F7D305244FF0000C00211FE000F0030133
:10DBA000BDE700F0F80ABFE7481C32F8113032F840
:10DBB00010A0534511D90127938132F8103022F873
:10DBC0001130938922F8103015F801A06B1893F8E2
:10DBD00001B005F801B083F801A0C1B2A142E3D3BE
:10DBE000641EE4B20CF1010C0CF0FF0CBCF1060F4A
:10DBF000D2D3002000E001E089F80000CFB3002478
:10DC0000BE4F08EB5402D31993F81514E00706D061
:10DC1000285D012817D0D8B1FF281ED01FE0285D4D
:10DC2000012803D038B1FF280AD018E001F0F8002D
:10DC300040F0010113E001F0F80040F002010EE0B5
:10DC400001F0F8010BE001F0C70040F0080106E028
:10DC500001F0C70040F0100101E001F0C70183F8B6
:10DC6000151402F2154003F083FD641CE4B2062C87
:10DC7000C7D3A44841780078C0EB001001EB8004C2
:10DC80009D4D0E352888A04207D86888A04204D947
:10DC900001210846FFF77EFEC6B26888A04207D879
:10DCA000A888A04204D901210220FFF773FEC6B262
:10DCB000A888A04207D8E888A04204D901210320FF
:10DCC000FFF768FEC6B2E888A04207D82889A042BC
:10DCD00004D901210420FFF75DFEC6B22889A042C5
:10DCE00007D86889A04204D901210520FFF752FE18
:10DCF000C6B26889A04204D801210620FFF74AFE77
:10DD0000C6B23046BDE8FC5F03E67C4809EB490833
:10DD100000EB880000F2B53001784478C1EB0111C6
:10DD200004EB810474490C808378C478C3EB03133B
:10DD300004EB83034B8003794479C3EB031304EBB7
:10DD400083038B808379C479C3EB031304EB8303D0
:10DD5000CB80037A447AC3EB031304EB83030B8178
:10DD6000C37A807AC0EB001003EB80004881002466
:10DD700002EB4805285DFF2832D15F484FF6FF715E
:10DD800020F814102146484611F01EF8E10741D052
:10DD9000C10801F0030119B3E1073ED000F0C70A42
:10DDA000FF2109EB4900800000EB440B5348584425
:10DDB00080F8B51380F8B6130BF2B53003F0D8FC39
:10DDC0000BF2B630FF2103F0D3FC4C4908EB5400B2
:10DDD000014481F815A400F21540514603F0C8FC37
:10DDE000641CE4B2062CC5D3DFF8149199F8000046
:10DDF000E8B30020404901F10E0231F8103022F85A
:10DE00001030401CC0B20628F7D305244FF0000C98
:10DE100000211FE000F00301BDE700F0F80ABFE7B2
:10DE2000481C32F8113032F810A0534511D901279F
:10DE3000938132F8103022F81130938922F8103093
:10DE400015F801A06B1893F801B005F801B083F83C
:10DE500001A0C1B2A142E3D3641EE4B20CF1010CF3
:10DE60000CF0FF0CBCF1060FD2D3002000E001E063
:10DE700089F80000CFB30024204F08EB5402D319D7
:10DE800093F81514E00706D0285D012817D0D8B103
:10DE9000FF281ED01FE0285D012803D038B1FF28DD
:10DEA0000AD018E001F0F80040F0010113E001F0A1
:10DEB000F80040F002010EE001F0F8010BE001F083
:10DEC000C70040F0080106E001F0C70040F0100173
:10DED00001E001F0C70183F8151402F2154003F0C8
:10DEE00047FC641CE4B2062CC7D30648417800788E
:10DEF000C0EB001008E00000240900201C6D002089
:10DF0000280000206811002001EB8004424D288881
:10DF1000A04207D86888A04204D900210120FFF759
:10DF200039FDC6B26888A04207D8A888A04204D9A3
:10DF300000210220FFF72EFDC6B2A888A04207D814
:10DF4000E888A04204D900210320FFF723FDC6B2D0
:10DF5000E888A04207D82889A04204D900210420DB
:10DF6000FFF718FDC6B22889A04207D86889A042E9
:10DF700004D900210520FFF70DFDC6B26889A04233
:10DF800004D800210620FFF705FDC6B23046FFF792
:10DF9000C0FC99F80200864204D020490120087193
:10DFA0008870487089F80260BDE8FC9FF0B50346B0
:10DFB0001B48194CC5180E3495F86702FF2824D069
:10DFC000002658B1411E012705290BD2C9B21548B8
:10DFD000FCF7FAFD012803D0E65416E0E65414E0FD
:10DFE000E75412E01049062806D1B1F90020002AB2
:10DFF00001DDE75400E0E654072806D1B1F902003C
:10E00000002801DDE75400E0E65495F86702002897
:10E0100001D16420E054F0BD3209002072110020CB
:10E020001C6D002094020020BE0000202DE9F0416C
:10E03000FB4C0023A370E370FB4D3C24F94F1826E2
:10E0400005EB8203002904D0012939D0022968D1C7
:10E0500057E0B0FBF4F104FB110197F802C06144F2
:10E06000C9B2B1FBF4FCB1FBF4F804FB1811D97090
:10E07000B0FBF4F104FB1101401A80B2B0FBF4F0E4
:10E08000B0FBF4F104FB1101614497F801C0614455
:10E09000C9B2B1FBF4FCB1FBF4F804FB18119970A0
:10E0A000B0FBF4F0397860440844C0B2B0FBF6F13C
:10E0B000B0FBF6F406FB1400587005F8221030E0AF
:10E0C000B978D970B0FBF4F104FB110197F801C0E5
:10E0D0006144C9B2B1FBF4FCB1FBF4F804FB1811C4
:10E0E0009970B0FBF4F0397860440844C0B2B0FBDA
:10E0F000F6F1B0FBF6F406FB1400587005F8221098
:10E100000FE0B978D9707978997039780844C0B23D
:10E11000B0FBF6F1B0FBF6F406FB1400587005F8FE
:10E120002210D8783B2801D13A20D870BDE8F08180
:10E1300010B5BB4BBC49BB4A002814D011F8204095
:10E14000DB789C422FD101EB800013784178994213
:10E1500027D181785378994221D1C078917888422B
:10E160001BD8012010BD08789B78984213D14878BD
:10E17000137898420DD188785378984207D1C8789F
:10E180009178884201D8012010BD002010BD0020E8
:10E1900010BD002010BD002010BD002010BD0020CB
:10E1A00010BD002010BD002010BD2DE9F14FDFF89B
:10E1B000708298F80C0001285AD10024814608F199
:10E1C0003E0B4FF0000A08F11A06984F4DE0651C0F
:10E1D000E8B2FFF7ADFF012801D1315D11B101288F
:10E1E0002CD041E097F8DB00032813D017F8CB0FB1
:10E1F000797800EB012080B2A8F8240006F804909A
:10E20000397ACB3F0122FFF711FF97F8DB00022894
:10E210000DD029E006F80490EAB23BF81400002182
:10E22000FFF704FF7E483B3000F80490EDE706F866
:10E2300004A088F80AA088F80CA015E0305D012839
:10E2400012D197F8DB00032814D017F8CD0F797896
:10E2500000EB012080B2A8F8240006F804A0B979E8
:10E26000CD3F0122FFF7E2FEECB200988442AED32C
:10E27000BDE8F88F6A48423030F8140030B106F833
:10E2800004A0EAB20021FFF7D1FEEDE7EAB23BF8C5
:10E2900014000021FFF7CAFEE6E7D21C884205D130
:10E2A000D1B25F4800221830FCF781BCD1B25C4883
:10E2B00001221830FCF77BBC10B50446002903D0BE
:10E2C000574900203231085555480122214618305F
:10E2D000FCF76DFCE41CE1B251480022BDE810409F
:10E2E0001830FCF764BC10B504464D482630015D7B
:10E2F0004F48005D821C91420DD9494800222146B9
:10E300001030FCF754FC214645480122BDE810407E
:10E310001230FCF74CBC801E81420DDA40480122CD
:10E3200021461030FCF743FC21463D480022BDE861
:10E3300010401230FCF73BBC394800222146103017
:10E34000FCF735FC214636480022BDE8104012306B
:10E35000FCF72DBC2DE9F04F89B00446334EDFF8B1
:10E36000C09096F86B00002807D0012844D0314FA8
:10E3700002287ED0032810D1AAE099F805000628CB
:10E380000CD096F8A903022815D0012813D02046F6
:10E39000FFF7A9FF0120FFF7A6FFC1E020480122F7
:10E3A00000211030FCF703FC1D48002211461230FA
:10E3B000FCF7FDFBB4E00120FFF795FF96F8A903F9
:10E3C00002280CD01648012200211030FCF7EFFB88
:10E3D0001348002211461230FCF7E9FBDAE7104837
:10E3E000002211461030FCF7E2FB0D48012200210B
:10E3F0001230FCF7DCFBCDE70120FFF774FF99F842
:10E400000400C8B10648002211461030FCF7CFFBCB
:10E410000348012200211230FCF7C9FB17E028E075
:10E420007200002068110020490900201C6D0020A6
:10E43000BF030020C803002001220021FE48FCF792
:10E44000B6FBFD4800221146801CFCF7B0FB99F892
:10E450000B0070B3401E89F80B0000221146F648ED
:10E46000FCF7A5FBF44800221146801CFCF79FFB3B
:10E4700056E096F89F02052804D096F89E020528DB
:10E4800007D00AE07888012801D0002505E00125A1
:10E4900003E0388801280DD000256DB10022114617
:10E4A000E548FCF784FBE44801220021801CFCF7CE
:10E4B0007EFB35E00125F0E701220021DE48FCF774
:10E4C00076FBDD4800221146801CFCF770FB27E03C
:10E4D0000221DA48FCF778FB10B9012089F807001F
:10E4E00096F89F02052804D096F89E02052807D0CA
:10E4F0000AE07888012801D0002505E0012503E025
:10E50000388801285DD00025F5B301220021CA48D2
:10E51000FCF74DFBC84800221146801CFCF747FB66
:10E52000A020A0EB4407C548C349D438C44AC05D05
:10E53000253104EB440B02EB4B08002628B30628D8
:10E5400056D010F808000855C81C12F81B200255B8
:10E55000DFF8E4A20AF1160A0AF10F011AF8040022
:10E56000095D0AF10905884204D305F10901095D35
:10E57000884224D9B148D43890F87900022801D0D3
:10E5800004283DD8214601E01DE028E0B9F812003A
:10E59000FCF7FCFA30B1A8481AF804102830005DE6
:10E5A00081420CD32146B9F81000FCF7EFFA38B3DA
:10E5B000A1481AF804102530005D814220D92E555B
:10E5C00069E10125A0E7002211469B48FCF7EFFA1C
:10E5D000994801220021801CFCF7E9FAA0E796483F
:10E5E000642228300255964810F81B000855AFE702
:10E5F0000E55934810F81B208F4828300255A7E786
:10E600002146B9F81000FCF7C1FAD0B30021A120CF
:10E610008A4AA0EB4400D43ADFF824E2105C05AB50
:10E6200008E0D25D01EB4B0C724412F80C205A54F6
:10E63000491CC9B2814AD43A8842F2D80022C0F1BA
:10E64000060C06E003EB020B022100F80B10521C33
:10E65000D2B29445F6DC1AF804004FF0030E0328FA
:10E6600002D802460AF804E01AF804009DF819C01E
:10E67000CDF820C0ACF1020C604503DA0621295523
:10E680001BE06FE09DF81410884201D92E5514E06C
:10E69000002103EB010B9BF801B0584509D913F891
:10E6A00001B0ABF1020B584503DA01F1010B05F89B
:10E6B00004B0491CC9B20429EBD39DF814108B1E79
:10E6C000984207DB884205D8295D012902D009B1AB
:10E6D000012129559DF815108B1E984208DB8842B0
:10E6E00006D8295D012903D0022901D0022129552C
:10E6F0009DF816108B1E984208DB884206D8295DCB
:10E70000022903D0032901D005F804E09DF8171071
:10E710008B1E984208DB884206D8295D032903D066
:10E72000042901D0042129559DF818108B1E984208
:10E7300008DB884206D8295D042903D0052901D0C9
:10E7400005212955604509DB0899884206D8295DCD
:10E75000052903D0062901D006212955032801D116
:10E760000AF804202146B9F81200FCF70FFAE8B3C2
:10E770000020324905AAD439C95D04E018F80030F8
:10E780001354401CC0B28142F8D800206623C1F166
:10E79000060705E002EB000C01F80C30401CC0B28B
:10E7A0008742F7DC9DF819701AF8040007F1020C93
:10E7B000604502D90C21295514E09DF814108842B7
:10E7C00001D22E550EE0002153185B78984205D2F5
:10E7D000535C9B1C984201D9CB1D2B55491CC9B2D7
:10E7E0000429F1D39DF81410884200E053E008D3C7
:10E7F000891C884205D8295D072902D009B1072163
:10E8000029559DF81510884209D3891C884206D8DD
:10E81000295D072903D0082901D0082129559DF831
:10E820001610884210D3891C88420DD8295D08290A
:10E830000AD0092908D005E082000020F06D0020F0
:10E8400055090020092129559DF81710884209D340
:10E85000891C884206D8295D092903D00A2901D0DC
:10E860000A2129559DF81810884209D3891C88422D
:10E8700006D8295D0A2903D00B2901D00B2129557F
:10E88000B84208D3604506D8285D0B2803D00C2871
:10E8900001D00C202855FE4F0DF11C0A385D0AF8F6
:10E8A00004002146B9F81800FCF770F978B1214648
:10E8B000B9F80E00FCF76AF948B9385DB8B1401CE8
:10E8C0003855F348002221461A38FCF770F904F154
:10E8D000030808F0FF01B9F81800FCF757F970B306
:10E8E0002146B9F80E00FCF751F9D8B127E0285DB0
:10E8F000062805D92146B9F81600FCF747F970B18A
:10E90000285D401E0628DCD22146B9F81400FCF729
:10E910003DF90028D5D1385D401C3855D1E7072096
:10E920003855CEE7385D072815D008B1401E385558
:10E93000D74808F0FF0100221A38FCF738F9285DA3
:10E940000D286ED2DFE800F06D091E3A586E8BA4D8
:10E95000B8D5F6EFEE003E55EAE7385D401E0628D2
:10E960000BD2CB48002221461A38FCF720F9385D3B
:10E9700022460121FFF791FC2EE101212046FFF7FD
:10E980009BFC29E1385D811E05290BD2C04800227D
:10E9900021461A38FCF70BF9385D22460221FFF7B1
:10E9A0007CFC19E1012804D001212046FFF784FCFA
:10E9B00012E100212046FFF77FFC0DE1385DC11E0A
:10E9C00004290BD2B248002221461A38FCF7EFF88E
:10E9D000385D22460321FFF760FCFDE0022806D0E7
:10E9E000012804D001212046FFF766FCF4E0002155
:10E9F0002046FFF761FCEFE0385D011F03290BD2D1
:10EA0000A348002221461A38FCF7D1F8385D224687
:10EA10000421FFF742FCDFE001212046FFF74CFC18
:10EA2000DAE0C0E0385D411F02290BD2984800228D
:10EA300021461A38FCF7BBF8385D22460521FFF75E
:10EA40002CFCC9E0401E032804D800212046FFF713
:10EA500033FCC1E001212046FFF72EFCBCE0385D0D
:10EA6000062807D0401E04280DD800212046FFF7B5
:10EA700023FCB1E08648002221461A38FCF797F8BB
:10EA800006203855A8E001212046FFF715FCA3E039
:10EA9000385D06280BD97E48002221461A38FCF73B
:10EAA00086F8385D22460721FFF7F7FB94E0012145
:10EAB0002046FFF701FC8FE0385D07280DD9744828
:10EAC0004FF000022146A0F11A00FCF770F8385D03
:10EAD00022460821FFF7E1FB7EE005D14FF000015F
:10EAE0002046FFF7E9FB77E001212046FFF7E4FB32
:10EAF00072E0385D08280DD965484FF000022146C4
:10EB0000A0F11A00FCF753F8385D22460921FFF7FF
:10EB1000C4FB61E009D0072807D001212046FFF798
:10EB2000CBFB59E02EE019E004E000212046FFF77E
:10EB3000C3FB51E0385D09280BD955480022214616
:10EB40001A38FCF734F8385D22460A21FFF7A5FB96
:10EB500042E000212046FFF7AFFB3DE0385D0A2888
:10EB60000BD94B48002221461A38FCF720F8385DB3
:10EB700022460B21FFF791FB2EE000212046FFF7F4
:10EB80009BFB29E0385D0B2808D94148002221462B
:10EB90001A38FCF70CF80C2038551DE000212046EF
:10EBA000FFF78AFB18E03A48002221461A38FBF7A3
:10EBB000FEFF385D38B1364808F0FF0101221A38EF
:10EBC000FBF7F5FF08E0285D3855314808F0FF01F4
:10EBD00000221A38FBF7EBFF1AF80400395D88426F
:10EBE00019D02B49012009310870487088702848D5
:10EBF000012221462438FBF7DAFF0A2089F80000B9
:10EC00000220CDE9000602960023642221A12448B7
:10EC1000039608F00CFC385D30BB1AF80400DFF8EE
:10EC20007080411EA8F10608A8F1030A06291CD22B
:10EC3000DFF870B09BF8660048B101222146A8F1C8
:10EC40001800FBF7B4FF9BF8660008F804009BF877
:10EC5000670048B10E48012221461C38FBF7A7FF88
:10EC60009BF867000AF804002AE0072828D3DFF899
:10EC700034B09BF8660048B10548012221461C3893
:10EC8000FBF795FF9BF866000AF804000CE0000013
:10EC9000A40000205374617465537769746368003D
:10ECA00059AA00081C6D00209BF8670040B10122A2
:10ECB0002146F948FBF77BFF9BF8670008F8040042
:10ECC00099F8010000280ED1A9F81860A9F814607D
:10ECD000A9F816602878072800D32E70285D3855CB
:10ECE000012089F8010009B0BDE8F08F2DE9FF4F40
:10ECF00081B081464D460024DFF8A083DFF898B349
:10ED000008F1D6000BF1270BA246009084B198F8C9
:10ED1000CD0098F8CE1000EB0126049800F00F010A
:10ED20000398052919D2DFE801F00D0F1113170020
:10ED300098F8CB0098F8CC1000EB01260298010956
:10ED40004846EEE7002508E0642506E0054604E0B5
:10ED5000322101EB500500E04508CF480830055549
:10ED6000002739460098FBF72FFF012807D108EB51
:10ED7000070090F8B910032901D190F88B511CB10C
:10ED80007F1CFFB2052FECD398F8D310012902D0D5
:10ED9000022904D006E0C6EB0610860002E04FF41C
:10EDA00061604643642206FB05F0B0FBF2F0BA4F07
:10EDB00080B22A3727F81400C5F164037343B3FB0C
:10EDC000F2F23B1D23F8142088B185B11BF8042012
:10EDD000012A0CD1A3F1420201261673621CD2B2A1
:10EDE000FFF724F9A7F1240006550BF804A037F823
:10EDF000140000B11DB9A848801D00F804A0641CCF
:10EE0000E4B2022C82D305B06EE72DE9F34F81B056
:10EE10000027DFF884A2DFF88892DFF880B20AF1D9
:10EE20001E0A0BEB0700009010F8B74F007B072875
:10EE300014D002987900005DC84000F00300022C55
:10EE40000ED24FF0A001A1EB44011BF801604FF07E
:10EE5000A101A1EB44011BF8018006E00198EEE757
:10EE600003D19BF89C609BF89D808E49097801290D
:10EE70000CD19BF8B710012901D107B902209BF8EA
:10EE8000B810012902D1012F00D1022030B1012890
:10EE90007ED0022804D0032801D164E00025CDE013
:10EEA0007D487D4912302131005D095D884235D2AF
:10EEB00016B91AF80410E9B11AF8041004EB440565
:10EEC000494406EB4502114411F8011C081A4FF49D
:10EED0007A71FBF759FE09EB450106EB0802114474
:10EEE00011F8011C90FBF1F54FF47A70854200D9BE
:10EEF0000546A3E004EB440508EB4501494411F83D
:10EF0000011C081A4FF47A71FBF73EFE09EB45012C
:10EF1000414411F8011C90FBF1F5E5E75E4924310D
:10EF2000095D88421DD91AF8041004EB44056FF0FE
:10EF30000602494402EB4502895C401A4FF47A719B
:10EF4000FBF722FE09EB4501314411F8011CC1F128
:10EF5000640190FBF1F5B5F57A7F6FD94FF47A75BE
:10EF60006CE000256AE04C484B4912302131005DCD
:10EF7000095D884239D20EB31AF8041004EB440537
:10EF8000494406EB4502114411F8011C081A00E03F
:10EF900052E04FF47A71FBF7F7FD09EB450106EB00
:10EFA0000802114411F8011C90FBF1F505F5FA7502
:10EFB0004FF47A70854241D905463FE01AF80410B3
:10EFC00004EB4405494408EB4502114411F8011CC7
:10EFD000081A4FF47A71FBF7D7FD09EB450141445C
:10EFE00011F8011C90FBF1F5E0E72B492431095D94
:10EFF00088421FD91AF8041004EB44056FF006028A
:10F00000494402EB4502895C401A4FF4FA71FBF760
:10F01000BBFD09EB4501314411F8011CC1F164014C
:10F0200090FBF1F505F5FA754FF47A70854205D934
:10F03000054603E0002501E04FF47A75009890F84A
:10F04000C300072830D002984021B940005D084035
:10F0500000B31148104912302131005D095D88422A
:10F060003BD2C6B11AF8041004EB4404494406EB41
:10F070004402114411F8011C081A4FF4FA71FBF70D
:10F0800083FD09EB440108EB0602114411F8011C51
:10F0900090FBF1F545E009E0860000201C6D0020A2
:10F0A00055090020430200200020D1E71AF804107F
:10F0B00004EB4404494408EB4402114411F8011CD8
:10F0C000081A4FF47A71FBF75FFD09EB44014144E4
:10F0D00011F8011C90FBF1F523E0F749095D884226
:10F0E0001ED91AF8041004EB44056FF006024944D7
:10F0F00002EB4502895C401A4FF4FA71FBF744FDBC
:10F10000A021A1EB44014FF0FF321BF8011002EBEC
:10F1100045024944895CC1F1640190FBF1F500E0CE
:10F1200000254FF47A70854200D90546009890F882
:10F130007B0011280DD0022817D003281FD00428E7
:10F140002FD028461DF056FFDC497A1D01EB8211B5
:10F1500048627F1CFFB2022FFFF463AE9BF8C3002E
:10F160000022D749022826D027E068081DF042FF78
:10F170000146D24A781D02EB80104162E9E705EBB7
:10F1800085000621B0FBF1F0C8301DF033FFCB49FC
:10F190007A1D01EB82114862CA4A9042D9DD4A6267
:10F1A000D7E7C5F57A701DF025FFC4497A1D01EB3C
:10F1B00082114862CDE70B881BB1032804D148882F
:10F1C00010B9BE48C0F864219BF8C400022801D1E0
:10F1D0000B8823B1032805D14888002802D1B748FD
:10F1E000C0F8A421BDE8FE8F30B5B749062813D07A
:10F1F00091F87C10B44A4C1F642392F85E0392F895
:10F200005D23801A0C2C32D2DFE804F009111919A1
:10F21000191919191919222691F87B10EAE7AB4937
:10F22000B1F90010484390FBF3F000B230BDA8499B
:10F23000B1F90010484390FBF3F000B230BDA04A92
:10F24000C91F32F91110484390FBF3F000B230BDF2
:10F25000A048B0F9000030BD9F49098809B2891A59
:10F260004FF47A72514391FBF0F000B230BD0020B0
:10F2700030BD2DE9F04F8BB0002501959748994995
:10F28000914F02789648002A06D097F86C200280A9
:10F2900097F86D00088005E097F87120028097F8D4
:10F2A0007000088000242046FFF754F8641CE4B284
:10F2B000032CF8D38048DFF800A23838AAF1060AF8
:10F2C000007A01280BD197F8A0008AF8000097F87F
:10F2D000C800C0EB00108100AAF1320041847A49D5
:10F2E0009AF8000001F51C72734E01F5B0710E36EC
:10F2F000CDE90912DFF8F091DFF8F0B1A6F12008AE
:10F30000062828D899F80010C319C1EBC10202F2EF
:10F3100003129A5C3280D1B10999415C059117F8CA
:10F32000A01F084498F8001010F80B00401A642140
:10F33000FBF72AFC797817F8A029114411F80B1073
:10F3400090FBF1F0C4B2642C2ED964242CE00A990D
:10F35000415C0591E3E799F80010C1EBC102131875
:10F3600097F8A120C2F106029B1A3B4493F803319F
:10F370003380E9B3811A394491F8601105915B49F2
:10F3800098F80020891F405C6421101AFBF7FCFBF1
:10F3900097F8A01011F80B10C1F1640190FBF1F087
:10F3A000C4B2642C00D964244348DFF840A1801F14
:10F3B0000AF1060A4078062832D899F8001041B3BD
:10F3C0004B49415C71800999415C039117F89E1F7C
:10F3D000084498F8011010F80A00401A6421FBF75D
:10F3E000D3FB797817F89E29114411F80A1000E030
:10F3F00009E090FBF1F000F0FF0BBBF1640F35D991
:10F400004FF0640B32E0811A394491F87012059183
:10F41000B5E73849415C71800A99415C0391D5E7B1
:10F4200099F80010F1B397F89F10C1F10601411A45
:10F43000394491F82621728091F86011039198F86F
:10F44000011010F80B00081A6421FBF79DFB97F8D8
:10F450009E1011F80A10C1F1640190FBF1F000F068
:10F46000FF0BBBF1640F01D94FF0640B12481F4929
:10F47000801F0C318078089106284ED899F800102A
:10F48000C9B11C493331415CB18017F89C1F01445C
:10F490000898085C98F80210401A6421FBF774FB86
:10F4A000387800E028E079789C3F01440898085CAF
:10F4B000B4FBF0F04DE02CE0AA0000200472002024
:10F4C000F011002000007A441C6D00206202002030
:10F4D00054000020600200205C0200203A0000205E
:10F4E000C4030020C60300203B0000205409002074
:10F4F000426E0020FB6F002097F89F10C1F10601BB
:10F50000411A394491F8DF22728091F87012039108
:10F5100095E7FC49415CB180B7E799F8001041B329
:10F5200097F89D10C1F10601411A394491F8121360
:10F53000B18098F8021010F80A00081A6421FBF74D
:10F5400023FB97F89C200899515CC1F1640190FB62
:10F55000F1F097F8DB00DFF8B0A3C0B30121002081
:10F5600002AA052816DA3B1893F8B930032B0AD003
:10F5700019E097F89D10C1F10601411A394491F83C
:10F580002013B180D5E7012902D0012150540AE0AF
:10F590000021FBE73B1893F87630112B03D10129AA
:10F5A00065D001215054401C00B20728D9DB9DF8DA
:10F5B00008001AF80000E8B39DF809001AF80000E6
:10F5C000C8B3039B5A4619465846FFF78FFB0024E1
:10F5D000DFF834B34FF0010A0BF1070BCA48005DA6
:10F5E000032861D004286BD00BF804001BF804003A
:10F5F000214636F81000FBF7C9FA0246C2482146F8
:10F600003238FBF7D4FA641CE4B2072CE6D3BE48C8
:10F61000BE4E52388079C0B3BB48523890F82000B3
:10F6200001900024381990F8B90001280DD0022863
:10F630000BD001E01DE030E0214601A8FBF7C4FA41
:10F640001DF0D8FC06EB84114862641CE4B2052C62
:10F65000E8D301210020DFF8B0B2ABF1380B052868
:10F6600060D23A1892F8B920032A48D068E0002105
:10F6700098E79DF809001AF8000038B15A4620466C
:10F68000039B0599FFF732FBA1E725E0059B224686
:10F6900019462046FFF72AFB99E722465846059B64
:10F6A0000399FFF723FB92E798F8000098F8011000
:10F6B000884202D20BF8045098E70BF804A095E7B3
:10F6C00098F8000098F80110884202D90BF804500D
:10F6D0008CE70BF804A089E700248B485238B0F877
:10F6E00020B02BFA04F000F001001DF083FC06EBC3
:10F6F00084114862641CE4B2052CF2D3A9E7012905
:10F7000008D001211BF80120012A05D006EB801248
:10F71000556215E00021F5E706EB80134FF07E52AD
:10F720005A620DE03A1892F87620112A08D1C9B130
:10F7300000211BF80120012A16D006EB8012556229
:10F74000401CC0B207288AD3002404F1B7000790F8
:10F7500002F00DF803280DD0079802F008F80428ED
:10F7600016D022E00121E4E706EB80134FF07E5231
:10F770005A62E5E798F8000098F80110884203D231
:10F78000381980F8B75010E0381980F8B7A00CE0AD
:10F7900098F8000098F80110884203D9381980F8C9
:10F7A000B75002E0381980F8B7A0641CE4B2022C0C
:10F7B000CBD35548DFF850A15238AAF1060A407958
:10F7C00080B1062829D0AAF11A021178062953D847
:10F7D00099F80000E0B34E48085C8DF8100004F082
:10F7E0000F0058E0BAF80000323000B2AAF800006A
:10F7F0004FF47A71884201DDAAF80050BAF802008D
:10F80000323800B2AAF80200002801DAAAF8021081
:10F810004FF4FA7008F014FC1AE197F8A6020428D5
:10F8200017D0AAF8005097F8A702042817D0AAF812
:10F830000250BAF900104FF47A70814201DDAAF843
:10F840000000BAF90210814201DDAAF80200FFE0CF
:10F850000BE00620FFF7C8FCAAF80000E3E707204A
:10F86000FFF7C2FCAAF80200E3E729480E30085C63
:10F870008DF8100020090EE099F80000E0B197F82B
:10F88000A100C0F10600081A384490F82D018DF847
:10F89000100004F00F0097F89F305178C3F1060371
:10F8A000CB1A06291AD899F800308BB1184BDB1DFA
:10F8B000C95C8DF8111019E0200997F8A130C3F147
:10F8C0000603C91A394491F83B118DF81010E2E78C
:10F8D0000C4B3A3BC95C8DF8111007E099F8001009
:10F8E000C1B1D91991F834118DF811109178062908
:10F8F0001BD899F800209AB1024A1A3A895C8DF80F
:10F9000012101FE03C700020C40000200472002090
:10F91000496E0020D91991F8E6128DF81110E5E72B
:10F92000B94A895C8DF812100CE099F80020F2B108
:10F9300097F89D20C2F10602891A394491F80613FE
:10F940008DF8121004A9FFF760FAB048052106905F
:10F95000FBF73AF9B0B197F8620397F86313000226
:10F9600000B208441DF02EFBC6F85C010DE097F8CC
:10F970009D20C2F10602891A394491F819138DF8B5
:10F980001210DFE7A248C6F85C0106210698FBF7D3
:10F990001BF958B197F8640397F86513000200B299
:10F9A00008441DF00FFBC6F89C0102E09848C6F819
:10F9B0009C01984CA07901284AD197F8B70004A976
:10F9C0004FF06409095CC1F3011149B101292CD040
:10F9D00004F13503DA1C022904D0032927D114E0ED
:10F9E000E58324E018F80010125C914203D9881ACC
:10F9F0004000E0831BE0185C814204D2C1F1320078
:10FA00004000E08313E0E58311E018F80010125C79
:10FA1000914201D9E1830AE0185C814203D2C1F12D
:10FA20006400E08303E0E58301E0A4F81E90072171
:10FA30000698FBF7C9F808B1607BE083B4F91E00B3
:10FA4000052801DAE58303E05F2801DDA4F81E90B4
:10FA50000024DFF8C481381990F8BE00012802D1D3
:10FA60006E49097861B1022802D1B8F8001039B1A5
:10FA7000032802D1B8F8021011B1042804D006E01E
:10FA800006EB841045622DE097F8DB1011B10528D4
:10FA90000AD00CE09BF80000012823D106EB84116A
:10FAA0004FF07E5048621DE097F8DB1011B1062838
:10FAB0000DD017E021465A48FBF786F89BF8001056
:10FAC00008401DF097FA06EB841148620AE097F8A7
:10FAD000DB00022806D14F48807A012802D106EBCC
:10FAE00084104562641CE4B2052CB4D30020DFF816
:10FAF00024914FF07E5899F809103A1892F8DC20BA
:10FB0000022A04D101291CD006EB80125562401C48
:10FB1000C0B20528F1D300243D4D002006EB84112E
:10FB200051F82020AA4217D051F8200010F0FF4FC2
:10FB30000CD0404514D1012221463948FBF72AF860
:10FB40000EE006EB8012C2F82480E0E70022214696
:10FB50003348FBF71FF803E0401CC0B21028DFD386
:10FB6000641CE4B2052CD8D399F80500002817D0FE
:10FB70000524002006EB841151F82020AA4207D06A
:10FB800051F820001DF0E2F9611F2AF8110003E08E
:10FB9000401CC0B21028EFD3641CE4B2072CE8D399
:10FBA0000BB0BDE8F08F1B4832300078011F0229EE
:10FBB00002D80A30C0B27047C11F022902D8C01E45
:10FBC000C0B27047A0F10A010229FAD8C01DC0B224
:10FBD000704770B50F4E0021308AFAF7D7FF044600
:10FBE0000A4DD63D95F8A10000B900240021708A85
:10FBF000FAF7CCFF28B1A41CE4B295F8A00000B934
:10FC00000024204670BD000035700020F26D0020F9
:10FC100000007F4372000020F01100203A00002015
:10FC200094020020B448016841F00101016041687C
:10FC3000B24A114041600168B14A11400160016857
:10FC400021F480210160416821F4FE0141604FF4FC
:10FC50001F0181607047A8490A6822F480320A6057
:10FC60000A6822F480220A60B0F5803F07D0B0F520
:10FC7000802F03D1086840F4A0200860704708680E
:10FC800040F48030086070470346002059099A4AC2
:10FC900001290AD002290AD0516A03F01F02012368
:10FCA00093400B4200D0012070471168F5E7116ABC
:10FCB000F3E718B5002000904FF4A0643120FFF75F
:10FCC000E3FF0099491C00910099A14201D000284E
:10FCD000F4D03120FFF7D8FF08B1012018BD002073
:10FCE00018BD854A116821F0F80141EAC000106092
:10FCF00070478449086070477F4B5A6822F47C1231
:10FD000008431043586070477E49086670477A4A36
:10FD1000516821F003010143516070477648406803
:10FD200000F00C007047744A516821F0F001014363
:10FD300051607047704A516821F4E061014351609D
:10FD400070476D4A516821F4605141EAC00050602B
:10FD50007047694A002903D0517A014351727047B4
:10FD6000517A8143517270476649D83108607047B3
:10FD7000614A516821F440410143516070475E4936
:10FD8000002220310A7001F82029012805D004281A
:10FD900002D1052081F820007047012081F8200061
:10FDA000704759490860704753490A6A02430A621A
:10FDB0007047554944390860704710B54E4A51683C
:10FDC00001F00C01514B002927D0042927D0082924
:10FDD00027D00360516801F0F00109094C4B5C5CCD
:10FDE0000168E1404160546804F4E064240A1C5D49
:10FDF00021FA04F48460546804F46054E40A1B5D3E
:10FE0000D940C160526802F44042920B404B1B1F24
:10FE10009A5CB1FBF2F1016110BD0360DAE70360A7
:10FE2000D8E7516801F47011536803F48033022459
:10FE300004EB914133B153689B0307D5354B5943CC
:10FE40000160C7E7334B59430160C3E72F4B594368
:10FE50000160BFE7284A002903D05169014351617D
:10FE600070475169814351617047234A002903D08B
:10FE70009169014391617047916981439161704734
:10FE80001D4A002903D0D1690143D1617047D1696E
:10FE90008143D1617047184A002903D0D1680143DA
:10FEA000D1607047D1688143D1607047124A002900
:10FEB00003D01169014311617047116981431161D8
:10FEC000704711494039086070470E49C86470474F
:10FED0000949C87170470848416A41F08071416220
:10FEE000704701460020044A92680A4200D001206F
:10FEF0007047014988727047001002400000FFF807
:10FF0000FFFFF6FE000042428004424200127A00E7
:10FF1000DE00002000093D0010B5FE4988420AD1EC
:10FF2000C41401212046FFF7B6FF2046BDE810406B
:10FF30000021FFF7B0BFB0F1804F0CD0F6498842E6
:10FF400013D101210220FFF7B1FF0021BDE81040CD
:10FF50000220FFF7ABBF01210846FFF7A7FF0021F2
:10FF6000BDE810400120FFF7A1BFEC49884209D14C
:10FF700001210420FFF79AFF0021BDE81040042072
:10FF8000FFF794BFE649884209D101210820FFF715
:10FF90008DFF0021BDE810400820FFF787BFE14931
:10FFA000884209D101211020FFF780FF0021BDE820
:10FFB00010401020FFF77ABFDB49884209D10121A8
:10FFC0002020FFF773FF0021BDE810402020FFF73D
:10FFD0006DBFD64988420AD1441401212046FFF75B
:10FFE0005AFF2046BDE810400021FFF754BFD0491A
:10FFF00088420AD10121CC042046FFF74CFF20465D
:020000040801F1
:10000000BDE810400021FFF746BFCA4988420AD127
:1000100001210C052046FFF73EFF2046BDE81040B9
:100020000021FFF738BFC44988420AD101214C059D
:100030002046FFF730FF2046BDE810400021FFF7C3
:100040002ABFBE49884209D101214020FFF72EFF77
:100050000021BDE810404020FFF728BFB849884282
:1000600009D101218020FFF721FF0021BDE81040C8
:100070008020FFF71BBFB34988420AD184150121B4
:100080002046FFF713FF2046BDE810400021FFF790
:100090000DBFAD4988420AD101210C042046FFF76B
:1000A000FAFE2046BDE810400021FFF7F4BEA74944
:1000B00088420AD101214C042046FFF7ECFE20467D
:1000C000BDE810400021FFF7E6BEA14988420AD1F1
:1000D00001218C042046FFF7DEFE2046BDE81040DB
:1000E0000021FFF7D8BE10BD30B50288894C8F4D76
:1000F000A0420DD0A8420BD0B0F1804F08D0864B63
:10010000984205D0854B984202D0854B984203D146
:1001100022F070034A881A43824B984206D0824BE1
:10012000984203D022F44073CA881A4302808A8816
:1001300082850A880285A0420AD0A84208D0824A55
:10014000904205D0814A904202D0814A904201D12A
:10015000097A01860121818230BD30B5028C22F0FE
:1001600001020284028C8388048B24F0700424F042
:1001700003050C882C4322F002020D8915434A889E
:100180002A43644DA8420BD0684DA84208D06E4D5A
:10019000A84205D06D4DA84202D06D4DA8420FD1A6
:1001A00022F008054A892A4322F004058A882A4356
:1001B00023F4807323F400738D891D43CB892B4373
:1001C00083800483C9888186028430BD70B5028C27
:1001D00022F010020284028C8388048B24F4E04411
:1001E00024F440760D884FF6FF7404EA0525354364
:1001F00022F020020E8904EA061616434A8804EA11
:1002000002123243434EB04202D0484EB04217D1A0
:1002100022F080024E8904EA0616164326F04006B4
:100220008A8804EA0212324323F4806323F40063D1
:100230008E8904EA86061E43CB8904EA830333438E
:1002400083800583C9880187028470BD70B5028CE4
:1002500022F480720284028C8388848B24F07004E0
:1002600024F003040D88254322F400720E894FF612
:10027000FF7404EA062616434A8804EA022232433F
:10028000244EB04202D0294EB04217D122F400666B
:100290004A8904EA0222324322F480668A8804EA08
:1002A0000222324323F4805323F400538E8904EA5C
:1002B00006161E43CB8904EA0313334383808583E8
:1002C000C9888187028470BD70B5028C22F4805287
:1002D0000284058C8288838B23F4E04323F44076E8
:1002E0000C884FF6FF7303EA0424344325F40055C9
:1002F0000E8903EA06362E434D8803EA0535354359
:10030000044EB04202D0094EB04226D122F48046BB
:100310008A891FE0002C01400004004000080040D2
:10032000000C004000100040001400400034014068
:10033000004C0140005001400054014000180040B2
:10034000001C0040002000400040014000440140EB
:100350000048014003EA8212324382808483C988C4
:10036000A0F84010058470BD828B22F44062828325
:10037000828B4FF6FF7303EA01210A4382837047A1
:10038000F0B5048C24F480540484868B048C4FF6DE
:10039000FF7505EA013726F4734605EA0222324367
:1003A00005EA03331343F74A90420ED0F64A9042CF
:1003B0000BD0B0F1804F08D0F44A904205D0F44AF7
:1003C000904202D0F34A904205D124F400513943BF
:1003D00041F4805104E024F402420A4342F4805183
:1003E00083830184F0BD828B22F00C028283828B96
:1003F0000A4382837047F0B5048C24F4807404842B
:10040000858B048C4FF6FF7707EA012625F0F3056C
:1004100007EA031313432B43DA4A90420ED0DA4A19
:1004200090420BD0B0F1804F08D0D84A904205D00E
:10043000D74A904202D0D74A904205D124F40071A5
:10044000314341F4807104E024F420620A4342F411
:10045000807183830184F0BD028B22F440620283A9
:10046000028B4FF6FF7303EA01210A4302837047B0
:10047000F0B5048C24F010040484068B048C4FF631
:10048000FF7505EA011726F4734605EA0333334383
:1004900005EA02221A43BB4B98420ED0BA4B98424F
:1004A0000BD0B0F1804F08D0B84B984205D0B84B74
:1004B000984202D0B74B984205D124F0200139432D
:1004C00041F0100104E024F0A0030B4343F01001BD
:1004D00002830184F0BD028B22F00C020283028BA6
:1004E0000A430283704770B5048C24F0010404842D
:1004F000058B048C25F0F3054FF6FF7606EA03130F
:1005000013432B439F4A90420ED09F4A90420BD0F8
:10051000B0F1804F08D09D4A904205D09C4A90424D
:1005200002D09C4A904205D124F002020A4342F0D4
:10053000010104E024F00A020A4342F001010383AE
:10054000018470BD70B505460C468E48854209D0C1
:100550008D48854206D0B5F1804F03D08B48854247
:1005600000D08B4820886188A288238958B104284C
:1005700011D0082817D02846FFF702FFE188284647
:10058000BDE87040F0E62846FFF7ADFFE188284659
:10059000BDE870409FE72846FFF76AFFE1882846DC
:1005A000BDE8704058E72846FFF725FFE188284658
:1005B000BDE8704017E72DE9F04107460C460025DD
:1005C00001266188002900D10225A288012A00D1D4
:1005D00002262088238988B13846FFF749FFE18841
:1005E0003846FFF739FF2389324629463846FFF758
:1005F0007AFFE1883846BDE8F0416CE73846FFF7FE
:1006000072FFE1883846FFF766FF238932462946A4
:100610003846FFF72DFFE1883846BDE8F0411BE77B
:1006200010B50A884B88CC881A438B8823431A4319
:100630000B891A434B8989891A430A43A0F844203D
:1006400010BD4FF6FF71818000210180C180418083
:10065000017270470021018041808180C180018149
:1006600041818181C1817047002101804180012247
:100670008280C1800181704700210180418081809A
:10068000C1800181418181817047002904D00188A6
:1006900041F0010101807047018821F001010180D2
:1006A0007047002905D030F8441F41F40041018013
:1006B000704730F8441FC1F30E0101807047002AD3
:1006C00003D082890A438281704782898A4382816A
:1006D0007047818270471143A0F848107047002A84
:1006E00003D082890A438281704782898A4382814A
:1006F0007047018921F0070101817047028922F0CA
:1007000070020A430281704700B503461846FFF79E
:10071000F5FF188940F00700188100BD70B50D463F
:1007200004461146602D0CD001222046FFF7DBFE67
:1007300029462046FFF7E2FF208940F0070020818C
:1007400070BD01222046FFF793FEF1E730B5048922
:10075000E4B24FF6FF7505EA032313430B4323432B
:10076000038130BD10B504462046FFF7EFFF208916
:1007700020F0070040F0070020F0700040F070000B
:10078000208110BD002C01400034014000040040D5
:1007900000080040000C004010B504462046FFF75A
:1007A000D5FF208940F480402081EAE701858282DC
:1007B0007047028822F070020A430280704770B5C9
:1007C0000589048B068C25F007050D434FF6FC4187
:1007D0000C4040F201110C4326F022064FF6FF7147
:1007E00001EA03111143314305810483018470BD83
:1007F000028B22F070020A4302837047028B22F4BC
:10080000E0424FF6FF7303EA012111430183704771
:10081000828B22F070020A4382837047828B22F41B
:10082000E0424FF6FF7303EA0121114381837047D1
:10083000002904D0018841F08001018070470188BF
:1008400021F0800101807047002904D0818841F0A7
:10085000040181807047818821F004018180704704
:10086000002904D0818841F0080181807047818887
:1008700021F0080181807047002904D0818841F06F
:10088000010181807047818821F0010181807047DA
:10089000028B22F008020A4302837047028B22F483
:1008A00000624FF6FF7303EA012111430183704791
:1008B000828B22F008020A4382837047828B22F4E3
:1008C00000624FF6FF7303EA0121114381837047F1
:1008D000028B22F004020A4302837047028B22F447
:1008E00080624FF6FF7303EA0121114301837047D1
:1008F000828B22F004020A4382837047828B22F4A7
:1009000080624FF6FF7303EA012111438183704730
:10091000028B22F080020A4302837047028BC2F3EB
:100920000E024FF6FF7303EA012111430183704762
:10093000828B22F080020A4382837047828BC2F34B
:100940000E024FF6FF7303EA0121114381837047C2
:10095000028C22F002020A4302847047028C22F0C9
:1009600008020A4302847047028C22F020024FF6EC
:10097000FF7303EA0111114301847047028C22F0D6
:1009800080024FF6FF7303EA01111143018470479F
:10099000028C22F400724FF6FF7303EA0121114327
:1009A00001847047028C22F400624FF6FF7303EA61
:1009B0000121114301847047028C22F400524FF64A
:1009C000FF7303EA013111430184704710B501231D
:1009D0008B40048C9C430484038C8A40134303841F
:1009E000CFE610B504238B40048C9C430484038C15
:1009F0008A4013430384C4E630B500F11803012490
:100A00008C40058CA5430584002911D008290FD0FE
:100A1000091FC1F34E001844016821F4E041016050
:100A200001684FF6FF7303EA02221143016030BDF3
:100A300003EB5100016821F070010160016811436E
:100A4000016030BD002904D0018841F0020101801D
:100A50007047018821F0020101807047002904D00D
:100A6000018841F0040101807047018821F00401F0
:100A700001807047002904D0818841F08001818085
:100A80007047818821F0800181807047028822F0C0
:100A90000802028002880A4302807047828822F09E
:100AA0007002828082880A4382807047028922F025
:100AB0000702028102890A4302817047028922F0FB
:100AC0008002028102890A43028170478184704753
:100AD000818570478186704701877047818770479D
:100AE000A0F840107047028822F440720280028809
:100AF0000A4302807047808E7047008F7047808F56
:100B00007047B0F840007047808C7047008D704788
:100B100002460020128A0A4200D001207047C943D1
:100B20000182704702460020138A0B4092890A40D6
:100B3000002B02D0002A00D001207047C943018257
:100B40007047000010B5E14988420AD101218C03A9
:100B50002046FFF7A0F92046BDE810400021FFF72E
:100B60009AB9DB4988420AD101214C042046FFF79B
:100B70009DF92046BDE810400021FFF797B9D549FF
:100B800088420AD101218C042046FFF78FF92046C4
:100B9000BDE810400021FFF789B9CF4988420AD14A
:100BA0000121CC042046FFF781F92046BDE8104022
:100BB0000021FFF77BB9C94988420AD101210C0500
:100BC0002046FFF773F92046BDE810400021FFF7EB
:100BD0006DB910BD30B585B004460D46208A4CF67F
:100BE000FF710840E98801432182A0894EF6F31184
:100BF0000840A9882A8911436A8902431143A181C7
:100C0000A08A4FF6FF410840A9890143A1826846A6
:100C1000FFF7D3F8AD48844201D1039800E0029871
:100C2000A189090408D500EBC00101EB0010296877
:100C30004900B0FBF1F007E000EBC00101EB001050
:100C400029688900B0FBF1F06422B0FBF2F10901E0
:100C50000B096FF018056B4300EB8300A3891D049B
:100C60004FF0320307D503EBC000B0FBF2F000F009
:100C70000700084306E003EB0010B0FBF2F000F0C1
:100C80000F000843208105B030BD4FF416510160BC
:100C900000218180C18001810C22428181817047C5
:100CA00010B5038A4FF2FF0213400A884C88224392
:100CB0008C88C9880C4322431A43028210BD00214C
:100CC000018041808180C1807047002904D08189E2
:100CD00041F4005181817047818921F40051818163
:100CE000704710B540F66A13C1F3421301F01F04B8
:100CF0000121A140012B07D0022B07D014303AB1BB
:100D000002680A43026010BD0C30F8E71030F6E7C5
:100D100002688A43026010BD002A03D0828A0A4317
:100D200082827047828A8A4382827047028A22F0D6
:100D30000F020282028A0A4302827047828922F4E9
:100D40000062828182890A4382817047002904D02F
:100D5000818941F0020181817047818921F002017E
:100D600081817047028A22F020020282028A0A43AD
:100D700002827047002904D0018A41F48041018237
:100D80007047018A21F4804101827047C1F3080154
:100D9000818070478088C0F308007047818941F0E6
:100DA000010181817047028BD2B20283028B42EA39
:100DB000012101837047028B02F47F420283028B80
:100DC0000A4302837047002904D0818A41F0200140
:100DD00081827047818A21F0200181827047002939
:100DE00004D0818A41F0100181827047818A21F00C
:100DF000100181827047002904D0818A41F00801E6
:100E000081827047818A21F0080181827047002920
:100E100004D0818941F40041818170478189C1F307
:100E20000E0181817047002904D0818A41F400615C
:100E300081827047818A21F4006181827047828AB1
:100E400022F004028282828A0A4382827047002949
:100E500004D0818A41F0020181827047818A21F0A9
:100E60000201818270470246002012880A4200D0A7
:100E7000012070478A05C9430180704770B500247E
:100E800040F66A12C1F3421301F01F05012606FA6B
:100E900005F2012B0CD0022B0DD0838A1340090AD6
:100EA0008E40008830400BB100B10124204670BD57
:100EB00083891340F3E7038A1340F0E740F66A1290
:100EC0000A0A01219140C94301807047003801405E
:100ED0000044004000480040004C004000500040EA
:100EE00010B50120FEF7EDFFBDE810400020FEF731
:100EF000E8BF2049086070471E49091F0860704715
:100F00001C498431086070471B4A118821F46071C4
:100F1000014311807047184A118821F07F01014375
:100F20001180704708B5144A2C3A1044009000987C
:100F3000016008BD08B510492C390844009000989C
:100F4000008808BD0B489C300068C0B270470A4852
:100F50000830018841F00101018070470548A03048
:100F60000068C0B2704704480830018841F00201AF
:100F70000180704704860D422C6C004010B50121A1
:100F80000C072046FEF792FF2046BDE810400021E6
:100F9000FEF78CBF214908627047204908617047FD
:100FA0001F4A116821F0E0010143116070471B499D
:100FB000A031086070471A4B1A6822F003020243FE
:100FC0001A601848026842F004020260012905D044
:100FD00020BF016821F004010160704730BFF8E7CD
:100FE0000F48016841F004010160016841F002010D
:100FF00001600C48016841F00401016030BF704796
:1010000001460020064A52680A4200D0012070477B
:1010100003490A6842EA80000860704700000E42F7
:101020000070004010ED00E07FB5B14CA088ADF835
:101030000C0048258DF80F5002268DF80E6003A98C
:101040002068F7F7F2FD208AADF808008DF80B5004
:101050008DF80A6002A9E068F7F7E7FDA08BADF80C
:1010600004008DF807508DF8066001A9A069F7F714
:10107000DCFD208DADF800008DF803508DF8026086
:101080006946606AF7F7D1FD7FBD70B5984D583D50
:10109000B5F85C10A86DF7F723FE964C18B32078CE
:1010A00020F004002070B5F86810686EF7F718FE9D
:1010B000F0B1207820F002002070B5F87410286F8D
:1010C000F7F70EFEC8B1207820F001002070B5F8C7
:1010D0008010E86FF7F704FEA0B1207820F0080038
:1010E0002070207870BD207840F004002070DAE78E
:1010F000207840F002002070DFE7207840F0010007
:101100002070E4E7207840F008002070E9E72DE93E
:10111000F047012006F074FFFFF7B7FF0446754E55
:10112000DFF8D481093E4FF0000770794FF00105D8
:1011300034EA000015D098F87F00032811D0F5702C
:101140006E48077098F8ED006D49C0EB00104FF63F
:10115000FF7202EA8000088018B101216948F7F7A0
:10116000D3FDF078684B012876D1717931EA04001B
:1011700072D098F87A0002286ED0F7706348057034
:10118000634A64201070B1716248077018780128B2
:101190000FD072784FF00D0C05204FF00E0962B39E
:1011A000012951D002293DD0042960D0082976D1E7
:1011B00069E03079172801D0182803D108290AD00E
:1011C000042908D001290DD0022908D004290CD007
:1011D00008290FD10CE01920B07237715FE0182098
:1011E000B07207E01720B07204E01620B07201E080
:1011F0001520B072B07A307151E001294FD0022928
:101200004DD0042902D0082949D105E086F80AC04A
:101210007570B570307042E086F80A907570B570E0
:1012200030703CE0B278012A04D0022A05D0032AAB
:1012300006D007E00A22B27204E01122B27201E085
:101240001222B27230702AE0B278012A05D0022A46
:1012500006D0032A07D008E032E00922B27204E087
:101260000F22B27201E01022B272307017E086F8DD
:101270000AC07570B278032A02D2521CB27000E024
:10128000B57030700BE086F80A907570B278012A5C
:1012900002D9521EB27001E00322B27030700429EC
:1012A00008D0082906D0022904D0012902D098F8D4
:1012B000790028B918480770F571B581174807708B
:1012C00074710C2C11D1187878B998F87F00012826
:1012D0000BD0032809D0307A411C31721E2802D964
:1012E0001320B0721D70BDE8F0873772FBE7000075
:1012F000D8DE0208F70000201C6D002066000020E8
:101300003E00002000080140690000206700002026
:101310006F000020700000206A0000207100002093
:1013200038B5A54C208FADF8000048208DF803009B
:101330006946606BF7F779FC218F606BF7F7E4FC87
:1013400038BD38B59C4C208FADF8000010208DF8CA
:10135000030003208DF802006946606BF7F765FC17
:10136000218F606BF7F7D0FC38BD08B50820ADF8C9
:10137000000010208DF8030003208DF8020069465C
:101380008E48F7F752FC08BD08B50820ADF80000FC
:1013900048208DF8030069468848F7F746FC08BDE9
:1013A000854A002803D0918D906AF7F7ADBC918DE6
:1013B000906AF7F7ABBC804A002803D0118F506BBE
:1013C000F7F7A2BC118F506BF7F7A0BC7A48018FDA
:1013D000406BF7F785BC7848818D806AF7F780BC51
:1013E000F8B5754C0121606AFEF73FFDA08DADF8A0
:1013F000000010258DF8035003268DF80260694621
:10140000A06AF7F712FCA18DA06AF7F77DFC012115
:10141000206BFEF72AFD208FADF800008DF80350F9
:101420008DF802606946606BF7F7FFFB218F606BF8
:10143000F7F76AFCF8BD10B5FFF783FF0120FFF74F
:10144000BAFF0120FFF7ACFF042006F0D9FD002011
:10145000FFF7B1FF042006F0D3FDBDE810400020E7
:101460009EE710B5FFF76DFF0020FFF799FF002002
:10147000FFF7A1FF042006F0C3FD0120FFF790FF56
:101480000120FFF798FFBDE81040042006F0B8BD2A
:1014900010B500240120FFF78EFFFFF741FF012068
:1014A00006F0AEFD0120FFF77BFF012006F0A8FD4E
:1014B00007E0641CA4B2FA2C03D9FFF7D2FF012085
:1014C00010BDFFF783FF0028F3D1FFF769FF00206D
:1014D00010BD10B50020FFF763FFFFF732FF0020BB
:1014E000FFF769FF022006F08BFD0120FFF758FF90
:1014F000022006F085FDBDE81040002050E710B541
:101500000020FFF74DFFFFF71CFF0120FFF753FFFF
:10151000022006F075FD0120FFF742FF022006F0D1
:101520006FFDBDE8104000203AE770B50546FFF7B3
:1015300008FF0020FFF734FF0024E809FFF73BFF16
:101540006806050E022006F05BFD0120FFF728FF6C
:10155000022006F055FD0020FFF722FF022006F0D2
:101560004FFD641CE4B2082CE7D370BD70B506468D
:101570000024FFF7D5FE00250020FFF711FF022011
:1015800006F03EFD0120FFF70BFF6006040EFFF79B
:101590001DFF08B1641CE4B2012006F031FD6D1C92
:1015A000EDB2082DE8D31EB1FFF793FF204670BDC2
:1015B000FFF7A5FFFAE7000080DE020800080140FF
:1015C00038B5704CE06B002815D054F83C0F012161
:1015D000FEF74BFC2089ADF8000010208DF80300C9
:1015E00003208DF8020069466068F7F71EFB218929
:1015F0006068F7F789FB38BD624AD16B00290AD0D1
:1016000020B1B2F84410106CF7F77EBBB2F844106A
:10161000106CF7F77BBB704710B5FFF7E1FEBDE834
:101620001040CDE710B50446FFF705FF200AA021C2
:1016300001EB4000C0B2FFF778FFFFF729FFE0B2EF
:10164000FFF773FFFFF724FFFFF7F5FEA120FFF779
:101650006CFFFFF71DFF0020FFF788FF0446FFF730
:1016600000FF204610BD70B504460D460020FFF770
:10167000C3FFFFF7E0FE200AA02101EB4000C0B24B
:10168000FFF753FFFFF704FFE0B2FFF74EFFFFF74E
:10169000FFFE2846FFF749FFFFF7FAFEFFF7E1FEDE
:1016A0000120FFF7A9FFBDE87040052006F0C8BC87
:1016B0002DE9F04106460D461746002409E0E000FA
:1016C00025FA00F0C1B2301980B2FFF7CCFF641CDC
:1016D000E4B2BC42F3D3BDE8F0812DE9F04102460B
:1016E0000E4600200024971908E00502381B401E12
:1016F00080B2FFF797FF2844641CE4B2B442F4D3ED
:10170000E9E710B5FF20FFF78DFF55280AD05521D6
:10171000FF20FFF7A8FFFF20FFF784FF552803D025
:10172000012010BD002010BD002010BD70B5044682
:101730000E46154608E02046641CA4B2FFF772FF6F
:1017400006F8010B6D1EADB2002DF4D170BD70B561
:1017500006460D46144606E029783046FFF783FF1B
:10176000761CB6B26D1C641EA4B2F5D270BD59E7EA
:10177000054A1278012A03D0B72802D0B82800D031
:1017800071E7704780DE0208FD000020704730B529
:101790006423B0FBF3F4E4B2B0FBF3F503FB1500F4
:1017A000132C01D96430C0B200EB90030724B3FBC3
:1017B000F4F504FB1533A44D1A440D4415F8015CEF
:1017C0002A4492B2800703D1032901D2521E92B259
:1017D000B2FBF4F004FB102030BD810701D00020E3
:1017E00070476421B0FBF1F201FB120109B1012045
:1017F00070474FF4C871B0FBF1F201FB120008B161
:1018000000207047012070472DE9F047F7F727FBCC
:1018100006468E4FB6FBF7F38D488E4D01889942F0
:1018200033D0038040F2B2744FF4B7784FF4B679F6
:101830000FE02046FFF7D1FF38B1434502D3A3F5AF
:10184000B77304E0641CA4B205E0A3F26D13641C3A
:10185000A4B24B45EDD8AC800024DFF8EC8108F150
:101860000C080CE0A888FFF7B8FF08B1012C2FD0B6
:1018700018F80400984204D81B1A641CA4B21C2B4C
:10188000F0D2641CAC715B1CEB71B6FBF7F007FB8C
:1018900010604FF46161B0FBF1F22A70B0FBF1F21D
:1018A00001FB12033C22B3FBF2F36B70B0FBF1F3CC
:1018B00001FB1300B0FBF2F102FB1100A870EA7902
:1018C000A979A888FFF763FF28720020BDE8F08798
:1018D0001D2BD6D31D3BD0E770B500240420FFF7A5
:1018E00029FB45F25005A8423FD001214FF0C050DE
:1018F000FEF7C6FA0120FFF74DFBFFF7F1FA0120D2
:10190000FEF73DFA08E0641CE4B20A2006F098FBFA
:10191000C82C01D3012070BD4120FEF7B5F9002885
:10192000F1D0FA2C01D3012070BD4FF48070FEF786
:101930003BFA0120FEF73DFAF7F7CCFAF7F7DAFAAF
:1019400001210846F7F772FAF7F7C4FAF7F779FAC0
:1019500047F6FF70F7F799FAF7F7BCFAF7F778FA56
:1019600029460420FFF7DEFA07E0F7F7C3FA012162
:101970000846F7F75BFAF7F7ADFAFFF707FFFFF74F
:1019800043FF002070BD2DE9F05F0646DDF828A07A
:10199000894690460024A6F2B270822802D3012024
:1019A000BDE8F09F40F2B2752B4FDFF8B0B008E011
:1019B0002846FFF712FF08B13C4400E05C446D1C70
:1019C000ADB2B542F4D3A9F1010909F0FF07002532
:1019D000DFF87490DFF874B009F10C090FE019F822
:1019E000050040F2A321484304EBC0143046FFF742
:1019F000F4FE10B1012D00D15C446D1CADB2BD42AE
:101A0000EDD3A8F1010840F2A32008FB00F804EB95
:101A1000C810C3EB4311C1EB032100EB0110CAEB6B
:101A20000A1100EB81000B99441801214FF0C050BE
:101A3000FEF726FA0120FFF7ADFA2046F7F718FA6D
:101A4000F7F748FA0020ABE768DE02088051010092
:101A5000FE000020681100200085E2018033E101D2
:101A600070B5FA4B0024C3F88041F94A0125127A77
:101A7000042A02D3F74A156001E0C3F88851002216
:101A8000C3F88441060602D5C3F88C5101E0C3F8BF
:101A90008C41C3F884514006000E521CD2B2082A71
:101AA000EED30020C3F884410A0602D5C3F88C5156
:101AB00001E0C3F88C41C3F884514906090E401C6B
:101AC000C0B20828EED3C3F8805170BDC0F307221E
:101AD000C1B21046C4E730B5DC4A0023C2F88031F9
:101AE000DB49097A042902D3DA490B6001E0C2F824
:101AF000883100210124C2F88431050602D5C2F8DC
:101B00008C4101E0C2F88C31C2F884414006000EDD
:101B1000491CC9B20829EED3C2F8804130BD30B5A6
:101B2000CA4A0024C2F88041C9490123097A04291C
:101B300002D3C8490B6001E0C2F888310021C2F825
:101B40008441050602D5C2F88C3101E0C2F88C410F
:101B5000C2F884314006000E491CC9B20829EED3F0
:101B6000C2F8803130BD2DE9F04381468846C2F38A
:101B70000724D5B2C3F30726DFB22A20FFF7ABFF55
:101B80000020FFF7CCFF4846FFF7C9FF0020FFF712
:101B9000C6FF4046FFF7C3FF2B20FFF79CFF204600
:101BA000FFF7BDFF2846FFF7BAFF3046FFF7B7FF44
:101BB0003846FFF7B4FFBDE8F0432C208BE72DE952
:101BC000F0410746002240F23F13EF211046FFF795
:101BD000CAFF00254FF4A07600243846FFF776FFB1
:101BE000641CF02CF9D36D1CB542F5D3BDE8F0812F
:101BF00000B52820FFF76FFF10205DF804EB6AE7BF
:101C000010B51120FFF767FF782006F019FABDE83C
:101C1000104029205FE770B58F4C01252560052015
:101C200006F00EFA0020E0630A2006F009FAE563E8
:101C3000782006F005FA1120FFF74DFF782006F016
:101C4000FFF9CF20FFF747FF0020FFF768FFC32011
:101C5000FFF765FF3020FFF762FFED20FFF73BFF46
:101C60006420FFF75CFF0320FFF759FF1220FFF706
:101C700056FF8120FFF753FFE820FFF72CFF852058
:101C8000FFF74DFF1020FFF74AFF7920FFF747FFCE
:101C9000CB20FFF720FF3920FFF741FF2C20FFF773
:101CA0003EFF0020FFF73BFF3420FFF738FF022004
:101CB000FFF735FFF720FFF70EFF2020FFF72FFF7C
:101CC000EA20FFF708FF0020FFF729FF0020FFF7B9
:101CD00026FFC020FFF7FFFE2220FFF720FFC120D4
:101CE000FFF7F9FE1120FFF71AFFC520FFF7F3FEFB
:101CF0003D20FFF714FF2020FFF711FFC720FFF75B
:101D0000EAFEAA20FFF70BFF3620FFF7E4FEC8200B
:101D1000FFF705FF3A20FFF7DEFE5520FFF7FFFE35
:101D2000B120FFF7D8FE0020FFF7F9FE1320FFF7E0
:101D3000F6FEB620FFF7CFFE0A20FFF7F0FEA22046
:101D4000FFF7EDFEF620FFF7C6FE0120FFF7E7FEE6
:101D50003020FFF7E4FEF220FFF7BDFE0020FFF782
:101D6000DEFE2620FFF7B7FE0120FFF7D8FEE020B9
:101D7000FFF7B1FE0F20FFF7D2FE3F20FFF7CFFEA7
:101D80002F20FFF7CCFE0C20FFF7C9FE1020FFF735
:101D9000C6FE0A20FFF7C3FE5320FFF7C0FED52082
:101DA000FFF7BDFE4020FFF7BAFE0A20FFF7B7FE9F
:101DB0001320FFF7B4FE0320FFF7B1FE0820FFF762
:101DC000AEFE0320FFF7ABFE0020FFF7A8FEE120E8
:101DD000FFF781FE0020FFF7A2FE0020FFF79FFE25
:101DE0001020FFF79CFE0320FFF799FE0F20FFF75E
:101DF00096FE0520FFF793FE2C20FFF790FEA22011
:101E0000FFF78DFE3F20FFF78AFE0520FFF787FED4
:101E10000E20FFF784FE0C20FFF781FE3720FFF72E
:101E20007EFE3C20FFF77BFE0F20FFF778FE11209F
:101E3000FFF751FE782006F003F92920FFF74BFE4B
:101E4000BDE87040322006F0FBB80000008022425E
:101E50001C6D0020988121428081224210B5FB48F0
:101E6000002101604160C160C163A0F5C070F84A03
:101E7000127A042A02D3F748016001E0C0F8881101
:101E8000FFF7C9FEBDE8104047F6196097E62DE957
:101E9000F05FDDE90A7800281BD0EF4D18262424D6
:101EA000203B03EBC30000EB400005EB80058819E5
:101EB000401E00F0FF0C1319C8B25B1E6146FFF70D
:101EC00052FE7443E01704EB5070C0F3CF090026B4
:101ED0002CE0E24D302660242D2B07D0202B08D09B
:101EE000303B03EBC30005EB8015E0E705F5B45587
:101EF000DDE705F5C655DAE700244FEA182A4FEA70
:101F0000172B2878E040C00704D0F9B25846FFF7F5
:101F1000A7FD04E008F0FF015046FFF7A1FD641C97
:101F2000A4B2082CEDD36D1C761CB6B24E45E3D39B
:101F3000BDE8F09F2DE9FC470746DDE90A890C461C
:101F400016461D4609E0B2B2A1B23846CDE9008975
:101F5000FFF79DFF37B117346D1C2B78002BF2D1A2
:101F6000BDE8FC871F34F7E770B51646049A01FBFD
:101F700000F4A5B254181844401EC1B2641ED8B271
:101F80002346FFF7F0FD002407E036F81400C1B245
:101F9000000AFFF765FD641CA4B2AC42F5D370BD26
:101FA0002DE9F041089E069A01FB00F4A5B25418F1
:101FB0001844401EC1B2641ED8B22346FFF7D3FDB9
:101FC0000024370A05E0F1B23846FFF749FD641CEA
:101FD000A4B2AC42F7D309E62DE9FF5FA04F7978B0
:101FE00001297AD19A4991F86E200AB1462200E07F
:101FF000432291F8C5B00A236426DFF868E2202561
:10200000002441424FF0300A4FF02D0C4FF02E08C3
:102010004FF47A79BBF10A0F26D0002870DB4845CF
:102020006FDB90FBF9F130318DF8081090FBF9F17E
:1020300009FB110191FBF6F130318DF8091090FB8D
:10204000F6F106FB110191FBF3F130318DF80A1026
:102050008DF80B8090FBF3F103FB110030308DF80D
:102060000C008DF80D4074E1002858DB48451BDB5F
:1020700090FBF9F130318DF8081090FBF9F109FB74
:10208000110191FBF6F130318DF8091090FBF6F15A
:1020900006FB110090FBF3F030308DF80A008DF84C
:1020A0000B208DF80C4054E1642817DB90FBF6F10F
:1020B00030318DF8081090FBF6F106FB110090FB13
:1020C000F3F030308DF809008DF80A208DF80B50B0
:1020D0008DF80C508DF80D403BE15EE10A2811DBD4
:1020E00090FBF3F030308DF808008DF809208DF862
:1020F0000A508DF80B508DF80C508DF80D4028E1EA
:10210000C4E070E08DF808A08DF809208DF80A5021
:102110008DF80B508DF80C508DF80D4019E170457D
:102120001BDC8DF808C091FBF9F030308DF8090008
:1021300091FBF9F009FB101090FBF6F030308DF8B0
:102140000A0091FBF6F006FB101090FBF3F0303024
:102150008DF80B008DF80C40FBE010F1640F14DCDF
:102160008DF808C091FBF6F030308DF8090091FB36
:10217000F6F006FB101090FBF3F030308DF80A00FB
:102180008DF80B208DF80C40E3E010F10A0F16DCFF
:102190008DF808C091FBF3F030308DF809008DF810
:1021A0000A8091FBF3F003FB101030308DF80B0028
:1021B0008DF80C208DF80D408DF80E50C9E08DF88B
:1021C00008C08DF809A08DF80A8091FBF3F003FB9D
:1021D000101030308DF80B008DF80C208DF80D406C
:1021E0008DF80E50B5E064281BDB90FBF6F1303122
:1021F0008DF8081090FBF6F106FB110191FBF3F14D
:1022000030318DF809108DF80A8090FBF3F103FB53
:10221000110030308DF80B008DF80C208DF80D403A
:1022200097E00A2820DB90FBF3F130318DF808109D
:102230008DF8098090FBF3F103FB110030308DF82D
:102240000A008DF80C208DF80D4082E0808122423A
:102250001C6D00209881214250A0030814E0020860
:102260007211002018FCFFFF8DF808A08DF809807E
:1022700090FBF3F103FB110030308DF80A008DF86C
:102280000B208DF80C408DF80D5062E070451BDC82
:102290008DF808C091FBF9F030308DF8090091FB02
:1022A000F9F009FB101090FBF6F030308DF80A00C1
:1022B00091FBF6F006FB101090FBF3F030308DF838
:1022C0000B008DF80C4044E010F1640F14DC8DF825
:1022D00008C091FBF6F030308DF8090091FBF6F064
:1022E00006FB101090FBF3F030308DF80A008DF8EB
:1022F0000B208DF80C402CE010F10A0F16DC8DF845
:1023000008C091FBF3F030308DF809008DF80A8099
:1023100091FBF3F003FB101030308DF80B008DF8BB
:102320000C208DF80D408DF80E5012E08DF808C08D
:102330008DF809A08DF80A8091FBF3F003FB1010D3
:1023400030308DF80B008DF80C208DF80D408DF895
:102350000E50FB4E307880B1FA48007868B18DF8A5
:1023600008508DF809508DF80A508DF80B508DF8F3
:102370000C508DF80D408DF80E5047F617604FF653
:10238000FF71CDE9001002AB6C226A210120FFF73A
:10239000D1FD3078002800D17C70BDE8FF9F70B57A
:1023A00086B0E94DA978012941D10021E74B2024CD
:1023B00003AE01EBC0021A4492F8812352B1725469
:1023C000491CC9B20529F4D393F86F0000260128EF
:1023D00002D010E07454F3E7DD48007858B903F2F6
:1023E00089334F2018706E2058709E70DC701C71FD
:1023F0005C719C71DC71D74C207830B1D148007889
:1024000018B1D5A103A817F03DFE8DF8116047F66D
:1024100017604FF6FF71CDE9001003AB97226A21D8
:102420000120FFF787FD2078002800D1AE7006B0AC
:1024300070BD7FB5C44DE878002830D0C34890F80F
:10244000A903022803D0012806D050B10DE0C4A191
:1024500002A817F017FE08E0C3A102A817F012FEA9
:1024600003E0C3A102A817F00DFEC34C207830B1E1
:10247000B448007818B1C1A102A817F003FE47F6CE
:1024800017604FF6FF71CDE9001002ABC2226A213E
:102490000120FFF74FFD2078002800D1E8707FBDB4
:1024A000FEB5B84F387800284BD000203870FDF7C3
:1024B0007AFBB54947F619644FF6FF7509784FF472
:1024C0008976C1B3B8B33878012847D0AF4ACDE98F
:1024D0000065B6232D2128200294FFF745FDAC4866
:1024E0000178427880781144C14225D1A94800780A
:1024F00098B3012846D002284ED0032856D004288D
:1025000018D1FDF750FB01285AD0042858D00228D2
:1025100060D005285ED0032866D0062864D0002845
:1025200008D19D4ACDE90065DE232D210F200294BC
:10253000FFF71AFDFEBD06E0984A907901285DD0AC
:102540006CE00120B2E7964ACDE90065B6232D2163
:1025500028200294FFF708FDC1E709E0904ACDE981
:102560000065B6232D2128200294FFF7FDFCB6E775
:10257000894ACDE90065DE232D210F200294FFF763
:10258000F3FCD7E7874ACDE90065DE232D210F2034
:102590000294FFF7E9FCCDE7834ACDE90065DE232D
:1025A0002D210F200294FFF7DFFCC3E77F4ACDE91E
:1025B0000065DE232D210F200294FFF7D5FCB9E73B
:1025C000784ACDE90065DE232D210F200294FFF724
:1025D000CBFCAFE7744ACDE90065DE232D210F2047
:1025E0000294FFF7C1FCA5E7704ACDE90065DE2340
:1025F0002D210F200294FFF7B7FC9BE7D179012929
:102600000CD0117A012909D0CDE90065DE23654A95
:102610002D210F200294FFF7A7FC8BE7D179012928
:102620000ED101280CD0137A012B09D0CDE9006519
:10263000DE235D4A2D210F200294FFF795FC79E7F8
:10264000127A012A0DD101280BD0012909D0CDE938
:102650000065DE23554A2D210F200294FFF784FCEC
:1026600068E7CDE90065DE234B4A2D210F20029457
:10267000FFF77AFC5EE72DE9FE4FFDF7AAFA074661
:102680004B48DFF8C4800178B94203D0012188F8B3
:1026900005100770DFF8B4904FF6FF764FF0000A90
:1026A00099F8670299F8681299F86A22084499F82B
:1026B000691247F619641144C8424FF489753ED037
:1026C000DFF8D8B09BF8000001280DD19BF801106D
:1026D000012909D0CDE900560223364A2D213720A1
:1026E0000294FFF741FC18E09BF8011001290BD17F
:1026F000012809D0CDE9005602232F4A2D21372089
:102700000294FFF731FC08E0CDE9005402230022D7
:102710002D2137200294FFF743FC9BF8020001288B
:102720004ED19BF8031001294AD0CDE900563E2333
:10273000224A2D2137200294FFF716FC23E159E0AD
:102740003000002033000020721100201C6D00209A
:102750002F000020310000202020202020202000F9
:102760004865617420000000436F6F6C200000001A
:102770004175746F200000003200002020202020CE
:1027800020000000000100202C000020E844030885
:10279000896F00203B000020C02103084009002071
:1027A000D8360308062703084C2C03089231030887
:1027B0005E000020F85203084E66030814FB02086E
:1027C0009BF8031001290BD1012809D0CDE900564F
:1027D0003E23FD4A2D2137200294FFF7C5FBD2E0AE
:1027E000CDE900543E2300222D2137200294FFF72B
:1027F000D7FBC8E099F8B912F448012919D098F824
:10280000041000299AD00068002877D0CDE9005440
:102810000223EF4A2D2137200294FFF7A5FBCDE9D3
:1028200000563E23EB4A2D2137200294FFF79CFBF4
:10283000A7E00068C0B198F80400002813D0CDE9E3
:102840000054022300222D2137200294FFF7A8FB19
:10285000CDE900563E23DF4A2D2137200294FFF7B1
:1028600083FB88F804A08EE0DFF86CB39BF80000CF
:10287000092830D004DC012807D0042864D117E0EF
:102880000A283CD00B285FD14CE0CDE9005602234A
:10289000CF4A2D2137200294FFF766FBCDE9005681
:1028A0003E23CC4A2D2137200294FFF75DFB4BE0FD
:1028B000CDE900560223C64A2D2137200294FFF7A6
:1028C00053FBCDE900563E23BF4A2D213720029409
:1028D000FFF74AFB38E0CDE900560223BF4A2D211D
:1028E00037200294FFF740FBCDE900563E23B94A5A
:1028F0002D2137200294FFF737FB25E029E0CDE9B1
:1029000000560223B54A2D2137200294FFF72CFBF5
:10291000CDE900563E23AC4A2D2137200294FFF723
:1029200023FB11E0CDE90054022300222D213720A2
:102930000294FFF735FBCDE900543E2300222D2100
:1029400037200294FFF72CFBA5499BF80000087084
:1029500019E0A448007818B399F87600B0B3CDE92F
:10296000005402239D4A2D2137200294FFF7FCFAE0
:10297000CDE900563E23974A2D2137200294FFF7D8
:10298000F3FA88F804A099F86B0299F86C12C8421F
:1029900068D0DFF8549299F8040001282BD039E070
:1029A00099F8760098B1CDE900540223884A2D2188
:1029B00037200294FFF7D8FACDE900563E23824A29
:1029C0002D2137200294FFF7CFFADAE709E0CDE9AD
:1029D00000540223814A2D2137200294FFF7C4FAC4
:1029E000EAE7CDE900540223794A2D2137200294E9
:1029F000FFF7BAFABCE799F8051001290AD0CDE92A
:102A000000567A23794A2D2137200294FFF7ACFA39
:102A1000BDE8FE8F99F8051001290BD1012809D0D6
:102A2000CDE900567A23724A2D2137200294FFF710
:102A30009BFAEDE7012801D1012901D048B941B93C
:102A4000CDE900547A2300222D2137200294FFF78C
:102A5000A7FA99F80400642808D099F805006428BA
:102A600004D0D5E798F805000128D1D127B1012F6E
:102A70000CD0022F1DD113E0CDE900547A2300229F
:102A80002D2137200294FFF78BFA12E0CDE9005692
:102A90007A23574A2D2137200294FFF765FA08E080
:102AA000CDE900567A23514A2D2137200294FFF7B1
:102AB0005BFA88F805A0ABE71CB547F61964012856
:102AC00008D000944BA3C222002101200194FFF7FB
:102AD00031FA1CBD009447A36C220021012001940F
:102AE000FFF728FA009443A39722002101200194C4
:102AF000FFF720FA1CBD3EB547F619654FF6FF7487
:102B000067208DE8310000231A462D21EF20FFF7C2
:102B100047FA92208DE8310000231A462D21EF203C
:102B2000FFF73EFABD208DE8310000231A462D2123
:102B3000EF20FFF735FA3EBD2DE9FF4764250A2354
:102B400020244FF0000C4FF47A77202A29D02E262B
:102B50004FF0300900297DDBB9427CDB91FBF7F0B7
:102B600030308DF8080091FBF7F007FB101090FB58
:102B7000F5F030308DF8090091FBF5F005FB1010F1
:102B800090FBF3F030308DF80A008DF80B6091FB6C
:102B9000F3F003FB101030308DF80C008DF80D2091
:102BA000D3E0B9423FDB91FBF7F030308DF80800FD
:102BB00091FBF7F007FB101090FBF5F030308DF82B
:102BC000090091FBF5F01FE06A0E03084C0000209D
:102BD000F852030814FB0208370000204E66030871
:102BE0002E0000203B00002040090020FA8C030842
:102BF000A47903082020202020202020202020202D
:102C0000202020200000000005FB101090FBF3F0B6
:102C100030308DF80A0091FBF3F003FB10103030D8
:102C20008DF80B0046E064291EDB91FBF7F007FBF3
:102C3000101090FBF5F030308DF8080091FBF5F0A6
:102C400005FB101090FBF3F030308DF8090091FB7C
:102C5000F3F001E07CE034E003FB101030308DF83D
:102C60000A008DF80B4025E00A2914DB8DF8084096
:102C700091FBF5F005FB101090FBF3F030308DF870
:102C8000090091FBF3F003FB101030308DF80A00BF
:102C90008DF80B400EE000290CDB8DF8084091FB0D
:102CA000F3F003FB101030308DF809008DF80A4066
:102CB0008DF80B408DF80C408DF80D408DF80EC04E
:102CC000A7E064291BDB91FBF5F030308DF808009C
:102CD00091FBF5F005FB101090FBF3F030308DF810
:102CE00009008DF80A6091FBF3F003FB10103030FF
:102CF0008DF80B008DF80C208DF80D4025E00A2989
:102D000012DB91FBF3F030308DF808008DF809608C
:102D100091FBF3F003FB101030308DF80A008DF8B2
:102D20000C208DF80D4010E08DF808908DF80960AA
:102D300091FBF3F003FB101030308DF80A008DF892
:102D40000B208DF80C408DF80D408DF80EC060E022
:102D500048424FF02D0811F57A7F24DC8DF8088069
:102D600090FBF7F130318DF8091090FBF7F107FB7C
:102D7000110191FBF5F130318DF80A1090FBF5F15E
:102D800005FB110191FBF3F130318DF80B108DF83B
:102D90000C6090FBF3F103FB110030308DF80D0057
:102DA0008DF80E2033E011F1640F1DDC8DF80880E2
:102DB00090FBF5F130318DF8091090FBF5F105FB32
:102DC000110191FBF3F130318DF80A108DF80B6091
:102DD00090FBF3F103FB110030308DF80C008DF8FF
:102DE0000D208DF80E4012E08DF808808DF80990C6
:102DF0008DF80A6090FBF3F103FB110030308DF881
:102E00000B008DF80C208DF80D408DF80E408DF8DC
:102E10000FC047F619604FF6FF71CDE9001002AB05
:102E2000C22200210120FFF785F8BDE8FF877CB5AD
:102E30000E4647F619654FF6FF7403466C220021D3
:102E40000120CDE90045FFF775F8334697220021B0
:102E50000120CDE90045FFF76DF87CBD2DE9FE4F5F
:102E600005460C4647F619694FF6FF768DE8500285
:102E700008212B46FC4A0846FFF776F8A01C47F6C7
:102E8000176A80B28DE84104AB1D00220121712038
:102E9000FFF786F804F10800CDE9016A87B2AB1CA0
:102EA00000221C2102200097FFF77AF804F122008B
:102EB000CDE901691FFA80F8EB4A08212B468032E0
:102EC0000846CDF80080FFF74FF804F1270080B2E4
:102ED0008DE84104AB1D002201217120FFF760F84D
:102EE000CDE9016905F17303CDF80080082198460A
:102EF000DE4A0846FFF738F8DC4A8DE85002082120
:102F0000434680320846FFF72FF8CDE9016A05F104
:102F1000780300221C2101200097FFF741F804F1FB
:102F200028004BF69C6780B28DE8C1006B1D002223
:102F300002217320FFF734F88DE8D0006B1D0022CA
:102F400002217320FFF72CF8A41DA4B28DE8D00055
:102F50002B46002220210220FFF722F88DE8D00026
:102F600005F17903002220210220FFF719F84FE52F
:102F7000F0B5BF4D2E2764230A242026C2EB02128F
:102F80002A44002816DA2D215172404290FBF3F1B9
:102F90003031917290FBF3F103FB110191FBF4F1DD
:102FA0003031D172177390FBF4F104FB1100303013
:102FB000507358E0DFF8BCC24FF47A7561444FF0AB
:102FC000250CA84237DB91F8E51002291BD090FBB5
:102FD000F5F13031517290FBF5F105FB110191FBD8
:102FE000F3F13031917290FBF3F103FB110191FB8E
:102FF000F4F13031D172177390FBF4F104FB11003E
:10300000303050732FE090FBF5F13031517290FB6E
:10301000F5F105FB110191FBF3F13031917290FB59
:10302000F3F103FB110090FBF4F03030D07282F822
:103030000CC0567317E090FBF3F53035557290FBDA
:10304000F3F503FB150393FBF4F330339372D7725C
:1030500090FBF4F304FB13003030107391F8E5009B
:10306000022802D056739673F0BD82F80DC0FAE7BD
:103070002DE9F05F7F4890F8B812092902D909219B
:1030800080F8B81290F8B812002973D000243A27BB
:10309000DFF8E4814FF00A094FF0640A2025744EEE
:1030A00012E2081990F8BA02C01E0E281CD2DFE8FE
:1030B00000F0071E354C647B92A9C0FAE7E6E5DA1A
:1030C0000020C4EB041232440B1893F8A93163B109
:1030D0001354401CC0B20828F6D31772B8F9000088
:1030E00022460021FFF744FFECE11554F1E70020F0
:1030F000C4EB041232440B1893F8B13163B113548A
:10310000401CC0B20828F6D31772B8F90200224654
:103110000021FFF72DFFD5E11554F1E70020C4EBA6
:10312000041232440B1893F8B93163B11354401CA4
:10313000C0B20828F6D31772B8F90400224600215D
:10314000FFF716FFBEE11554F1E70020C4EB0412AF
:1031500032440B1893F8C1316BB11354401CC0B208
:103160000828F6D31772B8F9060022460021FFF7A7
:10317000FFFEA7E1AEE11554F0E70020C4EB041216
:1031800032440B1893F8C93163B11354401CC0B2D8
:103190000828F6D31772B8F9080022460021FFF775
:1031A000E7FE8FE11554F1E70020C4EB041232442E
:1031B0000B1893F8D13163B11354401CC0B20828E6
:1031C000F6D31772B8F90A0022460021FFF7D0FEA5
:1031D00078E11554F1E70020C4EB041232440B18D7
:1031E00093F8D93163B11354401CC0B20828F6D308
:1031F0001772B8F90C0022460021FFF7B9FE61E111
:103200001554F1E70020C4EB041232440B1893F874
:10321000E13163B11354401CC0B20828F6D31772D1
:10322000B8F90E0022460021FFF7A2FE4AE115542C
:10323000F1E7FCF7CEFCC4EB04105321315400EB52
:10324000060B74218BF8011061208BF802006720B7
:103250008BF8030065208BF804008BF80570FCF7F1
:10326000A2FC00210EE0F4E064C8030864C903086E
:10327000080100201C6D0020F0110020B3E074E074
:1032800022E010E0FB4AC0EBC00010440BEB01034E
:10329000425C9A71491CC9B20729F7D38BF80D50CB
:1032A0008BF80E500EE10020C4EB041232440B18D0
:1032B00093F8913133B11354401CC0B20E28F6D3A9
:1032C0009573FFE01554F7E7EB498879EB4B401E07
:1032D00000EB800003EB40004278C4EB0410325452
:1032E0008A793044521E02EB820203EB420292784A
:1032F00042708A79521E02EB820203EB4202D278BC
:103300008270C570CA79B2FBF9F230320271CA79A3
:10331000B2FBF9F309FB1322303242712C22827185
:103320008B884FF47A72B3FBF2F33033C3718B881E
:10333000B3FBF2FC02FB1C32B2FBFAF23032027237
:103340008A88B2FBFAF30AFB1322B2FBF9F230329D
:1033500042728988B1FBF9F209FB12113031817296
:10336000C572057345738573ACE0C4EB041054213A
:1033700031543044692141706D2181706521C170E3
:103380000571BF49097803291FD0BB4A1178B1FBE9
:10339000F9F1303141711178B1FBF9F309FB1311E7
:1033A00030318171C7715178B1FBF9F1303101725F
:1033B0005178B1FBF9F209FB12113031417285727B
:1033C000C5720573457385737CE045214171722197
:1033D0008171C1716F22027241728572C57205736B
:1033E000457385736EE0C4EB0410432131543044BF
:1033F0004F21417032218170C770A2494FF47A7217
:103400000988914204D3B1FBF2F33033037100E039
:103410000571B1FBF2F302FB1312B2FBFAF2303288
:103420004271B1FBFAF20AFB1212B2FBF9F230322E
:103430008271B1FBF9F209FB12113031C1717021B7
:10344000017241726D218172C57205734573857376
:1034500038E0C4EB041048213154304475214170E8
:103460006D2181706921C17080F804A041717421BF
:1034700081717921C17107728349B1F90010B1F5E9
:103480007A7F08DB3121417230218172C17225219E
:103490000173457315E091FBFAF23032427291FBF1
:1034A000FAF20AFB121292FBF9F2303282722E22E9
:1034B000C27291FBF9F209FB12113031017325211F
:1034C00041738573641CE4B2704991F8B802A0425C
:1034D0003FF6E7ADBDE8F09F2DE9FC5FFFF7C8FDC3
:1034E000DFF8A8816A4C6B4D98F8B812002647F6B1
:1034F00017674FF6FF7B99B90020491EC1EB0111F8
:1035000029440A5C2254401CC0B20A28F9D3A6728E
:10351000CDE900B75E4BED2200210120FEF70AFD48
:1035200098F8B802002842D0DFF86891401EA9F14F
:103530000809C0EB00104219D9F80410501C884249
:103540001CD80020531A03F10F0C05E011F800807D
:1035500004F80080401CC0B28445F7DC0020A1EBD9
:10356000020808E003EB000AA24415F800C08AF83C
:103570000FC0401CC0B28045F4DC06E000200B5CAC
:103580002354401CC0B20A28F9D30E328A4202D119
:10359000C9F8045002E0491CC9F80410A672CDE92C
:1035A00000B73B4BED221E210120FEF7C3FCBDE816
:1035B000FC9FF0B587B0044647F617664FF478478E
:1035C000CDE90176ED20002300901A461E21EF2060
:1035D000FEF7E6FC0021274A2E4D8C3204A802F1AA
:1035E0001E03083D14B1012C08D00EE095F801C06F
:1035F0008C4412F80CC000F801C006E095F801C038
:103600008C4413F80CC000F801C0491CC9B20A2947
:10361000E8D300248DF81A40CDE9007604ABED2202
:103620001E210120FEF786FC6878192803D2401C71
:10363000687007B0F0BD6C70FBE70EB555224FF611
:10364000FF71002809D0CDE90021029108218B23C8
:1036500000220846FEF7A4FC0EBDCDE9002147F686
:103660001960029008218B2300220846FEF798FC7F
:103670000EBD00004CDF020868110020C6D402080D
:10368000130300205C020020600200201C6D00205B
:103690007B110020080100202DE9FC470D464FF466
:1036A0007A7A47F619664FF6FF7700287AD14FF0FD
:1036B0000A094FF06408002D76DB2C46AFF65C73E8
:1036C000CDE90076202206210120FEF733FC554586
:1036D00034DB94FBF9F004B2642C0BDB94FBF8F0C0
:1036E0003030CDE90076C3B2052227210020FEF755
:1036F000CEFB07E0CDE9007620230522272100201C
:10370000FEF7C5FB94FBF8F008FB104090FBF9F0C6
:103710003030CDE90076C3B2052257210020FEF7F4
:10372000B6FB94FBF9F009FB10403030CDE9007690
:10373000C3B2052297210020FEF7A9FB554531DAD7
:10374000642D0BDB94FBF8F03030CDE90076C3B28A
:10375000052227210020FEF79AFB07E0CDE900763D
:103760002023052227210020FEF791FB94FBF8F08F
:1037700008FB104090FBF9F03030CDE90076C3B281
:10378000052257210020FEF782FB94FBF9F009FB8C
:1037900010403030CDE90076C3B2052297210020D9
:1037A000FEF775FB68E0FFE7684204B2642C2FDB8C
:1037B00094FBF8F03030CDE90076C3B20522272122
:1037C0000020FEF764FB94FBF8F008FB104090FB30
:1037D000F9F03030CDE90076C3B205225721002040
:1037E000FEF755FB94FBF9F009FB10403030CDE9B2
:1037F0000076C3B2052297210020FEF748FBCDE9F1
:10380000007630A3202206210120FEF793FB33E04F
:10381000CDE900762023052227210020FEF737FB83
:1038200094FBF8F008FB104090FBF9F03030CDE944
:103830000076C3B2052257210020FEF728FB94FB37
:10384000F9F009FB10403030CDE90076C3B2052213
:1038500097210020FEF71BFBCDE900761AA320225A
:1038600006210120FEF766FBCDE9007615A3202294
:1038700028210120FEF75EFB554503DD0020FFF700
:10388000DCFE02E00120FFF7D8FE104C2078012872
:103890000DD10F4890F86E0058B1CDE900760DA318
:1038A0003822D6210120FEF745FB00202070BDE81C
:1038B000FC87CDE9007608A33822D6210120FEF747
:1038C00039FBF2E72D0000002000000072110020FB
:1038D0001C6D0020460000004300000010B5254C80
:1038E00001212046FDF714F9012803D122490A6875
:1038F000521C0A602149088841F28832904203D262
:103900000A88521C0A8001E0002008802046BDE899
:1039100010400121FDF703B97FB504460D46012192
:103920001020FCF7ADFAADF80840ADF804500020C7
:10393000ADF80A00ADF806000E4C01A92046FCF7D0
:10394000D3FB36218DF8001001218DF801100322E0
:103950008DF802208DF803106846F4F7E2FE01228C
:1039600011462046FCF7ABFE01212046FCF78DFEF8
:103970007FBD000000100040380200206E060020CD
:10398000FE49097A05290BD2FD4A20B18832918877
:103990001068F5F7B9B9883291881068F5F7B6B9AB
:1039A000F84A18B102211046F5F7AEB902211046C7
:1039B000F5F7ACB9F149097A05290BD2F04A20B1E3
:1039C000943291881068F5F79FB994329188106805
:1039D000F5F79CB9EB4A18B101211046F5F794B9F7
:1039E00001211046F5F792B9E449097A05290BD26D
:1039F000E34A20B1A03291881068F5F785B9A0326A
:103A000091881068F5F782B9DE4A18B11021104686
:103A1000F5F77AB910211046F5F778B9D749097A40
:103A200005290BD2D64A20B1AC3291881068F5F73F
:103A30006BB9AC3291881068F5F768B9D14A18B102
:103A400008211046F5F760B908211046F5F75EB970
:103A5000CA49097A05290BD2C94A20B1B8329188DE
:103A60001068F5F751B9B83291881068F5F74EB97A
:103A7000C44A18B104211046F5F746B9042110468E
:103A8000F5F744B9BD49097A05290BD2BC4A20B1E2
:103A9000C43291881068F5F737B9C432918810683C
:103AA000F5F734B9B74A18B120211046F5F72CB90B
:103AB00020211046F5F72AB92DE9FC41F220ADF896
:103AC000040000258DF8075002248DF80640AE4E04
:103AD00001A93046F5F7A9F84FF00308ADF80480C6
:103AE0008DF807508DF80640A84F01A93846F5F724
:103AF0009CF8ADF804808DF807508DF80640DFF88B
:103B0000908201A94046F5F790F89C481025007A6C
:103B1000052816D21C20ADF804008DF807508DF84A
:103B2000064001A94046F5F780F8E020ADF8040012
:103B30008DF807508DF8064001A93046F5F775F865
:103B400015E03F20ADF804008DF807508DF80640D1
:103B500001A98C48F5F769F80C20ADF804008DF840
:103B600007508DF8064001A94046F5F75EF84FF47E
:103B70000076ADF800608DF803508DF8024069467C
:103B80003846F5F752F801213046FCF76EF9BDE8EA
:103B9000FC8110B586B04FF40040FCF7E9F8012134
:103BA0004802FCF762F9002001908DF808008DF8BA
:103BB00009004FF460210391049001208DF8140056
:103BC000744C01A92046F4F72FFE01212046F4F79A
:103BD00053FE2046F4F773FE2046F4F775FE0128E5
:103BE000FAD02046F4F777FE2046F4F779FE012854
:103BF000FAD006B010BD2DE9F0470546042B06D0DB
:103C0000062B04D0842B05D0862B03D004E04FF480
:103C1000FA7001E04FF47A70DFF860C105F1140327
:103C20006344DC7E1B7F04EB032340F2FF345A4FD6
:103C3000A14203DBBB6418B2BDE8F08701EB810150
:103C40004E0096FBF0F10CB2CAB1611C05EB4101CC
:103C50006144CA7E097F02EB012305EB4401614404
:103C6000CA7E097F02EB01255D1B00FB14636B43D9
:103C700093FBF0F000EB01201044B86433E005EB57
:103C80004401614411F8312F497802EB0122611C93
:103C900005EB4101614491F8315091F8328005EB18
:103CA0000821A2EB010919F0A5F98246484619F04E
:103CB00089F98146304619F085F90646601C19F0ED
:103CC00081F9514619F0DEF9314619F0B1FA494649
:103CD00019F0D8F9514619F043F819F037F900EB0B
:103CE00008202844B864B7F8480000B2A4E770B5CB
:103CF000224C294B0A281FD00A220B282BD0274DF3
:103D0000231835F9106093F8F73006FB031101EB27
:103D1000810149005B1C91FBF3F191FBF2F302FB83
:103D20001313052B00DB0A3191FBF2F325F8103059
:103D300091FBF2F000B270BD187A052800D25983C9
:103D400094F86000B3F91A2002FB0011401C91FBAB
:103D5000F0F05883EEE794F829035C8D04FB001122
:103D600001EB81014900401C91FBF0F090FBF2F166
:103D700002FB1101052900DB0A3011E01C6D002057
:103D800080DE02080018014000080140000C0140DC
:103D9000001001400024014040020020C811002012
:103DA00090FBF2F1598590FBF2F0C3E710B51222B7
:103DB0004FF4E164132907D0142932D0FE4B997CCB
:103DC000814251DD204610BDFC4B997C814201DDD2
:103DD000204610BD521E52B29C5C214481421DDD22
:103DE000081A64214843995C90FBF1F0042A09DB2E
:103DF000121F02EBC20101EB021100EB8100C0F3C4
:103E00000E0009E002EBC20101EB021100EB8100A0
:103E1000C0F5C87040F4004000B210BD002AD9D1EE
:103E200048E00921E64B5A8A824202DD4FF4AF7026
:103E300010BD491E49B233F811402244824210DDC0
:103E4000101AC0EB0010400033F8112090FBF2F084
:103E5000C1EB011100EB4100C0F30E00463000B28F
:103E600010BD0029E5D125E0521E52B29C5C2144D0
:103E700081421DDD081A64214843995C90FBF1F0F2
:103E8000042A09DB121F02EBC20101EB021100EB55
:103E90008100C0F30E0009E002EBC20101EB021148
:103EA00000EB8100C0F5C87040F4004000B210BDC6
:103EB000002AD9D1C34810BD2DE9F0410746C248B8
:103EC000B0F92C50B0F92E40281B19F07BF8BF4EEA
:103ED000314618F045FF8046C8204443684200EB55
:103EE000800004EBC00019F06DF8314618F038FF7F
:103EF000B74C214619F0C6F80546384619F07AF84D
:103F0000414619F0BFF8294618F0BCFE214618F0CA
:103F100027FF19F01BF800B2BDE8F0812DE9F0474A
:103F20001D46AC4E40F2062301FB03F796F87834A9
:103F30004FF47A784FF0640900283AD00E2838D030
:103F400063283CD04FF4966A01FB0AFC40F2FF3A2A
:103F5000802836D08B2834D0012835D00B2833D098
:103F60000D2831D0022855D082285ED0032867D092
:103F7000052865D0072863D0082861D009285FD0BC
:103F80000A285DD0832873D0852871D087286FD008
:103F900088286DD089286BD08A2869D0042873D0EE
:103FA000842871D0062870D086286ED00C286DD059
:103FB000D5E097FBF8F0434393FBF9F2CFE00A46D4
:103FC000CDE09CFBFAF2CAE0012816D00D2819D0EA
:103FD00088B21321FFF7EAFE010402D5C0F30E00F8
:103FE000404296F86E1031B100EBC000052190FB05
:103FF000F1F000F5A0704219B1E088B20221FFF79C
:10400000D5FEE9E788B21421FFF7D0FE4628E3DAAF
:104010004620E1E7084618F08CFB6F4A6F4B18F01A
:10402000DBFB18F057FB024699E0084618F081FBCD
:104030006B4A6C4B18F0D0FB18F04CFB02468EE03C
:10404000B1F5F17F09DC052805D0082803D00A283E
:1040500001D0012283E0002281E0032806D0072856
:1040600004D0092802D0012279E001E0002276E0A4
:104070004FF4FA7399420CDC852808D0882806D0C2
:104080008A2804D001226AE00FE032E055E00022E5
:1040900065E0994263DD832805D0872803D089280D
:1040A00001D001225BE0002259E0042802D08428DC
:1040B00003D004E097FBF8F201E09CFBFAF25343D3
:1040C00093FBF9F1404A38320428127802D0842850
:1040D00007D00CE0042309B20020FFF78CFD044652
:1040E00005E0842309B20020FFF785FD044662192C
:1040F00035E0062802D0862803D004E097FBF8F2CA
:1041000001E09CFBFAF2534393FBF9F12E4A38325B
:104110000628527802D0862807D00CE0062309B280
:104120000020FFF768FD044605E0862309B2002061
:10413000FFF761FD0446621911E0084618F0F9FA2C
:10414000294A2A4B18F048FB18F0C4FA4FF4C871FA
:10415000884200DA084680B2FFF7AEFE024610B28F
:104160006AE5811E0B2910D2DFE801F00B0F0F0664
:1041700006060606060606001D49401F31F9100016
:1041800070471148B0F93C00704700207047800824
:10419000704770B505460C4602212846F4F7BBFC73
:1041A0000523012221462846F4F7C8FB01212846B1
:1041B000F4F79DFB02211DE08CD402089FD4020875
:1041C000B2D40208E883FFFF400200200000204331
:1041D000000020411C6D002039B4C876BE9FBA3F54
:1041E000C1CAA145B6F3BD3F5C8FC2F5285CDF3F75
:1041F000F01100202846F4F787FC0028DAD0284682
:10420000BDE87040F4F7E0BB70B50F21F948FFF747
:10421000C0FF80B2FFF7BBFF01B20A20FFF767FDC6
:10422000F54D95F85F10132915D0142918D080B2D8
:104230000221FFF7BBFDF14CA08400EBC001052279
:1042400091FBF2F101F5A07109B2E18495F86E20BD
:104250005AB1A1870AE080B21321FFF7A7FDEAE770
:1042600080B21421FFF7A2FDE5E7A087A08FE087C9
:10427000218D0844A087E0480021D530F6F7A4FC42
:1042800038B195F87B0395F87A1300EB0120608430
:1042900070BD95F85F00A8B1022816D0132814D07D
:1042A000042815D0D649032818D010281ED011286C
:1042B00024D012282FD0421F072A3DD831F81200EF
:1042C00060843FE0A08F60843CE0A08F608439E090
:1042D000E08E94F900100844608433E0B1F90000E6
:1042E000B4F93C100844401060842BE0B1F90000A0
:1042F000B1F9021008444010608423E0B1F90000D5
:10430000B1F90220B1F9041010440844032190FBD4
:10431000F1F0608416E0B1F90000B1F90220104418
:10432000B1F90420B1F9061011440844C11700EB9B
:1043300091708010608405E0012808D0152809D00C
:10434000A08F608495F8A20015280FD019E0088886
:104350006084F7E795F82703FFF703FF034695F816
:104360002803FFF7FEFE181A6084EBE795F8270391
:10437000FFF7F7FE034695F82803FFF7F2FE181A39
:104380006087B4F922109F48814200DA6084B4F952
:10439000221040F6B83081427FF77AAF608470BD5A
:1043A00010B50D2827D009DC3DD2DFE800F02C2421
:1043B0002C242C242424242424243400862812D0C1
:1043C0000EDC83280FD006DC0E281CD080280AD0F3
:1043D000822828D107E0842805D0852823D102E04F
:1043E000873804281FD80120FFF7E4FABDE8104001
:1043F0000020FFF7C5BA0120FFF7DCFABDE8104046
:104400000120FFF7BDBA0020FFF7D4FABDE8104045
:104410000120FFF7B5BA0020FFF7CCFABDE8104045
:104420000020FFF7ADBA10BD10B508285DD2DFE857
:1044300000F0040F1A25303B46510020FFF708FB1F
:104440000020FFF7EBFABDE810400020FFF7CCBAE0
:104450000020FFF7FDFA0020FFF7E0FABDE810406A
:104460000120FFF7C1BA0020FFF7F2FA0120FFF7A1
:10447000D5FABDE810400020FFF7B6BA0020FFF7DC
:10448000E7FA0120FFF7CAFABDE810400120FFF764
:10449000ABBA0120FFF7DCFA0020FFF7BFFABDE856
:1044A00010400020FFF7A0BA0120FFF7D1FA00204A
:1044B000FFF7B4FABDE810400120FFF795BA0120DC
:1044C000FFF7C6FA0120FFF7A9FABDE81040002067
:1044D000FFF78ABA0120FFF7BBFA0120FFF79EFA27
:1044E000BDE810400120FFF77FBA10BD02464249E7
:1044F000092A08D2DFE802F00705080B0E1114178D
:104500001A0091F89E02704791F89F02704791F847
:10451000A002704791F8A102704791F8A20270477B
:1045200091F8A302704791F8A402704791F8A50290
:1045300070472DE9F84F00242F4FDFF8C480DFF8D3
:10454000B4A0DFF8B89007F1D40BA8F1140601204D
:10455000FFF798FA21465846F6F736FB50B107EBBD
:10456000440090F86B1390F86A0301EB002028F8E0
:10457000140065E0601CC0B2FFF7B8FF062843D006
:104580003D1995F8E500FFF70BFF2046FFF74CFFBC
:104590000A2003F055FD0B215046FFF7FAFD26F8DF
:1045A000140095F8E5000C2805D036F81400FFF744
:1045B000EEFD26F8140095F8E500032812D0052832
:1045C00010D0C11F03290DD983280BD0852809D00D
:1045D0008738032806D936F914102046FFF787FBE1
:1045E00026F8140095F8E500042812D0842810D08D
:1045F00018E00000002401401C6D00204002002053
:10460000F01100200CFEFFFFB9F8120028F814008A
:1046100016E099F80910082902D289F80A4001E049
:1046200089F8094036F9141000232246FFF776FC7A
:1046300026F81400F84931F81410084428F814003A
:10464000641CE4B2082C82D30A215046FFF7A1FD76
:10465000A9F80C0099F8010000287DD03220EF491C
:10466000009001230022081F01F077FAD9F84000DA
:1046700018F06CFCA9F83600D9F8440018F066FC74
:10468000308297F8D902002867D040F2DB20FDF78E
:104690006EF80002A9F8200040F2DA20FDF767F872
:1046A000B9F820100844A9F82000B9F920004FF407
:1046B0007A76B04201DDA9F82060B9F92000002720
:1046C000002801DAA9F82070B9F92010B9F93600EC
:1046D000F9F74FF8A9F818000025002408215046E2
:1046E000FFF757FD0544032003F0AAFC641CE4B265
:1046F0001E2CF3D31E20B5FBF0F018F07BFC044613
:10470000204618F03FFCA9F81400C549204618F0CF
:10471000B9FCC44918F024FBC34918F0B3FCC349E1
:1047200018F01EFB18F012FC01460B20FFF7DFFA11
:10473000A9F814000025002409215046FFF729FD9F
:104740000544012003F07CFC641CE4B2142CF3D378
:104750001420B5FBF0F001E04AE05FE0642148433B
:10476000000B00EB4000A9F8160001215046FFF7AE
:1047700010FD00B243F6D00148430014A9F8300000
:1047800004215046FFF705FD00B243F6D00148432F
:104790000014A9F832000C215046FFF7FAFCC0EBD8
:1047A000C0004000B0FBF6F0A9F80E000D21504605
:1047B000FFF7EFFCC0EBC0004000B0FBF6F080B2AA
:1047C000A9F81000B9F80E100F2901D80F285BD9ED
:1047D00099F80B000A2802D2401D89F80B0099F8BD
:1047E0000B000A2802D3012089F80200BDE8F88FE7
:1047F0000220F8F78AFE142003F022FC0220F8F7CA
:1048000049FF30820020F8F780FE322003F018FCC8
:104810000020F8F73FFFA9F8360032E797F80001CB
:10482000834C50B3B6F910100920FFF760FA2080CE
:10483000B9F81E100820FFF75AFAB9F834100844E6
:1048400080B2A9F81C004FF4C871884201D2A9F8BF
:104850001C1099F80100012812D0B9F93610B4F9EA
:104860000000F8F76EFFA9F820007249B9F820009F
:1048700009880844A9F8200017E7308A2080D7E784
:104880002088A9F82000F0E799F80B0010B1401E2D
:1048900089F80B0099F80B000028A7D189F802705D
:1048A000A4E710B5FFF708F9BDE81040FFF771B9AC
:1048B000014600208A1E0B2A0CD2DFE802F00C0B06
:1048C0000B06060606060606060053483830491F42
:1048D00030F91100704751484438B0F93C00704736
:1048E0002DE9F0414D4A0020443A10714A4E012111
:1048F000323E3578002D06D173880C2B02D93172E7
:10490000117100E030724C4B012D93F86E400CD1C8
:1049100093F86C54A54202D03172117100E03072EC
:10492000B5790DB1307200E031723B4F283F3E4601
:104930003D7876882DB90C2E02D93972117100E0BC
:104940003872012D0FD193F86DC4A44502D039728D
:10495000117100E0387297F806C0BCF1000F01D069
:10496000387200E03972DFF8B0C0ACF11E0C9CF870
:10497000007057B9BCF80280B8F1020F03D98CF867
:104980000810117101E08CF80800012F11D193F883
:104990006E74A74203D08CF80810117101E08CF8F6
:1049A00008009CF8064014B18CF8080001E08CF86F
:1049B0000810DFF864C0ACF10A0C64469CF8007083
:1049C00064883FB90E2C03D08CF80810117101E0F7
:1049D0008CF80800012F0FD1152C03D08CF808108B
:1049E000117101E08CF808009CF8064014B18CF8B5
:1049F000080001E08CF80810DFF81CC0ACF1140CC2
:104A000064469CF800706488D7B90E2C16D08CF8D8
:104A10000810117114E00000B81100208402002079
:104A200000803B4500F07F450000204100007C42B3
:104A30006C000020400000201C6D00208CF8080055
:104A4000012F0FD1152C03D08CF80810117101E043
:104A50008CF808009CF8064014B18CF8080001E0BE
:104A60008CF8081054793CB993F8B770022F02D033
:104A70009171117100E09071012C07D193F8B84049
:104A8000022C02D09171117100E09071002D05D1BE
:104A900093F8A230B34203D0D1711171BDE8F08117
:104AA000D071FBE770B5FFF71BFF3A4E96F86A042A
:104AB000012837D1384C3949A4F11405B4F9040060
:104AC000B5F90430364A984203DA042008701070B1
:104AD00002E0002008701070287818B9A878FFF755
:104AE000E7FEA8802C4D0A3D287818B9A878FFF772
:104AF000DFFEA880207818B9A078FFF7D9FEA08043
:104B000096F86B0401280DD1234926480A310A780A
:104B10000AB9028C8A80204914310A78002A01D10E
:104B2000008C888070BDF0B51A4C0125002194F8E6
:104B30006A241C48012A0AD0C170C078012805D116
:104B400019480288428004F89E1F6570F0BD027902
:104B50000AB1C170F1E70F4BDFF83CC00E4F5A7C31
:104B60009B7CACF1140C02EB0322BCF9043094F8EA
:104B70006B649A1AB7F904301EB19A4207DDC5700A
:104B8000DBE79A4201DDC570D7E7C170D5E7C17098
:104B9000D3E700001C6D00209A1100203B0000208C
:104BA0002C00002040020020540000202DE9F04F8E
:104BB000A1B001211020FBF758F901212020FBF7BB
:104BC00054F901210820FBF750F9FC4C4FF4005038
:104BD000217A04290BD30121FBF747F90121112088
:104BE000FBF743F901210220FBF74AF906E0012116
:104BF000FBF73BF901211120FBF737F9217AF04847
:104C000018274FF00308042908D34FF0C001ADF86E
:104C100060104FF03001ADF8201003E04FF47071D8
:104C2000ADF840100FD38DF863708DF8628018A92D
:104C3000F3F7FBFF8DF823708DF8228008A9E14877
:104C4000F3F7F3FF06E08DF843708DF8428010A96A
:104C5000F3F7EBFF207A04280BD301210920FBF79F
:104C600004F90121D848F4F771F80121D748F4F785
:104C70006DF8D24800250224007AD54E4FF0010984
:104C80004FF47A7B4FF0700A042824D3ADF858B063
:104C9000ADF85440ADF85A50ADF8565015A930460D
:104CA000FBF722FAADF844A0ADF84690ADF84C40C1
:104CB000ADF818B0ADF81440ADF81A50ADF8165074
:104CC00005A9C448FBF710FAADF804A0ADF80690AA
:104CD000ADF80C4011E0ADF838B0ADF83440ADF8A7
:104CE0003A50ADF836500DA93046FBF7FDF9ADF856
:104CF00024A0ADF82690ADF82C40B048007A0428E6
:104D000010D311A93046FBF728FA11A93046FBF75A
:104D10005DFA01A9AF48FBF720FA01A9AD48FBF7FE
:104D200055FA0FE009A93046FBF717FA09A93046F2
:104D3000FBF74CFA09A93046FBF788FA09A9304677
:104D4000FBF7C2FA08213046FBF7A2FD08213046E6
:104D5000FBF7A4FD9948007A042808D308219D4850
:104D6000FBF796FD08219B48FBF798FD0FE0082113
:104D70003046FBF78DFD08213046FBF78FFD0821FB
:104D80003046FBF795FD08213046FBF797FD0121E2
:104D90003046FBF77AFC01213046FBF782FC01210B
:104DA0000420FBF76DF88548007A042807D3012119
:104DB0000220FBF765F801218648FBF766FC01211C
:104DC0002120FBF752F801210803F3F7BFFF4FF44E
:104DD000E040ADF880008DF883708DF8828020A9C6
:104DE0007D48F3F722FFADF878B0ADF87440ADF828
:104DF0007A50ADF87650794D1DA92846FBF774F925
:104E0000ADF864A0ADF86690ADF86C4019A92846DD
:104E1000FBF7A3F919A92846FBF7D8F919A92846E1
:104E2000FBF714FA08212846FBF732FD0821284633
:104E3000FBF734FD08212846FBF73AFD01212846FF
:104E4000FBF723FC21B0BDE8F08F0B461146012B88
:104E500007D0022B07D0032B07D0042B07D1FBF779
:104E60003FBEFBF737BEFBF737BEFBF737BE7047D9
:104E700030B40346514A574C5548127A062B27D274
:104E8000DFE803F026191D030E21042A04D320466F
:104E90000A4630BC0121D8E70A4630BC0321D4E7DA
:104EA000042A04D320460A4630BC0221CDE70A4634
:104EB00030BC0421C9E70A4630BC0121C5E70A46D7
:104EC00030BC0221C1E70A4630BC01214348BCE79F
:104ED00030BC7047414B002804D04FF47A72032154
:104EE0001846B2E7002203211846AEE73B4B0028E4
:104EF00004D04FF47A7202211846A6E7002202215C
:104F00001846A2E72DE9F84F83463548421C02F1C6
:104F1000010A00789AF800101278BBF1080F6CD2E1
:104F2000DFE80BF06B040F1B27333F60002500F018
:104F3000010601F0010402F00107A8464FF0010943
:104F40005BE00125C0F34006C1F34004C2F3400713
:104F50004FF002084FF003094FE00225C0F380062E
:104F6000C1F38004C2F380074FF004084FF0050935
:104F700043E00325C0F3C006C1F3C004C2F3C00779
:104F80004FF006084FF0070937E00425C0F300167C
:104F9000C1F30014C2F300174FF008084FF00909DD
:104FA0002BE00525C0F34016C1F34014C2F34017AF
:104FB0004FF00A084FF00B091FE000001C6D0020A5
:104FC00000100140000C01400004300000081A00ED
:104FD000003401400004004000140140000800407B
:104FE000940200200625C0F38016C1F38014C2F39A
:104FF00080174FF00C084FF00D09B74245D1FF481C
:1050000041460089F5F7C2FD0090A6B10020009945
:10501000884220D08EB10022F84841460830F5F78A
:10502000C6FDF648F649009A0A3042B1294491F883
:105030004211415507E00120E9E70122ECE729444C
:1050400091F849114155405D28B1EC48012249468B
:105050000830F5F7ACFDE94D49462889F5F796FD8E
:10506000002812D185F801B007B90124BBF1080F5F
:105070000BD2DFE80BF00A040C131A21282F9AF840
:10508000000064F300008AF80000BDE8F88F9AF889
:10509000000064F341008AF80000F6E79AF8000087
:1050A00064F382008AF80000EFE79AF8000064F3E6
:1050B000C3008AF80000E8E79AF8000064F30410DF
:1050C0008AF80000E1E79AF8000064F345108AF8D6
:1050D0000000DAE79AF8000064F386108AF800000E
:1050E000D3E72DE9F84FC748DFF81C830078002884
:1050F00023D00124DFF804A34FF000090AF1040AC9
:10510000AAF10106F51EAF1C2046FFF7FBFE6878EA
:10511000002877D0012803D09AF80010CA0772D06F
:1051200038783178401C60F3000131709AF8000043
:1051300020F001008AF80000CDE0B8F90000C8288E
:1051400015DA4FF47A710120FFF792FE0021022058
:10515000FFF78EFE00210320FFF78AFE00210420C6
:10516000FFF786FE00210520FFF782FE61E0B0F523
:10517000C87F15DA00210120FFF77AFE4FF47A711B
:105180000220FFF775FE00210320FFF771FE0021CA
:105190000420FFF76DFE00210520FFF769FE48E0BF
:1051A000B0F5167F15DA00210120FFF761FE00211E
:1051B0000220FFF75DFE4FF47A710320FFF758FEDF
:1051C00000210420FFF754FE00210520FFF750FEC8
:1051D0002FE0B0F5487F17DA00210120FFF748FEE5
:1051E00000210220FFF744FE00210320FFF740FECC
:1051F0004FF47A710420FFF73BFE00210520FFF7F2
:1052000037FE16E069E027E000210120FFF730FEBD
:1052100000210220FFF72CFE00210320FFF728FECB
:1052200000210420FFF724FE4FF47A710520FFF7D8
:105230001FFE764CB8F8002002212046FFF705FE3D
:10524000B8F8022003212046FFF7FFFDBDE8F84F24
:105250004FF4FA7002F0F4BE022801D08A070BD591
:10526000387832784010401C60F34102327021F0EF
:1052700002008AF800002EE0032801D04A070BD56F
:10528000387832788010401C60F38202327021F04E
:1052900004008AF800001EE0042801D00A070BD59C
:1052A00038783278C010401C60F3C302327021F0AD
:1052B00008008AF800000EE0052801D0C8060AD5CB
:1052C000387832780011401C60F30412327021F0FB
:1052D00010008AF8000085F80190641CE4B2062CE6
:1052E000FFF412AFDFF818A1DFF824B10AF1D600FD
:1052F0009AF86A100090062917D0002421460098D9
:10530000F5F762FC78B30AEB040090F8B9000328C3
:1053100031D021463F48F5F757FC28B300223748E3
:105320002146C01CF5F736FC25E03B48007838B133
:105330002878C0070DD0E9880120FFF799FD4EE0DD
:1053400000210120FFF794FD287800F0FE0028706E
:1053500045E04FF47A710120FFF78AFD297841F08A
:10536000010129703BE001E00122D8E72C492B48DC
:1053700001EB8411C8619BF80000012820D19AF844
:105380005302022802D001280ED014E021462548FD
:10539000F5F71AFC30B1002218482146C01CF5F779
:1053A000F9FB08E00122F7E72CB98AF8D690002132
:1053B000D620FCF7DDF9042C02D103208BF8000085
:1053C000641CE4B2052C99D33078C0072ED000219C
:1053D0000120FFF74DFD287800F0FE00287030789E
:1053E00080073AD42878800732D44FF47A710220AB
:1053F000FFF73EFD297841F0020115E092020020FE
:105400001C6D002077000020BE0000200008004036
:105410005A000020827000203B00002000007F43E3
:1054200004720020706F002029701EE02878C007E9
:1054300004D0E9880120FFF71BFDD0E74FF47A7113
:105440000120FFF715FD297841F001012970C6E719
:10545000E9880220FFF70CFD07E000210220FFF79A
:1054600007FD287800F0FD0028703078400711D43F
:105470002878400709D44FF47A710320FFF7F8FC2D
:10548000297841F0040129700CE0E9880320FFF736
:10549000EFFC07E000210320FFF7EAFC287800F08A
:1054A000FB0028703078000711D42878000709D451
:1054B0004FF47A710420FFF7DBFC297841F00801F2
:1054C00029700CE0E9880420FFF7D2FC07E00021F6
:1054D0000420FFF7CDFC287800F0F7002870307822
:1054E000C00611D42878C00609D44FF47A7105207B
:1054F000FFF7BEFC287840F0100028700CE0E98827
:105500000520FFF7B5FC07E000210520FFF7B0FC00
:10551000287800F0EF0028709BF8000001280DD1DA
:105520009AF85302022809D1012205210098F5F7C3
:1055300031FB012206210098F5F72CFB052100988C
:10554000F5F742FB80B39BF80000012803D19AF8DD
:105550005302022811D09AF8620300029AF86313EA
:10556000084400B29AF87B1079B111290DD082B2AB
:1055700002215748FFF769FC26E09AF8560200021C
:105580009AF85512084400B2ECE7012805D0002231
:1055900002214F48FFF759FC16E04FF47A720221BE
:1055A0004B48FFF752FC0FE0FFE79AF87B00A8B1E9
:1055B00001281ED004281CD011280FD0B8F80020D4
:1055C00002214348FFF741FC06210098F5F7FCFA59
:1055D000F0B39BF80000012824D027E0387880063B
:1055E00003D50120FFF782FCEEE70020FFF77EFCE9
:1055F000EAE79AF86A0401280DD19AF86F04B8F91D
:10560000001000EB8002B1EB420F04DA00EB8000E7
:105610004000A8F80000B8F8002002212C48FFF74D
:1056200014FCD1E79AF85302022816D09AF86403C2
:1056300000029AF86513084400B29AF87C1091B100
:105640009AF87B1011290ED082B20321204800E085
:105650001AE0BDE8F84FFFF7F8BB9AF857020102CD
:10566000084400B2E9E7012806D0BDE8F84F00225F
:1056700003211748FFF7E9BBBDE8F84F4FF47A72F2
:1056800003211348FFF7E1BB9AF87C0068B10128B9
:1056900016D0042814D0112807D0B8F80220BDE88D
:1056A000F84F03210A48FFF7D0BB3878400603D5EE
:1056B000BDE8F84F01200DE4BDE8F84F002009E4F3
:1056C000B8F80220BDE8F84F03210148FFF7BDBB41
:1056D0000008004010B5FBF734FE0120FBF76BFE1D
:1056E000012002F08DFC0120FBF75AFE012002F0A0
:1056F00087FC0020FBF75FFE0A2002F081FC0020FF
:10570000FBF74EFEBDE810400A2002F079BC10B550
:10571000FBF717FE0020FBF743FE012002F070FCB0
:105720000020FBF748FE012002F06AFC0120FBF795
:1057300037FE0A2002F064FC0120FBF73CFEBDE8C6
:1057400010400A2002F05CBC70B50546FBF7F9FD7D
:1057500080242C4203D10020FBF72DFE02E0012023
:10576000FBF729FE052002F04BFC0120FBF718FE99
:10577000052002F045FC0020FBF712FE012002F09C
:105780003FFC6408002CE4D1BDE87040FBF780BE0C
:1057900070B504460025FBF7F7FD4FF47A7607E075
:1057A000641EE4B201D2042070BD304602F028FC31
:1057B000FBF711FE0028F3D0284670BD2DE9F0411B
:1057C00005460E461746002028700120FBF7F3FD22
:1057D000FBF7A6FD80240120FBF7E2FD012002F08B
:1057E0000FFC3846FFF7D4FF8046032002F008FC88
:1057F000FBF7BBFDFBF7EAFD10B1287820432870CA
:105800000020FBF7CDFD012002F0FAFB6408002C1C
:10581000E1D1FBF796FDBEB10120FBF7CCFD0120E5
:1058200002F0EEFB0120FBF7BBFD052002F0E8FBD8
:105830000020FBF7B5FD0120FBF7BDFD142002F0B1
:10584000DFFB4046BDE8F0810020FBF7B4FDE6E752
:1058500010B5FFF73FFF0020FFF776FF002803D1C8
:10586000BDE8104006206FE710BD0000F949400078
:10587000087040F0010048707047F7E7FFF747BF36
:1058800070B50546FF20002340F2311410E0EA5CB9
:1058900050400822060603D584EA4000C0B201E069
:1058A0004006000E521ED2B2002AF3D15B1CDBB2BE
:1058B0008B42ECD370BD10B51446FFF7E1FFA04258
:1058C00001D0022010BD002010BD7CB504460D465D
:1058D000002101A8FFF772FF28B9002211460DF13F
:1058E0000500FFF76BFF20B9002229466846FFF745
:1058F00065FF28B99DF80020022101A8FFF7DBFF12
:105900009DF805109DF8042041EA022121807CBD0C
:1059100010B5FFF7DFFECF484078BDE81040FFF735
:1059200013BF70B50446200AFFF70EFF0546E0B22C
:10593000FFF70AFF284370BD10B5FFF7CBFEC5483F
:105940000078BDE81040FFF7FFBEF8B50646FFF748
:10595000F3FF05464FF45E50FFF7E3FF40EA05040E
:1059600014B9FFF7D5FF04462CB96422002168461C
:10597000FFF7ABFF044634B9002201210DF102000C
:10598000FFF7A3FF0446FFF779FF34B9BDF8020023
:10599000BDF8001040EA014030602046F8BD70B507
:1059A0000546FFF7C9FF044624B94FF22D30FFF733
:1059B000B8FF044614B9FFF7ABFF04462CB9002228
:1059C00001212846FFF781FF0446FFF757FF2046D5
:1059D00070BD10B5FFF7B0FF044624B943F2410093
:1059E000FFF79FFF0446FFF749FF204610BD10B5A3
:1059F00017F000FB984917F045FB984917F042FB58
:105A0000BDE81040964917F0ABB910B517F0F2FA9F
:105A1000944917F037FB914917F034FB904917F080
:105A20009FF9BDE81040904917F002BC2DE9FC41F8
:105A30000746884616461D46FFF77EFF04462000AF
:105A400005D196B1012E0AD0022E02D0802494B145
:105A500020E042F21640FFF764FF0446F7E742F207
:105A60000B40FFF75EFF0446F1E74FF41050FFF7DD
:105A700058FF0446EBE74FF47A7606E0FFF748FF5D
:105A800004462CB1304602F0BBFA6D1EEDB2F5D2E1
:105A900005B9042464B90022114601A8FFF715FFD7
:105AA0000546002201216846FFF70FFF40EA050482
:105AB000FFF7E4FE54B9BDF80400FFF7A6FF386015
:105AC000BDF80000FFF793FFC8F800002046BDE8CE
:105AD000FC812DE9FC4106460F4615469846FFF726
:105AE0002BFF04462CB995B1012D0AD0022D02D00E
:105AF000802494B114E042F61040FFF712FF0446F0
:105B0000F7E742F60D40FFF70CFF0446F1E742F6D7
:105B10000640FFF706FF0446EBE7FFF7F9FE0446F1
:105B20002CB94246002101A8FFF7CFFE04462CB94C
:105B3000002201216846FFF7C8FE0446FFF79EFEDB
:105B40004CB9BDF80400FFF760FF3060BDF80000FD
:105B5000FFF74DFF38602046B9E730B4029C002BB8
:105B600004D0012B05D0802030BC7047234630BCC8
:105B7000AFE7234630BC59E770B505460E46FFF740
:105B8000DBFE04462CB97DB3012D2ED0022D04D0AE
:105B90008024FFF773FE204670BD052E22D2DFE879
:105BA00006F003090F151B0042F22F00FFF7B9FEA4
:105BB0000446EEE742F22D10FFF7B3FE0446E8E795
:105BC00042F22B20FFF7ADFE0446E2E742F2293015
:105BD000FFF7A7FE0446DCE742F22A70FFF7A1FEBA
:105BE0000446D6E78024D4E726E0052E22D2DFE85B
:105BF00006F003090F151B0042F22400FFF791FE87
:105C00000446C6E742F22610FFF78BFE0446C0E7C3
:105C100042F22020FFF785FE0446BAE742F2223026
:105C2000FFF77FFE0446B4E742F22170FFF779FEEA
:105C30000446AEE78024ACE7052E2FD2DFE806F05D
:105C400003161C22280042F23200FFF76AFE0446C7
:105C50009FE70000A40200200000C842000020418D
:105C600000FF7F4700002F430000E14342F2301065
:105C7000FFF757FE04468CE742F23620FFF751FE4D
:105C8000044686E742F23430FFF74BFE044680E7D5
:105C900042F23770FFF745FE04467AE7802478E742
:105CA0007CB505460E46FFF747FE044624B94FF47F
:105CB0006040FFF736FE044614B9FFF729FE04469C
:105CC0002CB90022114601A8FFF7FFFD04462CB9AC
:105CD000002201216846FFF7F8FD04464CB9BDF8E3
:105CE0000400FFF792FE2860BDF80000FFF77FFE7A
:105CF0003060FFF7C3FD20467CBD10B5FFF71CFEEA
:105D0000044624B943F26D00FFF70BFE0446FFF78B
:105D1000B5FD204610BD10B5FFF70EFE044624B9B0
:105D200043F26600FFF7FDFD0446FFF7A7FD20469E
:105D300010BD70B5FFF700FE054643F2A200FFF765
:105D4000F0FD40EA0504FFF799FD1CB94CF2503014
:105D500002F056F9204670BD10B5244C4FF080502B
:105D60002060234802F04CF9A0142060BDE81040E8
:105D70004CF2503002F044B938B5010A8DF80010E9
:105D80008DF8010002216846FFF77AFD04469DF870
:105D90000000FFF7D9FC18B99DF80100FFF7D4FC0B
:105DA000002802D12046FFF7CFFC38BD10B51149BD
:105DB00016F068FF104916F0D3FF104917F062F98A
:105DC00017F0E0F880B210BD10B50D4916F0C8FF0D
:105DD0000A4917F057F917F0D5F880B210BD0348FB
:105DE00008380068C0F3802070470000100C0140A4
:105DF000A08601000000344200002F4300FF7F47CF
:105E00000000C842F0B503460025084600260A2ACD
:105E100001D00670F0BD002B1DD005DA4FF02D0229
:105E200000F8012BC3F1000342F210724FF00A0791
:105E300093FBF2F454EA050C06D004F1300500F8A7
:105E4000015B04FB1233012592FBF7F2002AEFDC21
:105E500006700846F0BD3022027046700846F0BD5C
:105E60000FB430B585B005460AA800900EE05C2955
:105E700014D025292CD0521C28460992FAF786FF07
:105E800080212846FAF7EFFF0028F9D0099A117807
:105E90000029ECD105B030BC5DF814FB521C09920E
:105EA00010786E280CD0722802D0521C0992E7E7B5
:105EB0000D212846FAF76AFF0998401C0990DFE790
:105EC0000A212846FAF762FF0998401C0990D7E793
:105ED000521C09921078642819D0732802D0521CE1
:105EE0000992CDE7009810C8009009E02846FAF71B
:105EF0004DFF80212846FAF7B6FF0028F9D0641C30
:105F000021780029F2D10998401C0990B8E700983F
:105F100008C800900A2201A91846FFF773FF01ACD8
:105F200009E02846FAF732FF80212846FAF79BFF5E
:105F30000028F9D0641C21780029F2D10998401C6E
:105F400009909DE708B54FF4A060F2F7E5FB342017
:105F50008DF8000000208DF801008DF8020001206E
:105F60008DF803006846F2F7DCFB08BD10B586B07B
:105F70000121C804F9F784FF01211020F9F775FF0A
:105F80004FF48060ADF8140018208DF8170003203E
:105F90008DF81600F94C05A92046F2F746FEE114EB
:105FA000ADF8141004218DF8171005A92046F2F75A
:105FB0003CFE4FF4E13001900020ADF80800ADF850
:105FC0000A00ADF80C00ADF810000C20ADF80E0082
:105FD000EB4C01A92046FAF7FDFD012240F22551C4
:105FE0002046FAF77EFE012240F224412046FAF7CD
:105FF00078FEFFF7A7FF01212046FAF766FE06B0FC
:1060000010BD08B510208DF8030003208DF80200A4
:1060100001212020F9F729FF0420ADF8000069468E
:10602000D848F2F702FE08BD10B5FFF7EAFFFFF708
:106030009DFFBDE810400421D248F2F765BE10B5BF
:10604000D04C04212046F2F761FE4FF4FA7001F0C3
:10605000F7FF2046BDE810400421F2F755BE2DE9B8
:10606000F04706460D4691461F46DFF81C83B8F8F8
:1060700000046FF30E00A8F800040024DFF800A36A
:106080000BE0315D5046FAF781FE80215046FAF769
:10609000EAFE0028F9D0641CA4B2BC42F1D3B8F8DF
:1060A00000046FF30E00A8F8000498F8010420F033
:1060B000800088F80104002404E0322001F0C0FFD1
:1060C000F2F79FFE98F80104000604D42046641CF1
:1060D000A4B20A28F1D3B8F800140020C1F30E01CD
:1060E00008F8010085B1B9F1000F0DD02946A64886
:1060F00013F0B6FF28B94946A34813F0B1FF0028B2
:1061000000D00120BDE8F0873DB129469E4813F03C
:10611000A7FF0028F6D00120F4E749469A4813F07B
:106120009FFF0028EED00120ECE72DE9F0410E465C
:106130001746024695A19248FFF792FE56EA0700DD
:106140000ED0914DB5F800046FF30E00A5F80004D1
:1061500095F8010420F0800085F80104002407E090
:106160000120BDE8F081322001F06AFFF2F749FE1C
:1061700095F80104000604D42046641CA4B20A2841
:10618000F1D3B5F800140020C1F30E0168546EB1CC
:1061900067B131467C4813F063FF28B939467A4825
:1061A00013F05EFF0028DCD00120DAE73EB1314673
:1061B000754813F055FF0028D3D00120D1E73946A8
:1061C000714813F04DFF0028CBD00120C9E770B50E
:1061D000002404216B48F2F797FD4FF47A7001F028
:1061E0002FFF4FF4FA750CE02B46002269A16AA03C
:1061F000FFF79BFF08B1022070BDFFF720FF641C72
:10620000E4B20A2CF0D301D0012070BD002070BD93
:1062100040F6C413002805D0012807D0022809D071
:10622000002070475DA25BA15FA07EE75BA259A141
:1062300060A07AE759A257A161A076E700B59FB0A8
:106240000B46024661A101A813F008FD41F2883314
:10625000002250A101A8FFF768FF1FB000BD00B5E4
:106260009FB00B4602465EA101A813F0F7FC41F275
:106270008833002247A101A8FFF757FFEDE72DE97A
:10628000F041CEB0642135A813F0D8FF00245A4D58
:1062900013AE281906EB840190F86A000A22FFF772
:1062A000B1FD641CE4B2042CF3D300240FAF281911
:1062B00007EB840190F86E000A22FFF7A3FD641C2F
:1062C000E4B2042CF3D300240DF12C08281908EBB8
:1062D000840190F872000A22FFF794FD641CE4B276
:1062E000042CF3D312A811A9CDE9081010AACDE906
:1062F00006720EA80DA9CDE9041016A815A90CAABE
:10630000CDE90010CDE90282331D13AA3BA135A8C7
:1063100013F0A4FC35AA44A117A813F09FFC4FF476
:106320007A6300221BA117A8FFF7FFFE4EB018E703
:1063300000B59FB00B460092024640A101A813F0A1
:106340008DFC4FF47A73002212A101A8FFF7EDFE35
:1063500083E700B585B0002801D0012200E00022CB
:106360003CA1684613F07AFC4FF4FA73002209A1AD
:106370006846FFF7DAFE05B000BD000000100140DE
:10638000004C0040001401400E12002025730D0A3D
:10639000000000004F4B0000415400006E6F20636E
:1063A00068616E676500000041542B43574D4F44B0
:1063B000453D310041542B43574D4F44453D32003C
:1063C00041542B43574D4F44453D330041542B43DB
:1063D000574A41503D222573222C2225732200006A
:1063E00041542B43574A41505F4445463D22257353
:1063F000222C222573220000902200202225732EB9
:1064000025732E25732E2573222C2225732E25739A
:106410002E25732E2573222C2225732E25732E25CF
:10642000732E25732200000041542B4349505354CE
:10643000415F4445463D25730000000041542B4315
:10644000575341503D222573222C222573222C3193
:106450002C25640041542B4349504D55583D25642B
:1064600000000000F0B5B9B004460F4615461E46C0
:10647000642120A813F0E2FE14B1012C0FD107E033
:106480003B46F8A2F8A120A8009513F0E7FB06E030
:106490003B46F9A2F4A120A8009513F0DFFB052EDE
:1064A00006D220AB3246F5A102A813F0D7FB04E0D8
:1064B00020AAF7A102A813F0D1FB4FF47A63F8A247
:1064C000AFF2301102A8FFF730FE39B0F0BD2DE970
:1064D000F041BAB08046409F0E4615461C466421E6
:1064E00021A813F0ABFECDE900654346E2A2F0A17E
:1064F00021A8029413F0B2FB052F06D221AB3A4635
:10650000DEA103A813F0AAFB04E021AAE0A103A8DE
:1065100013F0A4FB4FF47A63E1A2AFF2881103A851
:10652000FFF703FE3AB01CE610B59EB04FF4FA74C4
:1065300000280ED00B460122E2A1684613F08EFB24
:1065400023460022AFF2B4116846FFF7EEFD1EB0FD
:1065500010BD0B460022DBA1684613F07FFB2346EB
:106560000022AFF2D0116846FFF7DFFDEFE710B56C
:106570004FF4FA730022AFF2E411D7A0FFF7D5FD74
:10658000D8B1D9A1DB4813F06BFD08B1022010BDD2
:10659000D9A1D84813F064FD08B1032010BDD9A1DA
:1065A000D44813F05DFD08B1042010BDD8A1D14836
:1065B00013F056FD08B1052010BD062010BD10B522
:1065C00000244FF4FA730022AFF23821C2A0FFF783
:1065D000ACFD00282DD0D1A1C64813F041FD00B17B
:1065E0000124D2A1C34813F03BFD10B144F00204D2
:1065F00001E024F00204D1A1BE4813F031FD10B136
:1066000044F0040401E024F00404D0A1B94813F0DC
:1066100027FD10B144F0080401E024F00804CFA1E4
:10662000B44813F01DFD10B144F0100401E024F053
:106630001004204610BD2DE9FE4380460E46174645
:106640004FF4FA794B460022AFF2B821C7A0FFF70A
:106650006CFD00250024C8A1A64813F001FD10B16F
:10666000C21D00203BE00020BDE8FE83115C2E2906
:1066700002D0032D27D028E0012C04D0022C06D014
:10668000032C0ED01BE09DF80810715517E09DF803
:1066900008109DF8093001EB810103EB41017155B0
:1066A0000DE09DF8083064214B439DF8091001EB83
:1066B000810103EB41019DF80A30194471556D1CAD
:1066C000EDB2002409E022290BD0303923460DF128
:1066D000080C641CE4B20CF80310401CC0B2B842B1
:1066E000C4D3012C04D0022C06D0032C0ED01BE006
:1066F0009DF80800705517E09DF808009DF80910F6
:1067000000EB800001EB400070550DE09DF8081093
:10671000642041439DF8090000EB800001EB40003C
:106720009DF80A10084470554B460022AFF29C3188
:1067300093A0FFF7FAFC0025002495A16D4813F003
:106740008FFC20B100F10B0300206E462BE00020EF
:106750008AE7195C3A2902D0052D0ED00FE0022CF1
:1067600007D19DF801109DF8002001EB021108F8F7
:1067700005106D1CEDB2002413E0222915D0A1F103
:106780003002092A04D82146641CE4B2725408E09D
:10679000A1F16102052A04D857392246641CE4B2EB
:1067A000B154401CC0B2B842D3D3022C07D19DF8DB
:1067B00001009DF8001000EB011008F805004B46A1
:1067C0000022AFF2304176A0FFF7AFFC002478A1A1
:1067D000484813F045FC18B10C300021774B0BE012
:1067E000002041E7425C222A08D025461D44641C53
:1067F000E4B2AA72491CC9B2B942F3D3012033E70B
:1068000010B54FF4FA7423460022AFF278416CA021
:10681000FFF78BFC38B123466DA2AFF28841BDE88B
:1068200010406CA081E4002010BD10B54FF47A70C8
:1068300001F006FC6AA16B48FFF712FBBDE81040AF
:106840004FF4FA7001F0FCBB70B51446ADF5087D4D
:106850000D461A46B4F5FA7F03D900200DF5087DE0
:1068600070BDC1E054435000222573222C222573B1
:10687000222C2573000000005544500041542B4346
:10688000495053544152543D25642C257300000057
:1068900041542B43495053544152543D25730000F9
:1068A000414C5245415920434F4E4E454354000000
:1068B000222573222C222573222C25642C25642C5E
:1068C0002564000041542B434950534552564552CC
:1068D0003D25642C2573000041542B4349505354EB
:1068E00041545553000000005354415455533A321B
:1068F0000D0A00000E1200205354415455533A33F0
:106900000D0A00005354415455533A340D0A000007
:106910005354415455533A350D0A00002B43495006
:106920005354415455533A302C0000002B434950E6
:106930005354415455533A312C0000002B434950D5
:106940005354415455533A322C0000002B434950C4
:106950005354415455533A332C0000002B434950B3
:106960005354415455533A342C00000041542B43A6
:10697000494653520000000053544149502C220014
:1069800041542B4349505354414D41433F00000073
:106990002B4349505354414D41433A2200000000DB
:1069A00041542B43574A41505F4355523F0000002A
:1069B0002B43574A41505F4355523A0090220020E2
:1069C00041542B4349504D4F44453D310000000098
:1069D0003E00000041542B43495053454E440000B3
:1069E0002B2B2B00004C0040B64E38B12A46AFF29C
:1069F00054113046FFF734FA01202FE7052A05D25B
:106A00002346B1A101A813F029F904E02246B3A15D
:106A100001A813F023F901AAAFF290613046FFF705
:106A20001FFAC82001F00CFB64200090A3B20022E2
:106A3000AEA12846FFF713FB10E700B59FB0642115
:106A400006A813F0FBFB06AAAAA101A813F006F9F9
:106A50004FF47A630022AFF2C46101A8FFF765FB2F
:106A60000CE42DE9F04781460027DFF89C82B8F856
:106A700000046FF30E00A8F8000498F8010420F059
:106A8000800088F8010440F20241404613F0B4FB54
:106A9000002400269D4D3DE0022001F0D1FA297826
:106AA000182904D0192913D0162918D030E0FFF77F
:106AB000E6FB68B39648974902780A7042784A70B4
:106AC00082788A70C078C870FFF7B9FA2E701FE01C
:106AD000FFF7B3FFE0B1FFF7B2FA2E7018E04FF402
:106AE000FA730022AFF254718BA0FFF71EFB00B1C6
:106AF0002E7088484021603813F07EFB85482021A5
:106B0000203813F079FB87490120487108F024FAF6
:106B1000F2F777F998F80104000604D42046641CC3
:106B2000A4B26428B8D3B8F80004C0F30E0008F883
:106B30000060B9F1000F01D0734F05E07AA17248EF
:106B400013F08EFA00B1704F3846BDE8F08770B58B
:106B5000027A2C2A01D0002082E6827A3A2A10D1C9
:106B6000437A303B092B0CD89BB2002205E08418F5
:106B7000E47A01F8014B521C92B29A42F7D31846BC
:106B80006EE6C37A6FF02F053A2B03D0047B3A2CC4
:106B90001AD03EE0437A303B092B3AD8302A38D31A
:106BA000392A36D803EB830305EB43031A4493B227
:106BB000002205E08418247B01F8014B521C92B29C
:106BC0009A42F7D318464BE6447A303C092C20D839
:106BD000302A1ED3392A1CD8302B1AD3392B18D877
:106BE00004EBC406303A06EB041402EB820203EB1A
:106BF000840305EB42021A4493B2002205E0841894
:106C0000647B01F8014B521C92B29A42F7D31846AA
:106C100026E6002024E610B504464021444813F03F
:106C2000EBFA434914B1012C03D004E0652008803D
:106C300001E0672008801D2048803E4802788A8055
:106C40004278CA8082780A81C2784A8109228A8180
:106C50008379CB812F4A14780C8254784C829478B3
:106C60008C82D478CC8232F8684C0C8361244C83BB
:106C7000007A888330480068C0F3072444EA00247F
:106C80004C8481F82430030C1B0243EA1060A1F805
:106C90003900002081F83B0032F8662C8A8781F8A1
:106CA0003E0081F83F0025490120087010BD0B0A05
:106CB0000370417000218170C170110A017142712D
:106CC00070470000004C004041542B43495053454D
:106CD0004E443D25642C25640000000041542B43A4
:106CE000495053454E443D256400000053454E44F1
:106CF000204F4B0041542B4357444843505F444579
:106D0000463D312C310000000E12002013030020FC
:106D10007A720020FA22002041542B524553544FDE
:106D2000524500004D0400202B4950440000000053
:106D3000101600201C6D00200C000020A70200206F
:106D400070B50024FE4D4FF4FA76FFF710FCA871E1
:106D5000401E032808D3304601F072F9F2F751F8CB
:106D6000641CE4B20A2CF0D3F649A879C881032840
:106D700007D13346BDE870400022F3A1F3A0FFF72E
:106D8000D4B970BD70B500244FF47A7504E0F2F701
:106D900038F8642001F054F92B460022EAA1EFA054
:106DA000FFF7C3F9002804D12046641CE4B214287C
:106DB000EDD370BD10B5002404E0F2F722F8642092
:106DC00001F03EF964230022DFA1E7A0FFF7ADF94F
:106DD000002804D12046641CE4B21428EDD310BD71
:106DE00010B5002404E0F2F70CF8642001F028F953
:106DF00064230022D4A1E0A0FFF797F9002804D172
:106E00002046641CE4B21428EDD310BD10B5DE4852
:106E1000C07801280CD14FF47A7001F011F9DB49E8
:106E20000120487108F098F8BDE81040F2F710B959
:106E300010BD2DE9F047D44E0025B570C04FB8798C
:106E4000012860D0387850B135704FF4FA730022C1
:106E5000BDA1C9A0FFF769F9C82001F0F1F83878A1
:106E600001281CD10020FFF7D3F9C82001F0E8F871
:106E70000024DFF8CC9209F14A0809F10A0904E07C
:106E8000F1F7BFFF642001F0DBF841464846FFF709
:106E9000E6F920B92046641CE4B20A28F0D37878D9
:106EA000A84F012829D100244FF47A7804E0F1F7A3
:106EB000A8FF404601F0C4F8FFF7E1F920B92146E8
:106EC000641CE4B20529F2D33C81002404E0F1F70C
:106ED00098FF642001F0B4F84346ADA29AA1AEA099
:106EE000FFF723F920B92046641CE4B20528EED34D
:106EF0007C81C82001F0A4F8B570B889401CB88125
:106F0000BDE8F0471CE7BDE8F0878CB0142009907D
:106F10009D4F00243C708A4D0220E87168884FF62E
:106F2000FF76002801D0B04202D14FF4FB70688098
:106F30008348A97A0A300B90FF2906D1E87AFF2806
:106F400003D140210B9813F057F97D4895F84A106A
:106F50004A300A90FF2907D195F84B00FF2803D14A
:106F600020210A9813F048F98748C470A88808B10E
:106F7000B04202D14BF6C020A88071480A2207A96E
:106F80004088FEF73FFF4FF4FA65284601F058F8B5
:106F9000FFF74AF8FFF753F8284601F051F8FFF7DA
:106FA00016F980460125B8F1020F02D064488571B8
:106FB00004E0634805218171FFF73BFF784E05200F
:106FC00001F03EF8F1F71DFFB8F1020FF7D1DFF83D
:106FD00070A19AF8060002284AD08AF86A408AF816
:106FE0006B408AF86C408AF86D40674F387840B93A
:106FF0004FF4FA73002254A15BA0FFF796F800B19A
:107000003D70387878B30027FFF7B1FA8AF80600A8
:10701000642001F015F8F1F7F4FE9AF80600032851
:1070200004D938467F1CBFB20528EDD3052F02D303
:10703000FFF7FFFEC3E740210B9813F0DDF8202196
:107040000A9813F0D9F85148457107F085FF4FF4BD
:10705000FA7300223CA148A0FFF767F8642000F013
:10706000EFFFF1F7F5FF4FF4FA6000F0E9FFA6E754
:10707000454FB87828B34FF480694946494813F022
:10708000BBF84946464813F0B7F80020FFF7E9FC83
:1070900001464A46424813F038F8F079303800F09B
:1070A000FF0940493E48FFF752FD0246100086D0D6
:1070B000A9F10200022840D83A490878EE283DD0CC
:1070C000BAE01F4928226A3101F10C00FFF7B3FA38
:1070D00060B19AF86A0040B99AF86B0028B99AF83A
:1070E0006C0010B99AF86D00A8B1BD704FF4FA7732
:1070F0003B46002214A12CA0FFF717F80120FFF750
:1071000028F9F1F77EFE3B4600220FA10FA0FFF702
:107110000CF8002703E0BC70E8E7F1F772FE00947A
:10712000BAF8041002230A4623A0FFF7D0F918B9D1
:1071300038467F1CBFB247E048E0A0E06DE00000A9
:1071400090220020E87500204F4B000041542B4353
:107150004950434C4F53453D3500000041542B529C
:107160004553544F5245000041542B43575354410B
:107170005254534D4152540041542B435753544F92
:1071800050534D4152540000A60200204D040020EF
:10719000726561647900000041542B525354000021
:1071A000A8160020901E002041542B4349504D4FFB
:1071B00044453D30000000003235352E3235352E45
:1071C0003235352E323535000528A6D3002740F25A
:1071D000D24901E0F1F715FE494602230A46AFF213
:1071E00028000095FFF773F920B938467F1CBFB21D
:1071F0000528EFD3002701E0F1F703FE09AA07A94C
:107200000120FFF791F900287FF414AF38467F1C66
:10721000BFB20528BFF40EAFEEE7487810280BD1B7
:10722000887848B9C87838B9087928B9487918B938
:10723000887908B9C879D8B1484A88799279904252
:1072400005D0FF28E0D1C87919283FF4F3AE4449AE
:10725000052006F0D5FBFA883AB1F079414930387B
:10726000C3B20020FFF7F0FAFC80FFF7CFFDA6E6DF
:107270007F210B20FAF77CFAF1F7EAFE9FE6B9F1DD
:10728000000F15D0B9F1010FF1D1DFF8D4E09EF86D
:1072900000006428EBD17D7000209AF86A309AF8DB
:1072A0006BC09AF86C909AF86DA0C2F3850B2CE035
:1072B00000232B4902A800950BF055F90246501EF9
:1072C000B0F5FF7FD3D80123254902A80CF098FC24
:1072D000BA88002ACBD0F07923493038C3B20020D5
:1072E000FFF7B2FABC806AE60EEB80014A789A4258
:1072F00009D18A78624506D1CA784A4503D109790D
:10730000514500D17C70401CC0B25845ECD3787810
:107310000028ACD00020FFF77EFC14498C77CC7796
:1073200081F8204081F8214000200C4A13180F18E2
:1073300093F8483387F82530401CC0B21428F5D3A1
:1073400011F83E0F40F002000870F079402230380A
:10735000C3B206490020FFF777FA30E61C6D002023
:10736000901E00209C1C0020A81A0020101600204F
:1073700070B50024F74D04EB840005EB800000F0AD
:10738000F9FB641C052CF6D3F248643000F0F2FBE4
:10739000F048783000F0EEFBEE488C3000F0EAFB6D
:1073A000EC48A03000F0E6FBEA48B43000F0E2FB25
:1073B000E849E948643141631431816370BD70B5B7
:1073C00004461546102204F1340012F05EFF00203E
:1073D00084F84300052D00D30425E562201D00F04C
:1073E000D4FB04F1180000F0D0FB2461C5F10500C6
:1073F000A061646270BD70B506460D46442000F081
:107400004FFC044644B1B60045B12846206348B15C
:10741000A5223146F1F7ECFD204670BD304600F064
:107420003FFCF3E7204600F091FC0024F4E72DE94F
:10743000FF4F81B08246DDE90E68109917469B46E2
:107440003846FFF7D8FF0446C34DECB3216B781ED6
:1074500001EB800020F00709009732462046119B7F
:107460000299FFF7ACFF5A465146484600F0C8FB68
:107470002060B8F1000F01D0C8F8004000F0EBFB2D
:10748000A868401CA860286810B1A86938B10BE052
:107490002C60A868012807D1FFF76AFF04E028687C
:1074A000C06AB04200D82C60E06A2969884200D9DD
:1074B0002861E96A491CE9626969884200D9686102
:1074C00000EB8001A34800E008E000EB8100211DF3
:1074D00000F05EFB012400F0C6FB01E04FF0FF343A
:1074E000012C07D1A86928B12868C06AB04201D22E
:1074F00000F0ABFB05B02046BDE8F08F70B5054647
:1075000000F0A9FB944E3068854200D10025FDB102
:107510002C46201D00F062FBA06A18B104F118008F
:1075200000F05CFB8B48211DA03000F031FB70683F
:10753000401C7060F06A401CF06200F094FBB0697F
:10754000002807D0002D05D1BDE8704000F07DBBBC
:107550003468DEE770BD70B57F4DE869002803D060
:10756000286A401C286270BDE868401CE860E86832
:107570004FF0FF3670B9686BA96B6963A863A86A9E
:10758000401CA862686B0068A0B1686BC068C068E6
:1075900040682863E868296B8842E4D3686B006818
:1075A00050B1686BC068C4686068E968814205D200
:1075B000286370BD2E63EDE72E6370BD201D00F0C3
:1075C0000DFBA06A18B104F1180000F007FBE06A97
:1075D0006969884200D968615E4900EB800001EB6F
:1075E0008000211D00F0D4FAD8E72DE9F0410027F2
:1075F00000F031FB584EF069401EF061F069E8BBC5
:10760000B068D8B30025DFF84C8108F18C081CE085
:10761000D8F80C00C46804F1180000F0DFFA201D4F
:1076200000F0DCFAE06A7169884200D9706149496A
:1076300000EB800001EB8000211D00F0A9FAE06A58
:107640003168C96A884200D30125D8F800000028B3
:10765000DED1306A28B908E0FFF77DFF306A401EAE
:107660003062306A0028F7D10125012D02D0706AFE
:10767000012806D101270020706200E001E000F03F
:10768000E4FA00F0F0FA3846BDE8F08170B504463F
:10769000314D28684460E868844206D22968A86BA6
:1076A000091DBDE8704000F081BA2968686B091DAA
:1076B00000F07CFA286B844200D22C6370BD26480F
:1076C000C169491CC161704770B503460C46002270
:1076D000FFF7F5FF186804441F49CD68A84206D992
:1076E000A0420AD9C868844207D9012205E0A04215
:1076F00002D8C868844200D901221C6032B10868EF
:10770000001D00F06BFA2046FFF7C0FFFFF76DFF8A
:10771000002803D1BDE8704000F097BA70BD10B5E5
:1077200002460020002A0DD0FFF7C9FF0A48C168B1
:107730008C180068001D00F051FA2046FFF7A6FFE4
:10774000FFF753FF002803D1BDE8104000F07DBAD9
:1077500010BD00000C230020B002002010B504462C
:1077600000F079FA0CB9F7480468E46A00F07BFA93
:107770002046EDE72DE9F04106460D460027052D90
:1077800000D3042500F067FADFF8B883D8F80000CA
:10779000864200D1002646B13446E06AA8422AD08B
:1077A000854205D936B1012704E0D8F80040F4E756
:1077B00006B90127E562C5F10501A161E24D00EBC3
:1077C0008000616905EB8000814210D1201D00F02E
:1077D00005FAE06AD8F81410884201D9C8F81400F4
:1077E00000EB800005EB8000211D00F0D1F9012F96
:1077F00001D100F02AFABDE8F04100F034BAD149D5
:10780000C869002802D0012048627047CE4A02E0D1
:107810004869401E4861486900EB800052F820002A
:107820000028F5D0486900EB800002EB8000426838
:107830005268426000F108039A4201D152684260E6
:107840004068C0680860704770B5054600F003FAEC
:10785000BC4E3068854200D10025C5B12C46201DA4
:1078600000F0BCF9A06A18B104F1180000F0B6F9F4
:10787000B548211DB43000F08BF900F0F4F9002D6B
:107880000FD1B06928B1BDE8704000F0DEB93468AE
:10789000E5E7AD48B4300068B168884202D1002005
:1078A000306070BDBDE87040A9E70021A64B426979
:1078B000B4339A4206D1806AA3F12802904201D0E3
:1078C00000B901210846704770B50446002C25D048
:1078D0009C4D2868844221D000F0BDF92046FFF776
:1078E000E4FF012816D1201D00F078F9E06A6969EB
:1078F000884200D96861944900EB800001EB800068
:10790000211D00F045F9E06A2968C96A884201D35F
:1079100000F09BF9BDE8704000F0A5B970BD70B5EE
:10792000044600252046FFF7C0FF012808D1854EF8
:10793000F06938B1844804F118018C3000F028F95E
:10794000284670BDE06A3168C96A884201D30125C2
:1079500000E00025201D00F041F9E06A71698842CD
:1079600000D97061784900EB800001EB8000211D97
:1079700000F00EF9E4E710B50446206B00F0E6F9DC
:107980002046BDE8104000F0E1B970B56D4D686863
:1079900000281FD0FFF793FE6B4EA0363068B8B1B9
:1079A0000024FFF722FE002C14D100F054F9F068F7
:1079B000C468201D00F012F9A868401EA86068681D
:1079C000401E686000F04FF92046BDE87040D2E7E5
:1079D0000124E6E770BD5C4CFFF7D7FF2068012863
:1079E000FAD900F032F9F7E71FB5002400940194AA
:1079F00002942346642255A156480394FFF717FDCD
:107A0000012809D1F0F760FC4E4801218161C46072
:107A1000BDE81F4000F005B91FBD10B5F0F754FCDC
:107A2000484900208861BDE8104000F00DB910B54C
:107A300000F011F94348C46800F015F9204687E6C4
:107A400010B5F0F741FC3F48C468F0F744FC20460D
:107A50007EE63C488068704770B50D46394C216819
:107A6000183100F0A3F82068001D00F0B7F8681C7A
:107A700004D0E0682844BDE8704007E62168BDE80E
:107A800070403148091DB43000F082B870B5C0684C
:107A9000C46804F11800064600F0A0F8294DEA6910
:107AA0005AB1294831468C3000F072F8E06A2968F2
:107AB000C96A884212D3012070BD201D00F08EF8E3
:107AC000E06A6969884200D968611F4900EB80005B
:107AD00001EB8000211D00F05BF8E7E7002070BD9E
:107AE00018498A6A0260C9684160704770B50446E7
:107AF0000D4600F0B0F82868411C0AD0114B2168EF
:107B00009A6A914207D06168DA68914203D80124E9
:107B100010E000240EE06268D968891A814208D218
:107B2000D968891A401A28602046FFF7D9FF002437
:107B300000E0012400F097F8204670BD01490120C3
:107B400048627047B00200200C23002049444C4595
:107B500000000000D779010805488169002903D099
:107B6000C06918B10220ECE70020EAE70120E8E74D
:107B7000B002002000F1080141604FF0FF32826046
:107B8000C1600161002101607047002101617047FF
:107B9000426853684B6043688B60536899605160DA
:107BA000416008610168491C0160704710B50B68AD
:107BB0005A1C02D000F1080202E0026904E0526897
:107BC000546824689C42FAD953684B6099608A6073
:107BD000516008610168491C016010BDD0E90121B4
:107BE0009160D0E90112516001694A68824201D175
:107BF00082684A60002202610868401E086070477F
:107C000020384FF08073C36181610021416140F8E9
:107C1000202970474FF0E0201E4941610721016192
:107C2000704710B51C48016841F47F01016001688C
:107C300041F07F410160FFF7EDFF18490020086027
:107C4000F0F71AFB002010BD704713494FF0805029
:107C50001C390860704710B5F0F736FB0F48016813
:107C6000491C016010BD0D490868401E08600028CD
:107C700001D1F0F730BB704710B507494FF0805085
:107C80001C390860F0F720FBFFF765FCBDE81040E9
:107C9000F0F721BB3F19010020ED00E0EC020020CD
:107CA0002DE9F04104460025FFF709FD384E06F1A5
:107CB0000801706801F1080360B9364808600020C7
:107CC00048604FF480425A60186032484260036056
:107CD000012070603CB11034600704D004F007004C
:107CE000C0F108000444601E43F6FF72904228D29F
:107CF000274A0832096801E00A4601464868A0425E
:107D000002D208680028F7D199421AD015681035B8
:107D1000086810604868001B20280ED90B195860AD
:107D20004C605C681A48083000E0104602685768EA
:107D3000A742FAD302681A60036048683168081ADB
:107D40003060FFF752FC2846BDE8F08110B50028EE
:107D500018D010380446FFF7B2FC60680C490831AF
:107D600000E011460A6853688342FAD3086820602D
:107D70000C6007486168026811440160BDE810406A
:107D8000FFF733BC10BD0248006870477047000021
:107D9000F0020020D8230020704770B50446874DBC
:107DA00040212846F9F75FF80028F9D0A1B228460B
:107DB000F8F7ECFF204670BDF0B587B0054601210D
:107DC00044F20400F8F751F87C4E3046F8F7BAFE5A
:107DD0007015ADF8180003208DF81A0018208DF8E2
:107DE0001B00774F06A93846F0F71FFF3015ADF896
:107DF000180048208DF81B0006A93846F0F715FF3B
:107E0000B415ADF8184010208DF81B0006A93846AF
:107E1000F0F70BFF21463846F0F776FF25208DF866
:107E2000040000248DF805408DF8064001208DF8EF
:107E3000070001A8F0F775FC0295ADF80C40ADF80D
:107E40000E40ADF81040ADF814400C20ADF8120013
:107E500002A93046F8F7BEFE012240F22551304615
:107E6000F8F73FFF01213046F8F72FFF07B0F0BDCC
:107E700070B586B0054601210820F7F7F6FF01210D
:107E80008804F7F7FDFF4F4E3046F8F75BFE3015DC
:107E9000ADF8140003208DF8160018208DF8170097
:107EA000494C05A92046F0F7C0FEE014ADF81400D7
:107EB00048208DF8170005A92046F0F7B6FE2720C8
:107EC0008DF8000000248DF801408DF8024001205B
:107ED0008DF803006846F0F724FC0195ADF80840E2
:107EE0007014ADF80A00ADF80C40ADF810400C204D
:107EF000ADF80E0001A93046F8F76CFE012240F201
:107F000025513046F8F7EDFE01213046F8F7DDFE49
:107F100006B070BD70B586B0054601211020F7F798
:107F2000A4FF01212020F7F7A0FF01210805F7F7A2
:107F3000A7FF264E3046F8F705FEB014ADF8140042
:107F400003208DF8160018208DF8170005A9204889
:107F5000F0F76BFE0420ADF8140048208DF81700F0
:107F600005A91C48F0F761FE35208DF800000024BB
:107F70008DF801408DF8024001208DF8030068461D
:107F8000F0F7CFFB0195ADF808407014ADF80A008A
:107F9000ADF80C40ADF810400C20ADF80E0001A972
:107FA0003046F8F717FE012240F225513046F8F727
:107FB00098FE01213046F8F788FEA9E70038014015
:107FC0000008014000480040000C01400050004003
:107FD00000100140001401404FF0E0210A6922F036
:107FE00004020A61224AC00810704FF47A735843A1
:107FF000012353804861086940F00100086170471F
:108000002DE9F04100244FF0E0277E69054618482D
:1080100000784543FFF71FFEBA69B9699142FCD069
:1080200003D2A2EB0100044403E0A6EB01001044DC
:1080300004440A46AC42F0D3BDE8F041FFF713BE5A
:1080400070B50446FFF788FD60B1094D6888844229
:1080500003D3B4FBF0F0FFF762FB6888B4FBF0F1E8
:1080600000FB11444FF47A706043BDE87040C7E7ED
:1080700008030020F749FF200870F749087070478F
:10808000F64900200860F64948738875012240F2DD
:108090002551F448F8F725BE10B5F14CE07B801E61
:1080A000C1B2F14805F0F4FCEF49E27BE37B0A44FE
:1080B00012F8012C194411F8021C02EB0121814233
:1080C00001D1012010BD002010BD2DE9F047DFF8DF
:1080D000948340F225514046F8F7D0FEDFF88CA398
:1080E00001270026DFF88893DD4C012829D040F2D3
:1080F000277529464046F8F7C1FE012855D18AF870
:10810000077099F82B20032A01D0002A4DD1E28B69
:10811000608B824273D340214046F8F7A4FE0028CA
:10812000F9D040214046F8F7A5FE002229464046F6
:10813000F8F7D7FDE683FFF7A3FFBDE8F0470BF0A4
:10814000B6BD8AF8087099F82B1003290AD00029C7
:108150002BD14046F8F71EFEC1B2BDE8F047C54836
:108160000BF007BD607BC04DDC2807D24046F8F716
:1081700011FE617B4A1C6273685401E0FFF780FFC7
:10818000607B01280DD0607B042810D0607B07281D
:108190001CD0607BDFF8E0824FF00309062841D055
:1081A00043E05020E073607D2075BDE8F087E878FB
:1081B000A97800EB01200A28F7D168780628F4D1C5
:1081C0000C20E073607D08302075EEE768780328A6
:1081D00016D0062814D010281DD029785529E4D1AE
:1081E000FF28E2D1A8780128DFD168790028DCD106
:1081F000A8790028D9D1277005206070D5E767E0FD
:10820000E878A97800EB01200A28CED00820E07396
:10821000607D2075C9E7A87900F10901E173083094
:108220002075C2E76878192826D0607BE17B8842F8
:10823000BBD16878032803D0062801D01028B4D118
:108240002878DFF838A2FF2803D09AF80610884271
:108250003BD1FFF721FFA0B3A078012822D09AF8E4
:10826000D80030B18649C0EB0010800008808548F6
:108270000670267500201DE0208B002895D1607ABD
:10828000002892D0607BE073267584F81690002059
:1082900004E0295C08F80010401CC0B2E17B884271
:1082A000F7D382E7BDE8F047EAE6295C08F800105A
:1082B000401CC0B2E17B8842F7D384F81690277245
:1082C00073E7FFE7BDE8F047DAE6BDE8F047D7E639
:1082D000501CE0836C48815C4046F8F757FDBDE8D0
:1082E000F0470BF0E4BC70B5684D40F225512846CC
:1082F000F8F7C4FD664CB8B12846F8F74BFDC2B29A
:10830000B4F8000440F2FF31C0F30E0088420BD2F3
:10831000B4F80004B4F80034C0F30E01481C60F354
:108320000E03A4F80034625440F224412846F8F7C2
:10833000A5FD01280AD194F8010440F0800084F8DA
:1083400001042846BDE87040F8F724BD70BD2DE952
:10835000F041504E40F225513046F8F78FFD002491
:108360003F4D01281DD040F2277739463046F8F7B7
:1083700085FD012813D12A8CA88B824260D340212D
:108380003046F8F770FD0028F9D040213046F8F764
:1083900071FD002239463046F8F7A3FC2C84BDE875
:1083A000F0813046F8F7F6FCC0B2374A01230A3AAA
:1083B000FF2801D1697C19B1697C012907D00AE045
:1083C0006B74A87BFF26411CA973165407E086280E
:1083D00013D0792811D0022916D0AC736C74A87B05
:1083E0000928DCD30020401CC0B20828FBD35078F9
:1083F00086280ED0792813D01DE002216974A97B4C
:108400004E1CAE735054EAE7A97B4E1CAE73505419
:10841000E5E7D078917800EB01201F4908800AE059
:10842000E9791E48152901D10470EC71E979142904
:1084300001D10370EC711A480370AC736C74AEE731
:10844000501C28840648AA30815C3046BDE8F041C3
:10845000F8F79CBCD0030020D1030020A0012142EA
:108460000C03002000380140046500207211002038
:108470005016002088930020046700201C6D002007
:108480005C0000205A0000200E690020004C0040D3
:108490000E120020004800405E02002090020020E2
:1084A0003C020020FA49012008607047F9494883DE
:1084B000012240F22771F848F8F713BCF549888388
:1084C000012240F22771F548F8F70BBC10B5FFF711
:1084D000D7FDF0480A214175017510BD2DE9F0471F
:1084E000EF4DDFF8C09354184FF00108B0F5FA6F64
:1084F00036D02F4607F14A060A37A0F5E061D33996
:1085000017D0891C38D0091F39D0491C3DD0C91E4D
:1085100041D0C91E1F2949D8C8062FD1402138464D
:1085200011F06AFEE11D3846BDE8F047402211F027
:10853000ECBD6079012821D1FEF724FC40213846AA
:1085400011F05AFE2021304611F056FE7C21D4480D
:1085500011F052FE89F80580BDE8F04706F0FCBC3A
:10856000FEF710FC6079287089F8058006F0F4FCAD
:10857000BDE8F047F0F76CBD6079687015E660798A
:10858000217900EB0120A8800FE66079217900EBCA
:108590000120688009E66079012803D0BDE8F04732
:1085A000FEF71EBCBDE8F047FEF704BCA0F2FA716E
:1085B0000F290CD80807E1D12021304611F01CFE0C
:1085C000E11D3046BDE8F047202211F09EBDA0F528
:1085D00000610A39D2D1A0F60A000C2190FBF1F219
:1085E00001FB12000028C9D1207A05F86A0FA07A91
:1085F0006870207BA870A07BE870207C2871A07C2C
:108600006871207DA871A07DE871207E2872A07E0F
:108610006872207FA872A07FE872C6E52DE9FF5F2F
:108620000446DFF870A24FF001088AF802800029A2
:1086300002D0042900D0A41DE078A17800EB01202D
:1086400085B26178984F10291ED11FFA80F9A07960
:10865000182801D91820A071A9F2B310072814D83E
:1086600000260EE004EB060906F2911099F80710B7
:10867000F9F77EF8B91999F8070081F89101761C8D
:10868000F6B2A079B042EDD8E2E1A9F2BB100390B6
:108690003F2870D8002688E0039804EB060B06EB11
:1086A000400000F2A1109BF8071080B2F9F760F8C3
:1086B000A9F58070BF381CD0001F20D0001F24D027
:1086C000001F28D0001F2CD0001F30D0001F34D036
:1086D000001F38D0001F3CD0001F40D0001F44D0E6
:1086E000001F49D0001F4DD0001F51D0001F55D092
:1086F00059E0B9199BF8070081F8A90153E0B919AD
:108700009BF8070081F8B1014DE0B9199BF807000B
:1087100081F8B90147E0B9199BF8070081F8C10158
:1087200041E0B9199BF8070081F8C9013BE0B9198C
:108730009BF8070081F8D10135E0B9199BF80700D3
:1087400081F8D9012FE0B9199BF8070081F8E10100
:1087500029E0B9199BF8070081F8E90123E0B9196C
:108760009BF8070081F8F1011DE0B9199BF807009B
:1087700081F8F90117E01DE0B9199BF8070081F8AD
:10878000010210E0B9199BF8070081F809020AE01C
:10879000B9199BF8070081F8110204E0B9199BF898
:1087A000070081F81902761CF6B2A079B0423FF6B4
:1087B00073AF4DE1A9F2E120029013281CD80026E6
:1087C00013E0029804EB060B06EB400909F2813036
:1087D0009BF8071080B2F8F7CBFF09EB07019BF875
:1087E000070081F88103761CF6B2A079B042E8D880
:1087F0002E4880F802802BE1A9F2CB20092814D85A
:1088000000260EE004EB060906F5527099F80710F1
:10881000F8F7AEFFB91999F8070081F84803761CFC
:10882000F6B2A079B042EDD812E1A9F5CD700628D4
:108830000FD80A208AF80700207DA17CCDE900101E
:10884000207A237CA27BA17A00F5FA60F9F79BF8E5
:10885000FEE0A9F22D30DFF858B00B282AD8002608
:108860000EE004EB460906F2B53099F80810F8F767
:108870007FFFB91999F8080081F8B503761CF6B2A4
:10888000A079B6EB500FECD38BF80080E0E000004D
:10889000A00121420C0300200038014000480040A4
:1088A000902200204D0400201C6D00207211002039
:1088B00028000020A9F239300B2817D800260EE036
:1088C00004EB460906F2C13099F80810F8F750FF9A
:1088D000B91999F8080081F8C103761CF6B2A0799D
:1088E000B6EB500FECD38BF80080B1E0A9F2453025
:1088F0000B2817D800260EE004EB460906F2CD300F
:1089000099F80810F8F734FFB91999F8080081F8B8
:10891000CD03761CF6B2A079B6EB500FECD38BF8F2
:10892000008095E0A9F251300B2817D800260EE000
:1089300004EB460906F2D93099F80810F8F718FF49
:10894000B91999F8080081F8D903761CF6B2A07914
:10895000B6EB500FECD38BF8008079E0A9F25D30D4
:108960000B2817D800260EE004EB460906F2E53086
:1089700099F80810F8F7FCFEB91999F8080081F881
:10898000E503761CF6B2A079B6EB500FECD38BF86A
:1089900000805DE0A9F269300B2817D800260EE0B0
:1089A00004EB460906F2F13099F80810F8F7E0FEFA
:1089B000B91999F8080081F8F103761CF6B2A0798C
:1089C000B6EB500FECD38BF8008041E0A9F2753084
:1089D0000B2817D800260EE004EB460906F2FD30FE
:1089E00099F80810F8F7C4FEB91999F8080081F849
:1089F000FD03761CF6B2A079B6EB500FECD38BF8E2
:108A0000008025E0A9F281300B2817D800260EE05F
:108A100004EB460906F2094099F80810F8F7A8FE99
:108A2000B91999F8080081F80904761CF6B2A07902
:108A3000B6EB500FECD38BF8008009E0A9F5FA6093
:108A4000642805D80023224619464846FFF746FD0C
:108A5000607806287ED1EDB3022D7CD0DFF844B4D7
:108A60004FF00009062D77D0102D76D0082D75D047
:108A70000E2D74D0142D73D00A2D72D0162D71D0F6
:108A8000172D70D0A5F5407022386DD0401E6CD0E7
:108A9000652D6BD0672D6AD0682D69D0692D68D09F
:108AA0006A2D67D06B2D66D06C2D65D0DFF8F8B3DA
:108AB000FE486D2D73D00F2D72D06F2D71D0712D9A
:108AC00070D0DFF8ECB3722D6DD0732D6CD0742D97
:108AD0006BD000E074E0752D68D0782D67D0152D2F
:108AE0007DD0792D7CD0822DFCD04FF0080B7A2DD3
:108AF00077D07B2D76D07C2D75D07D2D74D07E2DBA
:108B000073D07F2D72D0802D71D0812D70D0A5F1C2
:108B1000830BBBF1070F6CD86079217900EB012042
:108B200086B20BF0FF01E348F2F74EF8002871D04F
:108B300007EB4B0595F86B0395F86A1300EB0120E2
:108B4000B04202F0E98640F26A3000EB4B00217936
:108B500080B212E0F8E35EE07BE0B2E0D0E0E3E078
:108B6000E9E0F9E029E12FE122E037E13EE150E1DF
:108B70005AE169E16FE175E17BE1F8F7F9FD40F257
:108B80006B3000EB4B00617980B2F8F7F1FD207992
:108B900085F86A03607985F86B0302F0BDBE6FE16A
:108BA000FFE108E214E21BE269E2BBE2EEE2FEE270
:108BB000617987F8271340F22730F8F7D9FDECE701
:108BC0009AF80A00C107E8D1617939702179797082
:108BD00040F001008AF80A00617900200AE004E30D
:108BE00030E387E394E3A1E3AFE3BCE3C9E3D6E377
:108BF000E3E3F0E3F8F7BCFD21790120F8F7B8FDD5
:108C00009AF80A104FF45A70F8F7B2FD0D208AF85E
:108C10000700C2E7E0E39AF80A008107BDD4617952
:108C2000B9702179F97040F002008AF80A00617980
:108C30000220F8F79DFD21790320F8F799FD9AF8B5
:108C40000A104FF45A70F8F793FD0E208AF80700C7
:108C5000A3E7607997F8CF1088429ED397F8D11098
:108C600088429AD89AF80B00012807D097F8F302A7
:108C700020B18AF80B808AF80C908EE787F8F3927F
:108C800040F2F32500212846F8F772FD61790620AD
:108C9000F8F76EFD6079ABF8000001228149864843
:108CA000EFF78DFC6079B87160798AF8100087F869
:108CB000F38201212846F8F75BFD0C208AF80700B3
:108CC000D9E76179F9728E2904D09F290DD07F29C7
:108CD00010D062E710208AF8070000214FF45A7084
:108CE000F8F746FD8AF80A9057E7F4F791FDF3F795
:108CF000F7FD52E70B20F8F73BFD8AF807804CE7B9
:108D00009AF80A00000784D4617939720820F8F7CC
:108D10002FFD9AF80A0040F008018AF80A104FF473
:108D20005A70F8F725FD38E7617987F8D710D72012
:108D3000F8F71EFD31E7207987F89702617987F807
:108D4000961240F29620F8F713FD97F8971240F22A
:108D50009720F8F70DFD20E7207955280CD06628DC
:108D600019D0772824D0607987F87701617940F2AB
:108D70007710F8F7FDFC10E76079B871617906208B
:108D8000F8F7F6FCB879ABF80000012245494A48EB
:108D9000EFF715FC01E7607938B1C0EB00108000F7
:108DA000AAF818008AF80980F7E68AF80990F4E62C
:108DB000AAF818908AF80980EFE66079012888D12E
:108DC00016208AF80700E8E6617901298CD93B482A
:108DD000017040F29C40F8F7CBFCDEE6617987F841
:108DE00028134FF44A70F8F7C3FCD6E6617987F888
:108DF000A91340F2A930F8F7BBFC87F86B9000216B
:108E00006B20F8F7B5FC2E4880F8058080F80380C9
:108E1000C3E6617987F86A106A20F8F7A9FC294946
:108E200097F86A000870B8E697F86E006179884292
:108E300091D087F86E106E20F8F79AFC204880F8E1
:108E40000080F2F7FEFEA8E6617987F86F106F20C8
:108E5000F8F78EFCA1E6617987F878107820F8F7AA
:108E600087FC9AE6617987F87A107A20F8F780FC17
:108E700093E6607901288DD102208AF807008CE6FC
:108E800097F89E1204295ED097F89F1204295AD0B1
:108E900061790E4ACB070C492FD081F80080797A8E
:108EA00016E00000500000204C0000202C000020A4
:108EB00096000020F06D0020007700084C04002090
:108EC00072110020770000203A0000206E00002080
:108ED00041F001017972F84B197839B997F86310AC
:108EE00021B1C1EB01118900CBF8001004211970E8
:108EF00087F89B100170117013E081F80090797A67
:108F000001F0FE017972EC4981F8009087F89B909E
:108F100080F80090E94880F80090CBF8009082F843
:108F20000090E74880F8028080F8048080F8018093
:108F3000797A0920F8F71CFCDF48017887F89B1044
:108F40009B20F8F715FC60798AF81300797A00F015
:108F5000040201F004039A420CD0400706D541F008
:108F6000040179720920F8F703FC03E0F2F7E4FB4F
:108F7000F3F7B6FC6079800607D5787A40F02000D8
:108F8000787204208AF8170006E0787A00F0DF0093
:108F9000787202208AF81700797A0920F8F7E8FB3E
:108FA000FBE5617987F865106520F8F7E1FB04209F
:108FB0008AF80700F1E5617987F863106320F8F714
:108FC000D7FB6079C0EB00108000CBF80000E4E52F
:108FD00061796B20F8F7CCFB607987F86B00DCE5F2
:108FE000207987F8CC00607987F8CB002179CC20F4
:108FF000F8F7BEFB6179CB20F8F7BAFB217909B904
:109000006079B8B397F8DB00012801D002280CD1B1
:10901000CE20F8F7ADFB207987F8CE006179CD201E
:10902000F8F7A6FB607987F8CD0097F8CD0097F8A0
:10903000CE1000EB012080B2ABF80000A14981F80E
:109040000090A14981F8008010B1A04981F800800A
:1090500097F8DB10032907D19C4981F800909C49BF
:1090600081F8008081F8018097F8D3100122F4F78D
:10907000DDFF92E5FFE7954880F800908DE52079C7
:1090800087F8CE00607987F8CD002179CE20F8F7F7
:109090006FFB6179CD20F8F76BFB217909B9607915
:1090A000D8B397F8DB00012801D002280CD1CC20DE
:1090B000F8F75EFB207987F8CC006179CB20F8F7D0
:1090C00057FB607987F8CB00CC377878B97800EB1C
:1090D000012080B2ABF800007A4981F800907A490B
:1090E00081F8008017F8CC1911B997F8CB1011B19D
:1090F000764981F8008097F8DB10032907D173497E
:1091000081F80090724981F8008081F8018097F819
:10911000D3100122F4F78AFF3FE5FFE76B4880F8A0
:1091200000903AE5617987F8DB1097F8CC0010B928
:1091300097F8CB0058B197F8CE0010B997F8CD202A
:109140002AB1032907D0614981F800800BE05F480C
:1091500080F8009021E55D4981F800905C4981F834
:10916000008081F80180584981F80080554981F8D4
:10917000009097F8CD1001EB002080B2ABF8000012
:1091800097F8D3100122F4F751FF06E5617987F8CB
:10919000D810D820F8F7ECFA97F8D8004D49C0EB72
:1091A0000010800008804C4880F80090F5E4607959
:1091B00001280BD0022810D000218220F8F7D8FA1D
:1091C00087F8829009208AF80700E6E401218220CE
:1091D000F8F7CEFA87F88280F4E702218220F8F7C8
:1091E000C7FA022087F88200ECE760793B4D01283E
:1091F00018D10B208AF807009AF8030090B985F877
:109200002B9087F8928001219220F8F7B1FA002183
:10921000D620F8F7ADFA87F8D69005F0E5FD0020E6
:109220000AF01EFD6079002894D1032085F82B00F8
:1092300087F8929004208AF8070000219220F8F71E
:1092400097FAAAE400212648F1F7BEFC30B1207954
:1092500087F87A03607987F87B039EE42079617947
:1092600001EB002081B297F85F00022804D0132898
:1092700002D0042816D090E41A481B4C0088081A23
:109280002080C1B25B20F8F773FA2088C0F3072171
:109290005C20F8F76DFA208887F85B00000A87F8F1
:1092A0005C007AE411480078081A11490870C1B2CC
:1092B0005D20F8F75DFA70E43B000020D800002044
:1092C000721100208C000020D90000207E000020B8
:1092D000AD0000205C0000205A0000205016002045
:1092E000F16D00207E02002068020020760200203E
:1092F000400200206179E520F8F73AFA607987F8B2
:10930000E500FE4880F800B0FD4880F800B044E475
:109310006179E620F8F72CFA607987F8E600F748DB
:1093200080F800B0F64880F800B036E46179E720B4
:10933000F8F71EFA607987F8E700F04880F800B087
:10934000EF4880F800B028E4EDE36179E820F8F711
:109350000FFA607987F8E800E84880F800B0E8483C
:1093600080F800B019E46179E920F8F701FA607932
:1093700087F8E900E14880F800B0E14880F800B0E3
:109380000BE46179EA20F8F7F3F9607987F8EA00ED
:10939000DA4880F800B0DA4880F800B00FE461796C
:1093A000EB20F8F7E5F9607987F8EB00D34880F80F
:1093B00000B0D34880F800B02BE46179EC20F8F7D6
:1093C000D7F9607987F8EC00CC4880F800B0CC4839
:1093D00080F800B01DE418E0CA48CB4C30F81B0000
:1093E000301A24F81B00C1B2472000EB4B0080B2BA
:1093F000F8F7BEF934F81B00C0F30721482000EB52
:109400004B0080B2F8F7B4F922E44FF481728B2D4F
:1094100014D08C2D26D08D2D3AD08E2D3FD0A5F195
:109420008F01092943D805F16800617980B2F8F706
:109430009FF97919607981F8680009E460792179E8
:1094400000EB0120B149B24C0988401A2080C0F3DA
:1094500007211046F8F78CF9217840F20110F8F74F
:1094600087F90AE46079217900EB0120A949AA4C27
:109470000988401A2080C1B240F27D30F8F778F9AF
:109480002088C0F3072140F27E30F8F771F920E41C
:10949000617987F8D410D420F8F76AF919E4607973
:1094A00087F8600061796020F8F762F911E4992D7E
:1094B00022D09A2D28D09B2D3AD09C2D4CD09D2D7A
:1094C0005ED09E2D76D09F2D6FD0A02D6ED0A12D79
:1094D0006DD0A22D6CD06CD1207987F856006079C0
:1094E00087F8550061794FF05100F8F741F921797B
:1094F0005220F8F73DF916E4884960790870C1B246
:109500005D20F8F735F90EE4257961795B377D70D8
:1095100039705B20F8F72CF929465C20F8F728F918
:10952000397878785B3FF1F7C1FB7D49088012E418
:109530002579617947377D7039704720F8F718F938
:1095400029464820F8F714F938787978473F00EB36
:1095500001206D4908800EE42579617949377D70D5
:1095600039704920F8F704F929464A20F8F700F93C
:1095700038787978493F40EA01206349488009E416
:10958000257961794B377D7039704B20F8F7F0F809
:1095900029464C20F8F7ECF8387879784B3F40EAC8
:1095A00001215948818007E404E017E02BE03FE007
:1095B00053E067E0257961794D377D7039704D2032
:1095C000F8F7D6F829464E20F8F7D2F838787978A7
:1095D0004D3F40EA01204C49C88006E44F372079CE
:1095E00078706079387061794F20F8F7C1F8217987
:1095F0005020F8F7BDF8387879784F3F40EA0120DD
:109600004149088104E451372079787060793870D5
:1096100061795120F8F7ACF821795220F8F7A8F8D1
:1096200038787978513F40EA0120374948810AE487
:109630005337207978706079387061795320F8F762
:1096400097F821795420F8F793F838787978533FD0
:1096500040EA01202C4988810AE455372079787046
:109660006079387061795520F8F782F821795620B1
:10967000F8F77EF838787978553F40EA012022499A
:10968000C8818DE4A72D68D0A82D76D0A92D6ED0E5
:10969000AA2D6DD0AB2D6CD0AC2D6BD0AD2D6AD07A
:1096A000AE2D69D0DFF87CB0AF2D6FD0B02D6ED06D
:1096B000B12D6DD0B22D6CD0B32D6BD0B42D6AD03E
:1096C000B52D69D0B62D68D0B72D67D0B82D6FD025
:1096D000B92D6ED0BA2D6DD0BB2D6CD0BC2D6BD0FA
:1096E000BD2D6AD0BE2D69D0BF2D68D0C02D67D0EA
:1096F000C12D6FD0C22D6ED0C32D15E049020020C0
:109700004A020020DC110020B81100205E02002077
:10971000740200206C000020400000204002002065
:10972000680200207802002071D0C42D70D0A5F10D
:10973000CA0104296DD8A5F11100617980B2F8F74A
:1097400017F87919607901F8110C6179F648491E0A
:1097500002297DD280F8008022E4607987F89E0299
:10976000617940F29E20F8F703F819E405E016E06D
:1097700027E031E039E041E04CE0607987F89F0272
:10978000617940F29F20F7F7F3FF09E44BE068E0CE
:1097900074E081E08FE09DE0ABE0B9E0C7E0607984
:1097A00087F8A00261794FF42870F7F7E1FF0EE423
:1097B000CCE0DAE0F6E012E120E12EE13CE14AE122
:1097C00058E1607987F8A102617940F2A120F7F7AA
:1097D000CFFF04E45DE16BE1607987F8A202617973
:1097E00040F2A220F7F7C4FF43E4607987F8A302B0
:1097F000617940F2A320F7F7BBFF3AE4607987F87C
:10980000A40261794FF42970F7F7B2FF31E45EE109
:109810006CE18EE1607987F8A502617940F2A520BC
:10982000F7F7A6FF25E46079F87620793877617933
:109830001B20F7F79DFF21791C20F7F799FFF87E91
:10984000397F00EB012197F82F0000EB002000E0AA
:109850006CE1814202D28BF800800AE48BF8009020
:1098600007E4607978772079B87761791D20F7F778
:109870007FFF21791E20F7F77BFF4DE46079F877B1
:10988000207987F8200061791F20F7F771FF21798F
:109890002020F7F76DFF3FE4607987F821002079F9
:1098A00087F8220061792120F7F762FF21792220D1
:1098B000F7F75EFF30E4607987F82300207987F8B6
:1098C000240061792320F7F753FF21792420F7F74B
:1098D0004FFF21E4607987F82500207987F826007A
:1098E00061792520F7F744FF21792620F7F740FF1B
:1098F00012E4607987F82700207987F828006179D9
:109900002720F7F735FF21792820F7F731FF08E402
:10991000607987F82900207987F82A006179292061
:10992000F7F726FF21792A20F7F722FF12E4607962
:1099300087F82B00207987F82C0061792B20F7F726
:1099400017FF21792C20F7F713FF1EE4607987F8C1
:109950002D00207987F82E0061792D20F7F708FF78
:1099600021792E20F7F704FF0FE41B376079387553
:109970002079787561792F20F7F7FAFE2179302068
:10998000F7F7F6FE3878797800EB0121387D1B3F38
:1099900000EB0020814202D28BF8008006E48BF8B5
:1099A000009012E4607907F8310F207978706179BE
:1099B0003120F7F7DDFE21793220F7F7D9FE38782C
:1099C000797800EB0121387D313F00EB00208142A6
:1099D00002D28BF8018034E48BF8019031E4607995
:1099E00087F83300207987F8340061793320F7F75E
:1099F000BFFE21793420F7F7BBFE22E4607987F8B7
:109A00003500207987F8360061793520F7F7B0FE08
:109A100021793620F7F7ACFE13E4607987F8370038
:109A2000207987F8380061793720F7F7A1FE21798E
:109A30003820F7F79DFE04E4607987F83900207933
:109A400087F83A0061793920F7F792FE21793A20B8
:109A5000F7F78EFE0FE4607987F83B00207987F8EE
:109A60003C0061793B20F7F783FE21793C20F7F732
:109A70007FFE16E4607987F83D00207987F83E0084
:109A800061793D20F7F774FE21793E20F7F770FEEB
:109A900007E4607987F83F00207987F84000617912
:109AA0003F20F7F765FE21794020F7F761FE2EE4AD
:109AB000607987F84100207987F842006179412078
:109AC000F7F756FE21794220F7F752FE1FE460793E
:109AD00087F84300207987F8440061794320F7F73D
:109AE00047FE21794420F7F743FE10E431376079CF
:109AF00038752079787561794520F7F739FE217935
:109B00004620F7F735FE3878797800EB0121387D6B
:109B1000313F00EB0020814202D28BF8018004E447
:109B20008BF801900FE4EFE37800002080F80090BC
:109B300009E4CF2D18D0D02D1ED040F2663BD12D98
:109B400022D0F74BD22D2BD0D32D4CD0A5F1D5015F
:109B5000062968D87919607981F86D006D356179C9
:109B6000A8B2F7F705FE0BE4607987F87B0061790E
:109B70007B20F7F7FDFD11E4607987F87C006179BF
:109B80007C20F7F7F5FD09E497F8660361798842D0
:109B90008DD05846F7F7ECFD607987F866030BE443
:109BA00005211846F1F710F800288FD0207987F8A2
:109BB0006203607987F86303217940F26230F7F736
:109BC000D7FD617940F26330F7F7D2FD60792179F2
:109BD00000EB012082B20221D248FBF736F9D248CD
:109BE00080F8008010E406211846F0F7EDFF002809
:109BF00095D0207987F86403607987F86503217927
